:020000040800F2
:1000000000040020A51F0008F71F0008F71F0008C4
:10001000F71F0008F71F0008F71F00080000000086
:10002000000000000000000000000000F71F0008B2
:10003000F71F000800000000F71F0008D91402088D
:100040006516020867160208691602086D1602088E
:100050008D1602088F16020891160208B5160208BE
:10006000D9160208FD1602082117020845170208D2
:1000700047170208491702084B1702084D170208D4
:100080004F1702085117020853170208F71F0008FC
:10009000F71F0008F71F0008F71F00085517020890
:1000A000A1170208A3170208A5170208A71702083C
:1000B000A9170208AD170208D91702084918020843
:1000C0004B1802084D1802084F1802085118020870
:1000D00055180208C5190208ED180208891A020805
:1000E0004D1B0208111C0208131C0208151C0208F3
:1000F000191C0208811C0208831C0208851C0208C6
:10010000871C0208891C02088B1C02088D1C02082F
:10011000911C0208651D0208671D0208691D02087E
:10012000751E0208771E0208791E02087B1E02084F
:1001300000000000000000000000000000000000BF
:1001400000000000000000000000000000000000AF
:10015000000000000000000000000000000000009F
:10016000000000000000000000000000000000008F
:10017000000000000000000000000000000000007F
:10018000000000000000000000000000000000006F
:10019000000000000000000000000000000000005F
:1001A000000000000000000000000000000000004F
:1001B000000000000000000000000000000000003F
:1001C000000000000000000000000000000000002F
:1001D000000000000000000000000000000000001F
:0401E0005FF8E0F1F3
:1001E800032A70B404460D4626D941EA000313F0E9
:1001F800030F13D020782B78984208BF294606D0E1
:100208001EE014F8010F11F8013F984218D1012A95
:1002180002F1FF32F5D1002070BC70470B4604464E
:1002280051F8045B50F8046BAE4204D1043A04461A
:10023800032A0B46F2D81D461046002ADAD1EBE70E
:10024800C01AE9E7032A2DE9F00109D82AB10023E9
:10025800CC5CC45401339342FAD1BDE8F001704735
:100268000B468218014603E02478013301F8014B5C
:1002780011F0030F1C46F7D113F003055DD06E4251
:10028800C5F1040CED009B594FEACC0C08E004348E
:10029800A7593B4607FA0CF748EA070741F8047BD9
:1002A800571A23FA05F8032FF1DC03E014F8013B91
:1002B80001F8013B8A42F9D8CFE753F8404C41F89E
:1002C800404C53F83C4C41F83C4C53F8384C41F8FE
:1002D800384C53F8344C41F8344C53F8304C41F80E
:1002E800304C53F82C4C41F82C4C53F8284C41F81E
:1002F800284C53F8244C41F8244C53F8204C41F82E
:10030800204C53F81C4C41F81C4C53F8184C41F83D
:10031800184C53F8144C41F8144C53F8104C41F84D
:10032800104C53F80C4C41F80C4C53F8084C41F85D
:10033800084C53F8044C41F8044C561A1D460C4618
:10034800403340313F2EB8DC2B460FE053F8101CE9
:1003580044F8101C53F80C1C44F80C1C53F8081CE7
:1003680044F8081C53F8041C44F8041C161B2146C6
:100378001D46103410330F2EE8DC2B4602E02468AB
:1003880041F8044B551A1C46032D03F10403F6DC0F
:1003980090E700BF032AC9B270B408D82AB103464F
:1003A800121803F8011B9342FBD170BC70478218E6
:1003B800044601E004F8011B14F0030FFAD14FF0D2
:1003C800013303FB01F31FE044F8403C44F83C3C94
:1003D80044F8383C44F8343C44F8303C44F82C3C6D
:1003E80044F8283C44F8243C44F8203C44F81C3C9D
:1003F80044F8183C44F8143C44F8103C44F80C3CCD
:1004080044F8083C44F8043C161B254640343F2E6B
:10041800DADC2C4607E044F8103C44F80C3C44F87D
:10042800083C44F8043C161B254610340F2EF2DC19
:1004380001E045F8043B541B032CFADC01E005F805
:10044800011B9542FBD3B0E710F0030F38B5044603
:1004580012D10368A3F1013222EA030313F0803FAB
:100468000AD1031D184653F8042BA2F1013525EAD9
:10047800020212F0803FF5D003782BB1431C1846D6
:1004880013F8012B002AFAD100F076F9204638BD7E
:10049800C9B2F0B4002950D010F0030F10D003787F
:1004A800002B79D0994246D0431C05E013F8012B64
:1004B800002A3FD091423ED013F0030F1846F5D1E1
:1004C800036841EA01270646A3F1013247EA0747D4
:1004D80022EA030212F0803F1DD187EA0303A3F149
:1004E800013222EA030313F0803F14D1043002E002
:1004F80012F0803F0FD1064650F8043BA3F10135B6
:1005080087EA030225EA0303A2F1013413F0803FCE
:1005180024EA0202ECD033783046002B3CD09942D2
:1005280009D0731C01E0914205D0184613F8012B3D
:10053800002AF8D11046F0BC704710F0030F0CD019
:100548000378002BF7D0431C03E013F8012B002A93
:10055800F1D013F0030F1846F7D102680346A2F151
:10056800013121EA020212F0803F0AD10430034629
:1005780050F8042BA2F1013121EA020212F0803F67
:10058800F5D01A781846002AD5D00133184613F842
:10059800012B002AFAD1CEE71846CCE780EA0102FF
:1005A80012F0030F3AD110F0030220F0030021F0FB
:1005B800030150F804CB08BF51F8043B0DD082F07A
:1005C80003024FEAC2026FF07F4323FA02F251F8A6
:1005D800043B4CEA020C43EA020300BFACF10132CF
:1005E8009C4501BF22EA0C0212F0803F50F804CB70
:1005F80051F8043BF2D04FEA0C604FEA1C2C01285A
:1006080028BFB0EB036F08BF1B0AF4D003F0FF0349
:100618004FEA1060A0EB0300704700BF10F0030F13
:100628000AD010F8012B11F8013B012A28BF9A4281
:10063800F4D0A2EB030070474DF8045D4DF8044D6B
:100648004FF0010242EA022242EA024201F0030CA0
:1006580021F0030150F8044B51F8045BBCF1020F80
:1006680026D04BD824F07F4CBCEB152FA4EB02030B
:1006780023EA04030DD113EAC21308BF51F8045B3F
:100688000AD18CEA040CBCEB056F0CD150F8044B72
:10069800E8E74FEA15255CE033F07F4352D10D7847
:1006A8004FEA146C55E04FEA146C05F0FF0550E072
:1006B8004FEA044CA4EB02034FEA1C4C23EA040360
:1006C800BCEB154F17D113EAC21308BF51F8045BEE
:1006D80007D18CEA040CBCEB054F08D150F8044B49
:1006E800E6E71B042ED10D884FEA144C31E04FEA9F
:1006F80005454FEA144C4FEA15452AE004F0FF0C73
:10070800BCEB156FA4EB020323EA04030DD113EA33
:10071800C21308BF51F8045B0AD18CEA040CBCEB85
:10072800052F0AD150F8044BE8E74FEA156510E0A9
:1007380014F0FF0F06D051F8045B4FEA142C25F093
:100748007F4506E04FF000005DF8044B5DF8045B60
:1007580070470CF0FF0205F0FF00012828BF904207
:1007680004BF4FEA1C2C2D0AF3D0A2EB00005DF861
:10077800044B5DF8045B704780EA0102844612F07E
:10078800030F4FD111F0030F32D14DF8044D11F082
:10079800040F51F8043B0BD0A3F101329A4312F035
:1007A800803F04BF4CF8043B51F8043B16D100BF0E
:1007B80051F8044BA3F101329A4312F0803FA4F19F
:1007C80001320BD14CF8043BA24312F0803F04BF26
:1007D80051F8043B4CF8044BEAD023460CF8013B93
:1007E80013F0FF0F4FEA3323F8D15DF8044B70473D
:1007F80011F0010F06D011F8012B0CF8012B002A7B
:1008080008BF704711F0020FBFD031F8022B12F069
:10081800FF0F16BF2CF8022B8CF8002012F47F4F24
:10082800B3D1704711F8012B0CF8012B002AF9D12C
:10083800704700BF20F0030110F00300C0F1000072
:1008480051F8043B00F1040C4FEACC0C6FF00002A5
:100858001CBF22FA0CF213434FF0010C4CEA0C2C8B
:100868004CEA0C4CA3EB0C0222EA030212EACC126B
:1008780004BF51F8043B0430F4D013F0FF0F1FBF3E
:10088800013013F47F4F013013F47F0F18BF01308C
:10089800704700BFF0B4002A46D041EA000313F0C5
:1008A80003032CD1032A07460E4643D904680D6872
:1008B800AC423FD1043A37D0A4F1013525EA04040B
:1008C80014F0803F18BF18462CD1041D0D1D0EE0F2
:1008D80054F8043B55F8041BA3F101308B4220EA7D
:1008E800030027D1043A1FD010F0803F1ED1032AFD
:1008F80027462E46ECD820462946002A1DD00478E3
:10090800013A0D78AC420CD172B18CB1002302E0EF
:1009180093420BD064B1013310F8014FCD5CAC4267
:10092800F6D0601BF0BC70471046FBE70020F9E7E3
:100938002046F7E738463146E1E724782D78F0E796
:1009480041EA000313F0030F0B4670B414BF0024F0
:100958000124032A94BF002404F001040546D4B9F5
:10096800BAB10E782B46013A03F8016B56B1AC1CAC
:100978007AB111F8015F2346013A04F8015C0134A9
:10098800002DF5D12AB19A18002103F8011B9342D2
:10099800FBD170BC7047194653F8044BA4F10136DB
:1009A80026EA040616F0803FDAD1043A45F8044BEB
:1009B800032A1946EFD8D3E701232DE9F0071D468E
:1009C80000264FF0FF37AC1900EB070C8C420DD214
:1009D8001CF805C010F80480E0452ED201252646F3
:1009E800E31BAC198C4200EB070CF1D34FF0010963
:1009F80000264D464FF0FF3C1360AC1900EB0C0885
:100A0800A1420ED918F8058010F804A0C2451AD9D9
:100A180001252646CCEB0409AC19A14200EB0C08D1
:100A2800F0D80CF101000137B8423CBF994638466E
:100A3800C2F80090BDE8F00770470BD00123374695
:100A48001D46F618BFE709D04FF00109B4464D46D8
:100A58004E44D2E79D4205D00135B4E74D4505D057
:100A68000135CAE72B4626460125ACE7A9462646A6
:100A78000125C2E72DE9F04FADF5826D81B014462E
:100A8800074610460DF580628B460C3219461D4606
:100A9800FFF792FF03AE04A901F57E72331F0090A1
:100AA80043F8045F9342FBD14DB1681E0023E25C1A
:100AB800C11A013303AEAB4246F82210F7D1DDF874
:100AC8000C142046009A6118FFF78AFB002877D19A
:100AD8000099814605F1FF380646C1F101020192ED
:100AE8005A46AB4609EB0B0501F1FF3AB81800214D
:100AF800AA1A00F0E5F900284FD1002D00F0C080B7
:100B08007B1903A913F8013C51F82330002B4CD171
:100B1800009B9E4228BF334698450FD903EB090135
:100B2800E05C7A18795C884205D038E012F8011F39
:100B3800E05C884233D101339845F7D8009A964251
:100B480080F0A48007EB090214F80A10534612F843
:100B58000A20914204BF0AEB0901791807D095E0F1
:100B680014F802C011F8010D844503D113465A1E2A
:100B7800B342F5D101369E4200F28D80DDF80C6457
:100B88002A46B144C6EB0B0609EB0B05B818002141
:100B9800AA1A00F095F90028AFD0002071E0019A58
:100BA8000026914499442A46EEE7002EFAD0DDF853
:100BB8000C2493423CBFC2EB0B0306469944F2E770
:100BC800009E4FF000080099AB1BB34238BF334674
:100BD800C1F101026E1E019201F1FF3A5A4689469F
:100BE800AB460133CDF80C3408EB0B05B8180021DF
:100BF800AA1A00F065F90028CFD1002D40D07B1942
:100C080003A913F8013C51F82330002B30D1B1452A
:100C180013D208EB090314F80910FA18FB5C99427F
:100C280018BF4B4627D14B4604E012F8011FE05C81
:100C3800884220D10133B342F7D3BAF1FF3F53467C
:100C48002CD007EB080C14F80A101CF80A20914263
:100C58000CD10AEB0802BA1804E0E05C12F8011D96
:100C6800884203D1013BF8D260460AE0DDF80C3433
:100C780098442A46B8E701992A4688449844B3E735
:100C8800284605B00DF5806DBDE8F08F009B013654
:100C98009E427FF673AF07EB0900F2E707EB080CFB
:100CA8006046EEE72DE9F04F8346037885B00C46A1
:100CB800002B00F0F9800A78A2B106460131012024
:100CC80002E011F8012B8AB1934214BF002000F012
:100CD800010016F8013F0D46002BF2D12B782BB1FD
:100CE8004FF0000B584605B0BDE8F08F0028F9D149
:100CF8000BF101002178FFF7CBFB2D1BA5F10102B9
:100D0800534243EB0203002808BF43F001030746A0
:100D180083B90BEB0508404594BFC0EB08084FF0BA
:100D280001081F2D08D9414622462B46FFF7A2FE8F
:100D38008346D7E78346D5E7294603AA2046FFF727
:100D48003BFE03996118814620464A46FFF748FA58
:100D580000284FD109F1FF33C9F10102064601927B
:100D680082464246C84699460AEB050BB818002148
:100D7800C2EB0B0200F0A4F80028B1D1BBF1000FC0
:100D8800B0D046452CBF334643469D420FD903EBAE
:100D98000A01E05C7A18795C884205D075E012F89F
:100DA800011FE05C884270D101339D42F7D1B04504
:100DB8007DD907EB0A0214F809104B4612F80920EE
:100DC800914202BF09EB0A01AC46791806D06EE0E1
:100DD800A55C11F8010D854203D113465A1EB34292
:100DE800F6D1654601369E4267D8039E5A46B244FC
:100DF800AE1BB9E7C9F10101C9EB0503424600265C
:100E080009F1FF3A88464B4538BF4B4601330393F7
:100E180006EB050BB8180021C2EB0B0200F050F8E6
:100E280000287FF45DAFBBF1000F3FF45BAF4D4589
:100E380012D906EB090314F80910FA18FB5C994259
:100E480008BF4B4605D026E012F8011FE05C884237
:100E580022D101339D42F7D1BAF1FF3F534628D042
:100E680007EB060C14F80A101CF80A20914217D157
:100E78000AEB0602BA1804E0E05C12F8011D884289
:100E88000ED1013BF8D2E3462CE7019A00269244A2
:100E98005A469A4468E74B4646445A46F618B7E716
:100EA800039B5A46F618B3E70D46012016E743465A
:100EB80098E707EB060CE34614E707EB0A0B11E784
:100EC80010F0030F034670B4C9B211D0002A22D023
:100ED80003788B421DD0013A013005E0DAB110F8F1
:100EE800014B013A8C4218D010F0030F0346F5D19C
:100EF800032A14D87AB1187888420ED0541E5D1C83
:100F080003E015F8016B8E4203D0013C2846F8D265
:100F1800002070BC70471046FBE71846F9E741EA25
:100F2800012646EA0646184653F8044B86EA0404A6
:100F3800A4F1013525EA040414F0803F03D1043AF2
:100F48001846032AEFD80346D4E700BF0000000084
:100F5800C1F30A5C0246ACF57E7C2DE9F84FACF192
:100F68000704132C0B4606460F468946804627DCA5
:100F7800002C52DB4FF6FF7CC0F20F0C4CFA04FA3F
:100F88000AEA0105054317D037A3D3E9002300F087
:100F980075F80022002300F0B3FC002856D0002F7B
:100FA80005DD4FF4801353FA04F407EB040929EA2A
:100FB8000A0900264B46324610461946BDE8F88F06
:100FC800332C07DDB4F5806FF6D100F057F80246F0
:100FD8000B46F1E74FF0FF3BACF11B0C2BFA0CFB77
:100FE8001BEA000FE8D020A3D3E9002300F046F85D
:100FF8000022002300F084FC40B3002F0ADD142CEB
:1010080006D00126C4F13404A64016EB080601D325
:1010180007F1010926EA0B0619E013A3D3E9002317
:1010280000F02CF80022002300F06AFC78B1002FB1
:1010380013DB46EA07054FF000094D45C3F6F07982
:101048000CBF2E46002608BFA94600E0B9464B460D
:10105800324610461946BDE8F88F00264FF0004981
:10106800F5E700BFAFF300809C7500883CE4377E4D
:1010780081F0004102E000BF83F0004330B54FEA41
:1010880041044FEA430594EA050F08BF90EA020FAE
:101098001FBF54EA000C55EA020C7FEA645C7FEA41
:1010A800655C00F0E2804FEA5454D4EB5555B8BF64
:1010B8006D420CDD2C4480EA020281EA030382EAD5
:1010C800000083EA010180EA020281EA0303362D67
:1010D80088BF30BD11F0004F4FEA01314FF4801C3A
:1010E8004CEA113102D0404261EB410113F0004F4C
:1010F8004FEA03334CEA133302D0524263EB430303
:1011080094EA050F00F0A780A4F10104D5F1200EA0
:101118000DDB02FA0EFC22FA05F2801841F10001FB
:1011280003FA0EF2801843FA05F359410EE0A5F1CF
:1011380020050EF1200E012A03FA0EFC28BF4CF000
:10114800020C43FA05F3C01851EBE37101F00045B6
:1011580007D54FF0000EDCF1000C7EEB00006EEBC3
:101168000101B1F5801F1BD3B1F5001F0CD349084D
:101178005FEA30004FEA3C0C04F101044FEA4452A4
:1011880012F5800F80F09A80BCF1004F08BF5FEA2B
:10119800500C50F1000041EB045141EA050130BD0B
:1011A8005FEA4C0C404141EB010111F4801FA4F1AE
:1011B8000104E9D191F0000F04BF01460020B1FA03
:1011C80081F308BF2033A3F10B03B3F120020CDA3B
:1011D8000C3208DD02F1140CC2F10C0201FA0CF019
:1011E80021FA02F10CE002F11402D8BFC2F1200C7E
:1011F80001FA02F120FA0CFCDCBF41EA0C01904034
:10120800E41AA2BF01EB0451294330BD6FEA04047C
:101218001F3C1CDA0C340EDC04F11404C4F1200267
:1012280020FA04F001FA02F340EA030021FA04F379
:1012380045EA030130BDC4F10C04C4F1200220FAD0
:1012480002F001FA04F340EA0300294630BD21FA0E
:1012580004F0294630BD94F0000F83F4801306BFD4
:1012680081F480110134013D4EE77FEA645C18BFC8
:101278007FEA655C29D094EA050F08BF90EA020F5F
:1012880005D054EA000C04BF1946104630BD91EA57
:10129800030F1EBF0021002030BD5FEA545C05D15A
:1012A8004000494128BF41F0004130BD14F5800499
:1012B8003CBF01F5801130BD01F0004545F0FE410D
:1012C80041F470014FF0000030BD7FEA645C1ABF42
:1012D800194610467FEA655C1CBF0B46024650EA79
:1012E800013406BF52EA033591EA030F41F40021A5
:1012F80030BD00BF90F0000F04BF0021704730B52B
:101308004FF4806404F132044FF000054FF00001FF
:1013180050E700BF90F0000F04BF0021704730B5C0
:101328004FF4806404F1320410F0004548BF404295
:101338004FF000013EE700BF42004FEAE2014FEAEA
:1013480031014FEA02701FBF12F07F4393F07F4FC5
:1013580081F06051704792F0000F14BF93F07F4FF7
:10136800704730B54FF4607401F0004521F000413A
:1013780020E700BF50EA010208BF704730B54FF0C0
:1013880000050AE050EA010208BF704730B511F0C5
:10139800004502D5404261EB41014FF4806404F1FD
:1013A80032045FEA915C3FF4DCAE4FF003025FEA7F
:1013B800DC0C18BF03325FEADC0C18BF033202EB07
:1013C800DC02C2F1200300FA03FC20FA02F001FA61
:1013D80003FE40EA0E0021FA02F11444C1E600BF00
:1013E80070B54FF0FF0C4CF4E06C1CEA11541DBFB3
:1013F8001CEA135594EA0C0F95EA0C0F00F0DEF87E
:101408002C4481EA030621EA4C5123EA4C5350EA62
:10141800013518BF52EA033541F4801143F48013B3
:1014280038D0A0FB02CE4FF00005E1FB02E506F044
:101438000042E0FB03E54FF00006E1FB03569CF099
:10144800000F18BF4EF0010EA4F1FF04B6F5007F9F
:1014580064F5407404D25FEA4E0E6D4146EB060611
:1014680042EAC62141EA55514FEAC52040EA5E509A
:101478004FEACE2EB4F1FD0C88BFBCF5E06F1ED844
:10148800BEF1004F08BF5FEA500E50F1000041EB7B
:10149800045170BD06F0004646EA010140EA020028
:1014A80081EA0301B4EB5C04C2BFD4EB0C0541EA4A
:1014B800045170BD41F480114FF0000E013C00F35F
:1014C800AB8014F1360FDEBF002001F0004170BD83
:1014D800C4F10004203C35DA0C341BDC04F114049C
:1014E800C4F1200500FA05F320FA04F001FA05F228
:1014F80040EA020001F0004221F0004110EBD370F5
:1015080021FA04F642EB06015EEA430E08BF20EA20
:10151800D37070BDC4F10C04C4F1200500FA04F3C3
:1015280020FA05F001FA04F240EA020001F0004155
:1015380010EBD37041F100015EEA430E08BF20EAC8
:10154800D37070BDC4F1200500FA05F24EEA020E10
:1015580020FA04F301FA05F243EA020321FA04F03F
:1015680001F0004121FA04F220EA020000EBD370F6
:101578005EEA430E08BF20EAD37070BD94F0000FF6
:101588000FD101F00046400041EB010111F4801F2A
:1015980008BF013CF7D041EA060195F0000F18BFDB
:1015A800704703F00046520043EB030313F4801F17
:1015B80008BF013DF7D043EA0603704794EA0C0FD1
:1015C8000CEA135518BF95EA0C0F0CD050EA4106E7
:1015D80018BF52EA4306D1D181EA030101F0004164
:1015E8004FF0000070BD50EA410606BF104619468C
:1015F80052EA430619D094EA0C0F02D150EA013698
:1016080013D195EA0C0F05D152EA03361CBF1046D8
:1016180019460AD181EA030101F0004141F0FE4177
:1016280041F470014FF0000070BD41F0FE4141F4FB
:10163800780170BD70B54FF0FF0C4CF4E06C1CEAFB
:1016480011541DBF1CEA135594EA0C0F95EA0C0FB0
:1016580000F0A7F8A4EB050481EA030E52EA03356B
:101668004FEA013100F088804FEA03334FF080558C
:1016780045EA131343EA12634FEA022245EA1115B9
:1016880045EA10654FEA00260EF000419D4208BF6A
:10169800964244F1FD0404F5407402D25B084FEA17
:1016A8003202B61A65EB03055B084FEA32024FF4C3
:1016B80080104FF4002CB6EB020E75EB030E22BF20
:1016C800B61A754640EA0C005B084FEA3202B6EBE0
:1016D800020E75EB030E22BFB61A754640EA5C008F
:1016E8005B084FEA3202B6EB020E75EB030E22BF1F
:1016F800B61A754640EA9C005B084FEA3202B6EB20
:10170800020E75EB030E22BFB61A754640EADC00DE
:1017180055EA060E18D04FEA051545EA16754FEA40
:1017280006164FEAC30343EA52734FEAC2025FEA5E
:101738001C1CC0D111F4801F0BD141EA00014FF0ED
:1017480000004FF0004CB6E711F4801F04BF0143BE
:101758000020B4F1FD0C88BFBCF5E06F3FF6AFAEDA
:10176800B5EB030C04BFB6EB020C5FEA500C50F16A
:10177800000041EB045170BD0EF0004E4EEA1131ED
:1017880014EB5C04C2BFD4EB0C0541EA045170BDF4
:1017980041F480114FF0000E013C90E645EA060E38
:1017A8008DE60CEA135594EA0C0F08BF95EA0C0F66
:1017B8003FF43BAF94EA0C0F0AD150EA01347FF4AE
:1017C80034AF95EA0C0F7FF425AF104619462CE785
:1017D80095EA0C0F06D152EA03353FF4FDAE1046E8
:1017E800194622E750EA410618BF52EA43067FF439
:1017F800C5AE50EA41047FF40DAF52EA43057FF4C9
:10180800EBAE12E74FF0FF3C06E000BF4FF0010CD3
:1018180002E000BF4FF0010C4DF804CD4FEA410C37
:101828007FEA6C5C4FEA430C18BF7FEA6C5C1BD004
:1018380001B050EA410C0CBF52EA430C91EA030F85
:1018480002BF90EA020F0020704710F1000F91EAE2
:10185800030F58BF994208BF90422CBFD8176FEAB0
:10186800E37040F0010070474FEA410C7FEA6C5C7E
:1018780002D150EA013C07D14FEA430C7FEA6C5C85
:10188800D6D152EA033CD3D05DF8040B704700BFB1
:101898008446104662468C461946634600E000BFFF
:1018A80001B5FFF7B7FF002848BF10F1000F01BDD1
:1018B8004DF808EDFFF7F4FF0CBF012000205DF89C
:1018C80008FB00BF4DF808EDFFF7EAFF34BF012021
:1018D80000205DF808FB00BF4DF808EDFFF7E0FFBA
:1018E80094BF012000205DF808FB00BF4DF808ED0B
:1018F800FFF7CEFF94BF012000205DF808FB00BF72
:101908004DF808EDFFF7C4FF34BF012000205DF853
:1019180008FB00BF4FEA4102B2F1E04324BFB3F530
:10192800001CDCF1FE5C0DD901F0004C4FEAC0024E
:101938004CEA5070B2F1004F40EB830008BF20F032
:101948000100704711F0804F21D113F13872BCBFEC
:1019580001F00040704741F480114FEA5252C2F141
:101968001802C2F1200C10FA0CF320FA02F018BF8A
:1019780040F001004FEAC1234FEAD32303FA0CFCDD
:1019880040EA0C0023FA02F34FEA4303CCE77FEA6C
:10199800625307D150EA01331EBF4FF0FE4040F4B6
:1019A8004000704701F0004040F0FE4040F4000065
:1019B800704700BF80F0004002E000BF81F00041A6
:1019C80042001FBF5FEA410392EA030F7FEA226CDD
:1019D8007FEA236C6AD04FEA1262D2EB1363C1BF6D
:1019E800D218414048404140B8BF5B42192B88BFDC
:1019F800704710F0004F40F4000020F07F4018BFFF
:101A0800404211F0004F41F4000121F07F4118BF1E
:101A1800494292EA030F3FD0A2F1010241FA03FCC6
:101A280010EB0C00C3F1200301FA03F100F00043AE
:101A380002D5494260EB4000B0F5000F13D3B0F176
:101A4800807F06D340084FEA310102F10102FE2AE5
:101A580051D2B1F1004F40EBC25008BF20F0010055
:101A680040EA03007047490040EB000010F4000F03
:101A7800A2F10102EDD1B0FA80FCACF1080CB2EB96
:101A88000C0200FA0CF0AABF00EBC25052421843F5
:101A9800BCBFD0401843704792F0000F81F400019A
:101AA80006BF80F400000132013BB5E74FEA41036D
:101AB8007FEA226C18BF7FEA236C21D092EA030FD9
:101AC80004D092F0000F08BF0846704790EA010F53
:101AD8001CBF0020704712F07F4F04D1400028BF80
:101AE80040F00040704712F100723CBF00F5000062
:101AF800704700F0004343F0FE4040F40000704798
:101B08007FEA226216BF08467FEA23630146420243
:101B180006BF5FEA412390EA010F40F48000704756
:101B28004FF0000304E000BF10F0004348BF4042FC
:101B38005FEA000C08BF704743F0964301464FF038
:101B480000001CE050EA010208BF70474FF0000394
:101B58000AE000BF50EA010208BF704711F00043D5
:101B680002D5404261EB41015FEA010C02BF8446A5
:101B78000146002043F0B64308BFA3F18053A3F504
:101B88000003BCFA8CF2083AA3EBC25310DB01FA4B
:101B980002FC634400FA02FCC2F12002BCF1004FCF
:101BA80020FA02F243EB020008BF20F00100704760
:101BB80002F1200201FA02FCC2F1200250EA4C00B4
:101BC80021FA02F243EB020008BF20EADC707047FA
:101BD8004FF0FF0C1CEAD0521EBF1CEAD15392EA08
:101BE8000C0F93EA0C0F6FD01A4480EA010C4002E4
:101BF80018BF5FEA41211ED04FF0006343EA50103E
:101C080043EA5111A0FB01310CF00040B1F5000F7F
:101C18003EBF490041EAD3715B0040EA010062F12E
:101C28007F02FD2A1DD8B3F1004F40EBC25008BF18
:101C380020F00100704790F0000F0CF0004C08BF36
:101C480049024CEA502040EA51207F3AC2BFD2F103
:101C5800FF0340EAC250704740F400004FF0000311
:101C6800013A5DDC12F1190FDCBF00F0004070474B
:101C7800C2F10002410021FA02F1C2F1200200FA89
:101C880002FC5FEA310040F1000053EA4C0308BF50
:101C980020EADC70704792F0000F00F0004C02BFA1
:101CA800400010F4000F013AF9D040EA0C0093F01C
:101CB800000F01F0004C02BF490011F4000F013B76
:101CC800F9D041EA0C018FE70CEAD15392EA0C0FE4
:101CD80018BF93EA0C0F0AD030F0004C18BF31F04F
:101CE800004CD8D180EA010000F00040704790F025
:101CF800000F17BF90F0004F084691F0000F91F0C9
:101D0800004F14D092EA0C0F01D142020FD193EA8E
:101D18000C0F03D14B0218BF084608D180EA010016
:101D280000F0004040F0FE4040F40000704740F0F2
:101D3800FE4040F4400070474FF0FF0C1CEAD052C0
:101D48001EBF1CEAD15392EA0C0F93EA0C0F69D01C
:101D5800A2EB030280EA010C49024FEA402037D087
:101D68004FF0805343EA111143EA10130CF000407E
:101D78008B4238BF5B0042F17D024FF4000C8B426E
:101D880024BF5B1A40EA0C00B3EB510F24BFA3EB4E
:101D9800510340EA5C00B3EB910F24BFA3EB91031E
:101DA80040EA9C00B3EBD10F24BFA3EBD10340EA78
:101DB800DC001B0118BF5FEA1C1CE0D1FD2A3FF6BE
:101DC80050AF8B4240EBC25008BF20F00100704773
:101DD8000CF0004C4CEA50207F32C2BFD2F1FF0316
:101DE80040EAC250704740F400004FF00003013A47
:101DF80037E792F0000F00F0004C02BF400010F4EB
:101E0800000F013AF9D040EA0C0093F0000F01F0FE
:101E1800004C02BF490011F4000F013BF9D041EA20
:101E28000C0195E70CEAD15392EA0C0F08D1420253
:101E38007FF47DAF93EA0C0F7FF470AF084676E726
:101E480093EA0C0F04D14B023FF44CAF08466EE7FF
:101E580030F0004C18BF31F0004CCAD130F00042CD
:101E68007FF45CAF31F000437FF43CAF5FE700BF25
:101E78004FF0FF3C06E000BF4FF0010C02E000BF4E
:101E88004FF0010C4DF804CD4FEA40024FEA4103F0
:101E98007FEA226C18BF7FEA236C11D001B052EAA6
:101EA800530C18BF90EA010F58BFB2EB030088BF6C
:101EB800C81738BF6FEAE17018BF40F001007047DB
:101EC8007FEA226C02D15FEA402C05D17FEA236CBD
:101ED800E4D15FEA412CE1D05DF8040B704700BF04
:101EE800844608466146FFE70FB5FFF7C9FF00289B
:101EF80048BF10F1000F0FBD4DF808EDFFF7F4FFD4
:101F08000CBF012000205DF808FB00BF4DF808ED6C
:101F1800FFF7EAFF34BF012000205DF808FB00BF8F
:101F28004DF808EDFFF7E0FF94BF012000205DF8B1
:101F380008FB00BF4DF808EDFFF7D2FF94BF012062
:101F480000205DF808FB00BF4DF808EDFFF7C8FF5B
:101F580034BF012000205DF808FB00BF42000ED20C
:101F6800B2F1FE4F0BD34FF09E03B3EB126209D4CC
:101F78004FEA002343F0004323FA02F070474FF082
:101F88000000704712F1610F01D1420202D14FF0F7
:101F9800FF3070474FF00000704700BF00F026F890
:101FA8000C4880F30888002103E00B4B5B58435032
:101FB80004310A480A4B42189A42F6D3094A02E009
:101FC800002342F8043B084B9A42F9D317F0E0FE8D
:101FD8007047000000C00020544A03080000002099
:101FE80090110020901100203C5500207047FEE71A
:101FF80010B586B0002301244FF46022114801A9CE
:1020080001938DF80930039204938DF808408DF8F8
:10201800144022F0EDFC0B48214622F00FFD094840
:1020280022F016FD074822F018FD0028FAD10548CD
:1020380022F017FD034822F019FD0028FAD106B056
:1020480010BD00BF00240140014610B50D48012213
:10205800032322F019FD0B48012122F00BFD7F20FC
:1020680023F048FB0748022122F058FD0028F6D04B
:102078000448022122F058FD0248BDE8104022F031
:102088004ABD00BF002401400C4A0C2303FB012376
:1020980010B59C880CB9588010BD5B8803F11304F7
:1020A800844204DA142B07D9133B834204DC0C2343
:1020B80003FB012102238B8010BD00BFA02B002051
:1020C8000A4B10B500241C7021464FF4E0720848F2
:1020D800FEF760F9074B43F601501C70064B1C7065
:1020E8000FF03AFB054B187010BD00BF54140020C8
:1020F800201600206B180020E8170020EA1700209F
:10210800074B1978013101F01F011970054B1A7836
:102118008A4203D1013202F01F021A70704700BFD1
:10212800E81700206B18002010B50E4A0E2303FB99
:1021380000200D4A014614780C4A03FB042300F1E1
:102148000C0251F8044B914243F8044BF9D10A8828
:1021580000211A800E22FEF71DF9BDE81040FFF796
:10216800CFBF00BF58140020E81700202016002019
:10217800084B1A5C002352FA03F111F0010FD8B290
:1021880002D00130C0B270470133082BF3D10120CF
:10219800704700BF3119002000F07F0000F574502F
:1021A8002DE9F84306300C46154698460FF0D4FA48
:1021B80000284FD043F63937002638460FF0CCFABE
:1021C800C0B25FFA86F988B120280FD04FEA5900CB
:1021D80000F52C4043300FF0BFFAC0B208B1022816
:1021E80004D10123B340227813432370113743F6F7
:1021F800C13301369F42E0D14AF6EA200FF0ACFA2B
:10220800C0B280B120280ED02B784AF6D92043F0EE
:1022180001032B700FF0A0FAC0B220B1202802D021
:10222800012388F800304AF61B300FF095FAC0B247
:1022380080B120280ED02B784AF6D92043F002032B
:102248002B700FF089FAC0B220B1202802D00123E8
:1022580088F80030BDE8F883034610465A1E10B5CA
:10226800032A1CD8DFE802F00E0E0207114A527842
:1022780002F0100203E00F4A527802F00802D2B2CC
:1022880072B10BE00C4A927802F04002D2B23AB135
:102298000A4A127802F003029A4200D140B10022A1
:1022A8000748105C984203D00132052AF8D1002172
:1022B800084610BD4C5300209C3700203B3C0020B2
:1022C80018160020F8B5064643F639350024284686
:1022D8000FF042FAC0B2E7B268B120280BD07808F4
:1022E80000F52C4043300FF037FA012803D1A04005
:1022F80033781843307001341135082CE7D1F8BD14
:1023080003780E2202FB0313084AD3189978002396
:1023180051FA03F010F00100DAB202D0501CC0B23A
:1023280070470133082BF3D1704700BF20160020F7
:102338002DE9F04101248C40284A29490346E4B29A
:10234800107891F800C019E0264F0E2606FB00769B
:10235800F178A9B996F80680B8F1000F10D196F86F
:102368000580B8F1000F0BD196F80480B8F1000F82
:1023780006D1F67926B9013000F01F00054626E09F
:10238800FBB1012B05D0022B06D10E2101FB0077F2
:1023980039790C4218D014E0042B04D10E2101FB2A
:1023A8000077B9790CE0032B04D10E2101FB0077EB
:1023B800797905E0052B07D10E2101FB0077F97922
:1023C80011B11570BDE8F081013000F01F006045C3
:1023D800BAD11570FF20BDE8F08100BF6B1800204E
:1023E800E8170020201600202DE9F043444D454B06
:1023F8002A780E2101FB0232917A85B0044698466C
:1024080039B101390523594301F56E51413189B27A
:1024180001E043F6C131204604220FF0AEF92B78D3
:102428000E2505FB038393F80B80364E344FB8F125
:10243800000F25D131232371073363713B7801A83D
:102448006B430422F15E06F013FB3B7802A805FB00
:1024580003630222997A06F00BFB3B780DF10A0020
:1024680005FB03650322697A06F002FBA01D01A99A
:102478000922FEF765FA4FF00F0984F8108012E080
:10248800B8F1010F0FD132232371053363713B7803
:102498004FF0080905FB036393F90130E3713B78BA
:1024A8005D43735BA371002320461A4612E010F8BF
:1024B800011BA1F13005EDB2092D04D8EB18302924
:1024C800DBB203D004E037395B1800E00A33DBB233
:1024D8000132D2B24A45EAD10F21B3FBF1F108012A
:1024E800411A5B1AC3F10F03DBB2092BA35401D8BD
:1024F800303300E03733A35405B0BDE8F08300BFA4
:102508001E16002020160020024B1A7842F0010205
:102518001A707047BD1B002008B50C4B0C4A1B787D
:102528000E2101FB0323D97A21B101290CBF09210E
:10253800002100E0102140221346064806F0BCF8AE
:10254800054B1A7842F002021A7008BD1E160020C8
:1025580020160020EB170020BD1B0020034B1A7823
:1025680002F0F8026FF3C3021A707047BD1B002017
:10257800024B1A7842F004021A707047BD1B002003
:10258800024B1A7842F008021A707047BD1B0020EF
:1025980038B5114B1C7814F0010502D1FFF7B4FFD0
:1025A80005E004F00405EDB21DB9FFF7E1FF284688
:1025B80038BD04F00805EDB215B9FFF7E1FFF6E7FD
:1025C80004F00204E4B21CB9FFF7A6FF204638BDA8
:1025D800FFF7C4FF012038BDBD1B0020014B187850
:1025E800704700BF5414002030B51E4B85B01B78CF
:1025F8000446002B34D11C4D2B78034113F0010FF6
:102608002ED01A4B1A4A1B780E2101FB0323DA78C5
:10261800024112F0010F1CD11B79034113F0010391
:1026280017D110F0010001F1F1014FEA540206D070
:1026380001320091019302926D20FE3905E00132CA
:102648000091019002923C20012103220B460FF0D9
:1026580001F9012313FA04F42B7823EA04042C70FB
:1026680005B030BDEA170020E11700206B180020E4
:1026780020160020037830B513F0010F144A4FF0EC
:102688000E0419D104FB01210133012212FA03F3CC
:10269800CD7825EA0303CB7004780D79A41812FAD3
:1026A80004F425EA04040C7103789B189A408B788B
:1026B80023EA02028A7030BD04FB0121013B01229A
:1026C80012FA03F38A7822EA03038B7030BD00BF45
:1026D8002016002010B500230278590052FA01F4A0
:1026E80004F00304022C05D1013414FA01F122EAA2
:1026F800010202700133042BEED110BD2DE9F04F19
:1027080085B00192BDF838201C46744B0092DA78E7
:10271800054612F020028B4640F0D9808DF80E2035
:102728008DF80F208DF80D20DCB99B7803F040035D
:10273800DBB21BB101238DF80F3020E0684B5B78CA
:1027480003F00203DBB21BB101238DF80E3016E053
:102758000DF10F010DF10E020DF10D03FFF71CFD38
:102768000DE0012C0BD19B7803F04003DBB223B9B9
:102778000DF10F00FFF7A6FD01E08DF80F409DF861
:102788000F3023B99DF80E00002800F0A38044B94B
:1027980005F07F01490001F574510DF10A0062311D
:1027A8000AE0012C0BD1E90101F5124101F5BA71DA
:1027B8000DF10A0001EB4B0102220EF0DEFFBDF91C
:1027C8000A3013B9002C00F08480009B33B9454BC4
:1027D800454F93F80080FFF793FC08E0434B444FC4
:1027E80093F8008008F1010202F01F021A700DF13F
:1027F8000F00FFF76FFF002C44D1BDF80A3069B213
:1028080040F6B83212EA210238BF4FF47A72D21871
:102818000E2303FB08F3ADF80A20FA529DF80F9037
:10282800224649460120FE18FFF716FD4946F0707A
:1028380022460220FFF710FD86F8029030719DF8BD
:102848000E90224649460420FFF706FD4946B0711E
:10285800824622460320FFF7FFFC05F07F057071D2
:102868003572BAF1000F00D128B1224B1B7813B989
:102878009DF80D3000E00023F37186F809B0019A45
:10288800B2721CE0012C1AD10E2303FB08F3BDF829
:102898000A202046FA529DF80F6000223146FD18A2
:1028A800FFF7DAFC3146E87000220220FFF7D4FC7B
:1028B80000232871AE70AB716B71EB71AB720E2394
:1028C80003FB0877FC72009B0120BB8102E000201B
:1028D80000E0204605B0BDE8F08F00BF9C3700201F
:1028E8004C530020E8170020201600205314002025
:1028F80058140020A21B002073B5154B04461B7802
:102908000E46D3B11348214621F019FA0546A0B95D
:10291800012E04F1010606D12046FFF729FC009597
:102928000246812005E02046FFF722FC009502467A
:10293800982031462B46FFF7E1FE2146054821F055
:10294800E8F90548214602B0BDE8704021F0ECB92D
:10295800E91700206C1A0020801800202DE9F743A1
:102968007B4B04461B7843B17A4B1B7803F0240356
:10297800042B02D1002900F0E880774B774F1B78B1
:10298800002B00F0C7807648214621F0D8F90028AE
:1029980040F0C08007F5C470214621F0D0F9804688
:1029A800002840F0B7803B1993F880302D2B01D0D8
:1029B800532B3AD16B4E357845B30FF02DFA04F10D
:1029C8000108054650B12046FFF7D2FB337802468E
:1029D8001E33009393204146002307E02046FFF76B
:1029E800C7FB00950246414693202B46FFF786FE1B
:1029F8000FF012FA014628B1337813201E330093E2
:102A0800002101E0009013200A4680E02046FFF7ED
:102A1800AFFB611C02462B4693200095FFF76EFE24
:102A28000095132029462A4671E0542B09D12046E7
:102A3800FFF79EFBCDF800800246611C94204346B8
:102A480066E0462B474D20D12E78BEB10FF0E4F951
:102A580004F10109064648B12046FFF789FB2B78A7
:102A680002461E3300939A20494622E02046FFF78B
:102A78007FFB0096024649469A2025E02046FFF74C
:102A880077FB009602469A2039E02E78002E2CD04B
:102A98000FF0C2F904F11C09064660B12046FFF7A1
:102AA80067FB2B7802461E3369F07F000093C0B2A3
:102AB800611C434609E02046FFF75AFB024669F0CD
:102AC8007F000096C0B2611C3346FFF717FE0FF077
:102AD800A3F921B2024628B12B7803201E330093B4
:102AE800002214E00090032011E02046FFF740FB8D
:102AF800024604F11C0060F07F000096C0B2611C21
:102B08003346FFF7FBFD009603202146324601239A
:102B1800FFF7F4FD124821463F1921F0FAF897F81B
:102B280080302D2B0AD0532B08D0542B06D0462B9F
:102B380004D00D48214621F002F930B10B48214656
:102B480003B0BDE8F04321F0EFB803B0BDE8F0836F
:102B5800561400205A1A0020E9170020CC2900201A
:102B68006C1A0020C41A0020542B0020641A00207C
:102B7800002302780E2101FB0232044901338A182E
:102B88000021062B9170F4D1704700BF2016002059
:102B9800064B00201870064B1A78064B1B789A4291
:102BA80002D00146FFF7C4BBFF2070475414002031
:102BB800E81700206B1800200121814038B5114B1F
:102BC800C9431A78104BC9B202F0030203F5E07446
:102BD800012A04D1DD7801EA0505DD7005E0022A45
:102BE80003D11D7901EA05051D710E33A342EFD10A
:102BF800FFF7FAFC43F601500EF0AEFD034B1870D8
:102C080038BD00BF3B3C002020160020EA170020FA
:102C18002DE9F743A34D8DF807002B78A24C1BB183
:102C28002378C2B29A4204D043F601500EF094FDC4
:102C380028709DF8073023709C4C2278072A00F2F0
:102C48002D81DFE812F008002400360054005D00F2
:102C580072008D00BA00964A3C211170954A1946B7
:102C6800107800F00300FFF763FB934BFF28187000
:102C780000F036811FF098FD904B002093F87420E7
:102C880042F0010283F874208D4B187064E0884B81
:102C98001B78002B00F024811FF04EFF012840F024
:102CA8004D812378142201332370864B01381A7022
:102CB80047E17F4B1B78002B00F01281814E307862
:102CC80008B901234AE01FF037FF022804D01FF09B
:102CD80033FF032840F032811FF066FD2378042279
:102CE800013323701D233370774B1A7026E1704B24
:102CF8003C221A707548FFF777FB2378013323705D
:102D08006B4B1B78002B00F0EB806E4B1D78002D71
:102D180040F014811020FFF73BFC002800F01181DF
:102D280023782846013323700BE1614B1B78002B75
:102D380000F0D68005F02AFD002800F00281614BE2
:102D48007D221A705E4B002018705C4B93F874203B
:102D580042F0010283F87420237801332370F0E0F5
:102D6800534B1B78002B00F0BB801FF0E5FE0128B9
:102D7800544E03D01FF0E0FE03280FD19DF8072022
:102D8800012111FA02F2524B197821EA02021A7053
:102D980064233370237801332370CFE03078002820
:102DA80040F0CC80484A032323701378013BDBB200
:102DB8001370002B00F09480C3E0404A414E92F813
:102DC8006A201AB13278002A40F0B88000223270A6
:102DD800013212FA03F3DFF8E0803E4F98F8001052
:102DE8004FF00E0909FB0172DB4392F803E0DBB2F6
:102DF80003EA0E0E907882F803E092F804E003EA02
:102E08000E0E0340937082F804E00DF10700FFF7FF
:102E180031FC98F8003009FB0372D278DFF89490FF
:102E28002AB999F8002002F00302012A0AD00E22DA
:102E380002FB03721279B2B999F8002002F003027A
:102E4800022A10D10E2202FB0377BA785AB9224F10
:102E58003A789A4207D11848FFF78AFE3B7801333F
:102E680003F01F033B7099F800009DF8071000F06D
:102E78000300FFF75DFA144B0422FF281A7088F844
:102E88000000164B42D0987800F04000C0B20028ED
:102E98003CD1032323701A33337052E00020207092
:102EA8004FE000BFEA1700205714002054140020F8
:102EB800E21700203B3C00201E160020C03B0020EB
:102EC8005514002052140020E0170020EB170020B2
:102ED800E1170020201600206B1800209C370020E6
:102EE800FFF73CFB002323701FF05EFC2B78013BAF
:102EF800DBB22B702BB1144B9B7803F04003DBB291
:102F0800F3B19DF80700FFF757FE19E09B780E4ACA
:102F180003F04003DBB22BB1136843F400031360E2
:102F2800FFF7CEF8FFF71AFB1FF03EFC00232370D3
:102F380043F601500EF010FC287001E0002000E07C
:102F4800FF20BDE8FE8300BF9C370020044B1A78A1
:102F58000AB1013A1A701B780BB9FFF72DBE7047FA
:102F6800EA170020044A054B10781B7803EA501032
:102F780000F00100704700BF9C370020331A002082
:102F8800044B054A1B781078C3F3400303EA10107A
:102F9800704700BF331A00209C370020034B044AB7
:102FA8001B78D078C3F3800318407047331A002089
:102FB8009C370020044B054A1B78D078C3F3C00324
:102FC80003EA5000704700BF331A00209C370020E6
:102FD800044B054A1B78D078C3F3001303EA90002A
:102FE800704700BF331A00209C370020044B187824
:102FF800044BDB785B005BB2DB1103EAD01070474F
:10300800331A00209C37002008B5054820F06AFED6
:10301800044B5B78002814BF002003F0010008BDB2
:1030280074180020331A002070B500241BE03046C5
:10303800E9B21BF091FF80B14FF4D06363433422AF
:1030480002FB05330A4AD3181B7A13F0010F04D088
:10305800084B1878C0F3001070BD0135202DE6D15B
:103068000134022C02D0E6B20025E0E7002070BD52
:10307800143D0020331A002008B51BF00DF9034B4E
:103088001B7800EA931000F0010008BD331A0020F5
:10309800044B054A1B78D078C3F3401303EAD000E9
:1030A800704700BF331A00209C3700202DE9F74FE6
:1030B800FFF758FF8246FFF763FF8346FFF76EFF6F
:1030C8000190FFF777FF8146FFF782FF0446FFF77D
:1030D800ABFF0546FFF7DCFF8046FFF7CDFF07464D
:1030E800FFF784FF0646FFF78FFF019B45EA0404BC
:1030F8009B0043EA4B0343EA0A0343EAC90343EA52
:10310800481343EA871343EAC61343EA0023E0B2AD
:1031180043EA0010BDE8FE8F044B987800F00F00DA
:10312800A0F10203584240EB03007047D118002079
:10313800044B987800F00F00A0F10102504240EBD8
:1031480002007047D1180020044B987800F00F0057
:10315800A0F10301484240EB01007047D11800205C
:10316800054B987800F00F00A0F1060CDCF1000088
:1031780040EB0C00704700BFD1180020514AF0B551
:1031880013781446012B29D003D3022B40F09880E2
:103198005EE04D484D4B047819786FF3C304047012
:1031A80001F0F80158786FF3C301197000F080013D
:1031B800C9B2002900F08480012111709C78062290
:1031C80004F00F04544302464148005D60F30602D0
:1031D8005A701A7861F302021A70F0BD3B494D78B3
:1031E8000B4625F07F00002838D00A7802F0080244
:1031F800D2B222B9344A117841F0080111709A7894
:1032080002F00F02012A04D12F4A117841F001017E
:10321800117015F07F0F53D119789E7801F00700CF
:10322800062206F00F0602FB0606294F5D78BE5DF2
:10323800013066F3060500F007005D7090FBF2F5BB
:1032480002FB150262F30201197002232370F0BD1C
:103258001E494D780B4625F07F0028B98B7860F31E
:1032680003038B701070F0BD174A11786FF3C30118
:103278001170997801F00F01012903D111786FF3CA
:103288000001117015F07F0F1AD119789E7801F09E
:103298000700062206F00F0602FB06060C4F5D78B3
:1032A800BE5D013066F3060500F007005D7090FB17
:1032B800F2F502FB150262F3020119700123237073
:1032C800F0BD00BF201900207F180020D118002071
:1032D8009C57020810B51F4A1F4B92F9031009B1F9
:1032E800002231E008B1032119701978032930D878
:1032F800DFE801F00209192C1178002929D01548B6
:1033080081700121197092F90200124920B1134B02
:103318001A786FF3861217E0487808B9032213E089
:1033280088700221197092F902100A4889B90B4A6B
:10333800147861F386141470026861F30F22D1B215
:1033480061F31742026001221A7010BD002111605A
:10335800197010BDC81A00207D180020983A002066
:1033680038B5044643F6EF2343F6F020012A08BF98
:1033780018460D460EF0F0F92378C0B21842104CEA
:1033880009D043F6EE200EF0E7F9236860F307034F
:103398006FF30F230CE02B7818420AD043F6EE2087
:1033A8000EF0DAF92368C0B260F3070360F30F2365
:1033B800236094F9003013B1014B0F22DA7038BD45
:1033C800C81A002008B543F6F8200EF0C5F9014BDD
:1033D800187008BD7E180020014B1870704700BF98
:1033E8003D1A0020024B1A5C6FF303021A5470470F
:1033F8007A19002070B50C46C10001F5CE411B4872
:103408008B3108220EF0B9F9002518482946EEB28A
:1034180020F095FC08B9237823BB154B2278EB5C88
:103428001A421FD13046FFF7DDFFF6084AF6EB30A7
:1034380030180EF091F905F00703C0B2184110F0EA
:10344800010F0FD10B48294620F079FC50B12946CD
:10345800084820F069FC074B06F5CC40CA30995D56
:103468000EF070F90135402DCFD170BD3F1A002004
:1034780031190020D418002038B546F212754024BE
:103488002046FFF7AFFFA5F5CC43094AD23BD15CF4
:1034980011F0100F06D06FF30411D1542846002103
:1034A8000EF050F90134E4B20135B92CE8D138BD39
:1034B8007A1900203F287FB5054607D800F5E24075
:1034C8000D300EF049F9C3B22BB930E19C4A14789B
:1034D800002C00F031819B4E725D02F00F014C1CF4
:1034E80004F00F0464F303023F2D725533D8002C07
:1034F80000F0228101339C4240F01B81924B5A1903
:1035080092F88020522A725D03D161F3030272554A
:103518000FE16FF30302EC081B19725593F8902121
:1035280005F0070352FA03F313F0010F40F003818B
:103538002946864820F0EDFB844B04F5CC40195D04
:10354800CA3001240EF0FEF82D19022300930194CD
:10355800029518209EE0002C00F0EE80784B1B7836
:1035680001339C4240F0E580735D05F5CC406FF374
:103578000303D230012173550EF0E4F8735D43F074
:1035880010037355A5F14003DBB2072B07D80422BB
:10359800009201330232019202931920B3E0A5F19F
:1035A8004803DBB2072B07D8042200920133033209
:1035B800019202931A2061E0A5F15003DBB2062BB9
:1035C80007D80422009201330332019202931B2090
:1035D80054E0A5F15703DBB2032B07D8042200926D
:1035E8000133033201920293212047E0A5F15B03E6
:1035F800DBB2012B07D80422009201330232019278
:10360800029322207FE05D2D06D1042300930193CD
:10361800043B0293284684E05E2D07D104230093DF
:1036280001330193053B02935E207AE0A5F15F0325
:10363800DBB21F2B09D804220092013392180192A1
:10364800029333200121053A6DE005F16103DBB2F5
:10365800072B07D804220092013303320192029308
:103668005F200BE005F15903DBB2012B09D80422D6
:103678000092013303320192029360200121043A3F
:1036880051E0AA2D0CD1042300930124043B01949A
:10369800029361202146032223460EF0DBF84BE01B
:1036A800A92D07D104230093023B0193023B029307
:1036B800622036E0AD2D08D1042300930322043B99
:1036C80001920293632001212DE0AB2D06D1042342
:1036D8000093043B01930293642022E0AC2D06D1B1
:1036E80004230093043B01930293702019E005F131
:1036F8005203DBB2032B09D80422009201330232B1
:103708000192029368200121033A0CE04E35EDB294
:10371800062D10D804230093013502330193029536
:103728006A20012103220B460EF094F803E01C46A0
:1037380002E0002400E00124204604B070BD00BF70
:10374800000000207A190020CC290020D41800207D
:10375800024B185CC0F30010704700BF7A190020B4
:10376800F8B508220E4600210746FCF713FE46F27C
:103778008B7500243378234113F0010F08D02946B4
:10378800064808220DF0F9FF3846044920F08FFA60
:1037980001340835082CEDD1F8BD00BF491A0020C6
:1037A800024846F2CA6108220DF0E7BFD41800208B
:1037B80070B5044600F56A5044300DF0CDFF0B4D4E
:1037C80006462B7813F0010F02D1CC2021F0A4F883
:1037D8002B8843F001032B80054B1E55054B13F82E
:1037E800242042F0010203F8242070BD5A1A002058
:1037F800B118002090180020024B185C084100F016
:10380800010070473119002070B505460024094BA6
:10381800E0B2E618E35C4BB12946FFF7EDFF28B1AB
:10382800002333700448214620F07EFA0134402CEE
:10383800EDD170BD7C1A0020C118002038B50546AE
:1038480000242846E1B2FFF7D7FF10B1044BE35C30
:1038580023B90134082CF4D1002038BD012038BD2B
:10386800B118002038B505460EF0D6FAA0B10024EC
:103878002846E1B2FFF7C0FF40B1084B13F82430E7
:1038880013F0010F02D0064BE35C23B10134082C7E
:10389800EED1002038BD012038BD00BF90180020AF
:1038A800B1180020F8B5114800214022FCF772FD3C
:1038B80046F28B75002401270D4829460822A740A7
:1038C8000DF05BFFFFB200260948314620F037FAB9
:1038D80020B1064BF25C47EA0202F2540136402E50
:1038E800F2D101340835082CE5D1F8BD3119002092
:1038F800491A00202DE9FF4100263446B0461A4BEC
:103908001B78234113F00102184B23D0184F1D5D7B
:1039180017F82430A84538BFA84613F0010F1AD06D
:10392800CDB965F3000307F8243023B20122F71953
:1039380002935B2029462B46009201950DF08AFFE1
:103948007B78B878F9781843621C2B460095FEF707
:10395800D5FE00E01A5501340436082CCFD1054BAA
:1039680083F80080BDE8FF817E180020B118002090
:10397800901800207C18002010B50C4B1B78A3B1C0
:103988000B4B1B788BB100240A48214620F0D7F94D
:1039980040B10948214620F0D2F918B92046012142
:1039A800FEF7DCFF0134402CEED110BDE9170020F2
:1039B80056140020641A00204A2200202DE9F04302
:1039C800324C334A238800266FF386136FF3C403FF
:1039D8002380304B304F85B016701E709146984644
:1039E80017F8013B5BB32278D20052B243EAA21225
:1039F8002388402E62F3C40343F0400323801ED083
:103A080000253046E9B2FFF7F7FEA8B117F8013CE8
:103A180013F0010F06D00122AA4099F800100A43BA
:103A280089F8002013F0020F06D00123AB4098F864
:103A38000020134388F800300135082DE1D1013604
:103A4800F6B2412ECCD1237803F04005EDB2D5B9BA
:103A580003F02403042B0BD1FFF78EFFFF23009301
:103A68004020294602222B46019502950DF0F2FED0
:103A7800238800226FF345136FF382036FF3C403A7
:103A88002380064B1A7005B0BDE8F0835A1A00204F
:103A9800EC3900201C3A0020DF1800203E1A0020D4
:103AA80010B500240548214620F049F908B9044B0F
:103AB800E0540134402CF5D110BD00BF351A002068
:103AC800DF18002010B5127804469DF80810DAB106
:103AD800D3B111B10D4920F0DFF8ACB1082246F29C
:103AE800CA610B480DF049FE2146094820F0DFF86D
:103AF8000749082246F2CA600DF039FE0548044914
:103B0800BDE8104020F0E9B810BD00BF642B0020CC
:103B18006C180020D418002030B5064B04781D78A6
:103B280024EA05040C7001781B7823EA010313705A
:103B380030BD00BF7E18002038B50A4D002415F8A6
:103B4800013F2D2B09D0532B07D0542B05D0462BE2
:103B580003D00548214620F0E7F80134402CEED187
:103B680038BD00BF4B2A0020641A002010B50F484A
:103B780020F08AF800240E48214620F0E0F880B1B1
:103B88000C4BE31893F88030482B06D003D82D2B24
:103B980003D0462B00E0542B03D10448214620F0E3
:103BA800B8F80134402CE6D110BD00BF211900201F
:103BB800641A0020CC290020094A0A4B117831B137
:103BC800997801F00F01814201D0002111709A7893
:103BD80060F303029A705A7842F080025A70704774
:103BE80020190020D11800202DE9FF411E466C4BFA
:103BF800DDF82880154604461A780F4600236949DF
:103C080011F8231011F0010F03D00121994022EA85
:103C180001020133082BF2D1634B1A70002C6FD0CC
:103C280014F0010F0AD0FF2301210093FF3B0193F9
:103C3800029352200A460B460DF00CFE14F0020FB8
:103C48000AD0FF2301210093FF3B019302935320E5
:103C58000A460B460DF0FEFD14F0040F0AD0FF23B0
:103C680001210093FF3B0193029354200A460B461F
:103C78000DF0F0FD14F0080F0AD0FF230121009386
:103C8800FF3B0193029355200A460B460DF0E2FDD7
:103C980014F0100F0AD0FF2301210093FF3B01937A
:103CA800029356200A460B460DF0D4FD14F0200F5F
:103CB8000AD0FF2301210093FF3B01930293572071
:103CC8000A460B460DF0C6FD14F0400F0AD0FF233C
:103CD80001210093FF3B0193029358200A460B46AB
:103CE8000DF0B8FD14F0800F0AD0FF2301210093D6
:103CF800FF3B0193029359200A460B460DF0AAFD9B
:103D0800CFB100243046214620F019F860B1FF23D6
:103D18000093FF3B0193631C1BB2012102935A20BD
:103D28000A460B460DF096FD2146304601341FF039
:103D3800FBFF402CE6D1BDB10024404621461FF0D0
:103D4800FEFF70B1012D0CD104230093DB18019301
:103D5800631C1BB202937420294603222B460DF0E4
:103D680079FD0134402CE8D10F481049104AFFF77B
:103D7800D3FE104B00221A700132009206320192D3
:103D8800F832029209490A4A074809F087FE0A4BA5
:103D98003C2251201A7004B0BDE8F0410EF028B959
:103DA8007E18002090180020281C0020111D0020DB
:103DB800041D0020ED1B0020B018002037B5FFF7C8
:103DC80075F904460E481FF08DFFD0F101050D4826
:103DD80038BF00251FF086FF10B914F4807F03D187
:103DE80024B95DB1224602E0012200E00022054B21
:103DF800204600932946024BFFF7F6FE3EBD00BF62
:103E08007219002074180020054B03EBD00393F8B7
:103E1800903100F0070053FA00F000F001007047FD
:103E2800CC29002010B50F4B04461B7813F0010372
:103E380015D0FFF703FD28B90B4B1B1993F88030F9
:103E4800462B0DD10DF0E8FF18B92046FFF7DCFF2F
:103E580030B1064821461FF05CFF012010BD18460E
:103E680010BD00BF5A1A0020CC290020721900206A
:103E7800024B1878003818BF01207047B01800208E
:103E880010B5034C04EB830358709970DA7010BDB9
:103E98009018002010B500240948002100190E22AE
:103EA8000E34FCF777FAB4F5E07FF5D1054A002324
:103EB8001370054A002199520233AA2BF9D110BD7B
:103EC8005814002053140020861D00207FB5474B4E
:103ED80004461B780E46AA2B78D0454821461FF089
:103EE8002EFF0546002871D12046FFF79BFF0028CA
:103EF8006DD1404821461FF022FF50B93E48214667
:103F08001FF01DFF054620B92046FFF7D3FA002809
:103F18005DD13A4B1B7823B9394B1B7813F0010F4D
:103F280009D1384BDB7803F02003DBB21BB9364BE1
:103F3800032283F84020012E05D82E4821461FF081
:103F4800FEFE40B142E0022E07D12B4821461FF069
:103F5800F6FE10B13AE0274800E0274821461FF056
:103F6800D8FE2A4821461FF0DFFE022E15D1012572
:103F7800294603222B4600964A2066190195029687
:103F88000DF068FC2046FEF7F3F8002302463146A0
:103F980018200093FEF7B2FB19E0012E09D1022385
:103FA8000093631C02930196122031460322334684
:103FB80009E07EB90121022300936318029301915D
:103FC800112003220B460DF045FC03E0002528468E
:103FD80004B070BD2046FEF7CBF80246012000234E
:103FE800211800930125FEF789FBF0E73D1A002010
:103FF800D418002080180020BC1A00207E18002049
:10400800811D00209C370020DF1800206C1A00203A
:104018002DE9FF4704460D46754821461FF08FFEDF
:104028008146002840F0DF80214671481FF071FE6C
:10403800704821461FF078FE6F4E0DBB01274FF0E8
:104048000208E31902934246032039463B46CDF85D
:10405800008001970DF0FEFB327862B10DF0DCFEB6
:10406800024630B1337840461E33009321462A4633
:1040780004E0009000E00092404621463B4628E0DC
:10408800012D2BD15D4B04F5E2400D301F5D0DF085
:1040980063FB07F00F07874209DA631C02220293C9
:1040A8000E2029462B46009201950DF0D3FB32785D
:1040B80092B10DF0B1FE024638B14F4B0D201B787E
:1040C80021461E330093002202E000900D20214675
:1040D8000123FEF713FB5EE00092F7E7022D0BD1F8
:1040E80001230193E3180293142049462A464B46BC
:1040F80000950DF0AFFB4EE0032D4CD101272A4669
:104108004FF0020804EB070A4D2039463B46CDF82C
:1041180000800197CDF808A00DF09CFB35783DB3E1
:104128000DF07AFE024630B1337840461E330093D4
:1041380021464A4602E00090214640463B46FEF7AB
:10414800DDFA0DF069FE671C054648B12046FEF70A
:104158000FF8337802461E3300931A2039462CE0B4
:104168002046FEF705F80095024639461A202DE04C
:1041780021462A463B4640460095FEF7BFFA2046B0
:10418800FDF7F6FF514602462B461A200095FEF72A
:10419800B5FA384628E03578EDB10DF03DFE04F16A
:1041A8001C06054658B12046FDF7E2FF124B0246B1
:1041B8001B7830461E330093611C002307E020461D
:1041C800FDF7D6FF009502463046611C2B46FEF7E8
:1041D80095FA012008E02046FDF7CAFF009502463F
:1041E80004F11C00F1E7002004B0BDE8F08700BF2F
:1041F800641A00206C1A0020C41A00207A190020C2
:10420800064B1B1893F84001492804D0452814BFD1
:104218000320022070470120704700BFCC290020EE
:104228002DE9F041244F00243C70244821461FF01A
:1042380086FDE5B2224B002837D01E5D3B789E42B2
:1042480000D303B93E70002E30D131461C484022BD
:10425800FCF7A0F81B4B1C4803EBD50393F88881A7
:1042680004F0070348FA03F8214608F001081FF094
:1042780066FD68B9B8F1000F02D02846022101E0B6
:1042880028463146FFF7C4FE28460DF0B1FE0DE082
:10429800B8F1000F0AD12846FFF7B2FF0B4BDB78C5
:1042A80003F02003DBB20BB9094B18550134402C3D
:1042B800BBD1BDE8F08100BFC41A0020C11800209E
:1042C8007C1A0020CC290020641A00209C3700208A
:1042D800DF1800202DE9F04F914B89B01B7813F0BF
:1042E800010F06D08F4B1A786FF386121A7001F0FF
:1042F800E0BA8D498D4A0B7810788D4D984218BFD9
:104308008C49137018BF0B706B7803F00803DBB28D
:104318004BB143F6CF200DF01FFA864B18702B884F
:104328006FF3CB232B80844B1B78AA2B08D18349AE
:10433800AA3B0B702B8843F080032B8000F012BF40
:104348006A787B4B02F01002D2B27D4CA2B11A8877
:104358006FF30C321A807B4B1B7823B97A4B1B788E
:1043680013F0010F08D1E37803F02003DBB21BB987
:10437800764B032283F840202368754F6FF3186348
:1043880023603A7802F00202D2B232B96B494A7815
:104398001AB16B4A43F080731360E67816F0010691
:1043A80048D05D20FFF7D4F900285AD16B78DFF8A0
:1043B800808103F00203DBB22BBB5D30FFF77AF894
:1043C800064600BBB8F80030012143F40073A8F892
:1043D8000030042303220093019302900B460D2022
:1043E8000DF038FA45200DF003FE31460122334620
:1043F8000D200096FEF782F9092031463246012346
:104408000096FEF77BF96B7803F00203DBB243B347
:104418004C4B1B7823B94C4B1B7813F0010F20D160
:10442800E37803F02003DBB2DBB9484B032283F8BF
:10443800402016E06B7803F00203DBB26BB1314623
:10444800324601230A200096FEF758F98D2031469E
:10445800012233460096FEF751F92B886FF3492362
:104468002B802368354A6FF35963236093787BB1B7
:10447800D37823B93B7813F00C0F05D108E03B78CB
:1044880003F00C03042B03D0236843F0007323606C
:10449800E17801F00201C9B200295BD05E20FFF784
:1044A80057F9002865D16B78214F03F00403DBB27C
:1044B800EBB95E30FEF7FEFF0646C0B93B88012126
:1044C80043F480633B800423009301330322019368
:1044D80002900B4617200DF0BDF945200DF088FD20
:1044E8000D203146012233460096FEF707F96B7816
:1044F80003F00403DBB2002B3BD0124B1B7823B92B
:10450800114B1B7813F0010F33D1E37803F020032C
:10451800DBB273BB0D4B032283F8402029E000BFB8
:10452800291C0020983A0020471A0020481A002029
:104538005A1A0020C51A00203D1A002090110020A8
:104548009C3700207E180020811D0020DF180020E5
:10455800CA2900206B7803F00403DBB22BB18D204D
:1045680001220B460091FEF7C9F82B886FF38A23C6
:104578002B8023684FF05F0B6FF3DF7323600026F7
:1045880096E00598F9B21AF0E7FC002875D04FF4C8
:10459800D0637343342202FB0733A749A8F15E0AAC
:1045A800CB1803F108021B7A5FFA8AFA13F00103A9
:1045B8004DD02368404643F0004323600492FFF740
:1045C800C7F8049A002864D1937813F0040F20D117
:1045D8004046FEF76FFF049A8146D0B993780121CF
:1045E80043F00403937004230093DB180322019320
:1045F80032200B46CDF808A00DF02CF94A200DF01A
:10460800F7FC0C20514601224B46CDF80090FEF7EE
:1046180075F84FF4D0637343342202FB0733864A9C
:10462800D3189B7A13F0040F33D0844B1B7823B92B
:10463800834B1B7813F0010F2BD1E37803F0200391
:10464800DBB233BB7F4B032283F8402021E0927812
:1046580012F0040F05D08C20514601220093FEF77A
:104668004DF84FF4D0637343342202FB0733724989
:10467800CB189A7A6FF382020AE04FF4D06373433F
:10468800342202FB07336C4AD3189A7A60F3820209
:104698009A72013708F10108202F5FFA88F87FF431
:1046A80070AF01360BF1200B022E5FFA8BFB04D0A2
:1046B800F3B20593D846002763E72368624923F0DD
:1046C80080636FF39E7323600B79002B00F02584C1
:1046D8005E4ADFF87CB105924FF09F0800271BF86F
:1046E800011F3E460137002952D02368A8F15F0A0E
:1046F80043F080635FFA8AFA23605046FFF728F890
:1047080000285CD118237343DFF8489119F8032077
:1047180012F0100F23D150460493FEF7CBFE049BF2
:104728008246E0B919F80320012142F0100209F885
:10473800032004230093023301933BB20322029324
:104748000F200B460DF086F845200DF051FC0D208A
:10475800514601225346CDF800A0FDF7CFFF18239C
:10476800734319F8033013F0100F28D0334B1B781C
:1047780023B9334B1B7813F0010F20D1E37803F0F2
:104788002003DBB2DBB92F4B032283F8402016E06D
:1047980018237343DFF8BC9019F8033013F0100F97
:1047A80005D08D2001220B460091FDF7A7FF1823A5
:1047B800734319F803206FF3041209F80320059ACC
:1047C80012F8011F0592002946D02368404643F09D
:1047D80080432360FEF7BCFF002854D14FF018092E
:1047E80009FB06F9DFF86CA01AF8093013F0200F5E
:1047F80049D14046FEF75EFE0646002843D11AF826
:104808000930012143F020030AF8093004230093FA
:10481800033301933BB2032202934B200B460DF066
:1048280019F850200DF0E4FB1920314601223346D7
:104838000096FDF763FF26E0143D00207E18002057
:10484800811D0020DF18002090110020EE38002084
:104858001A3900202839002018237343DFF8A8925A
:1048680019F8033013F0200F05D0992001220B46C8
:104878000091FDF743FF18235E4319F806306FF3E4
:10488800451309F8063008F10108082F5FFA88F87F
:104898007FF425AF974ADFF874B205924FF05008BD
:1048A800083F1BF8011F3E460137002952D02368F4
:1048B80008F1620A43F080635FFA8AFA236050467F
:1048C800FEF746FF00285CD1DFF8449206EB06139A
:1048D80019F8032012F0400F23D150460493FEF735
:1048E800E9FD049B8246E0B919F80320012142F052
:1048F800400209F8032004230093023301933BB2DA
:104908000322029369200B460CF0A4FF45200DF00A
:104918006FFB0D20514601225346CDF800A0FDF74C
:10492800EDFE06EB061319F8033013F0400F28D0FC
:10493800714B1B7823B9714B1B7813F0010F20D1F1
:10494800E37803F02003DBB2DBB96D4B032283F875
:10495800402016E0DFF8B89106EB061319F803308B
:1049680013F0400F05D08D2001220B460091FDF772
:10497800C5FE06EB061319F803206FF3861209F833
:104988000320059A12F8011F0592002933D02368E5
:10499800404643F080432360FEF7DAFE002841D109
:1049A800DFF86CA106EB06191AF8093013F0200F8E
:1049B80038D14046FEF77EFD064698BB1AF8093006
:1049C800012143F020030AF809300423009303333C
:1049D80001933BB20322029310200B460CF03AFFDE
:1049E80050200DF005FB1920314601223346009670
:1049F800FDF784FE16E0DFF8189106EB061319F8A8
:104A0800033013F0200F05D0992001220B460091A6
:104A1800FDF774FE06EB061619F806306FF345131A
:104A280009F8063008F10108072F5FFA88F87FF4C3
:104A380038AF344ADFF8DCB005924FF05708073F2B
:104A48001BF8011F3E460137002967D0236808F18B
:104A5800570A43F080635FFA8AFA23605046FEF7EC
:104A680077FE002871D1DFF8B09006EB061319F82D
:104A7800032012F0400F23D150460493FEF71AFD8D
:104A8800049B8246E0B919F80320012142F0400254
:104A980009F8032004230093023301933BB2032255
:104AA800029367200B460CF0D5FE45200DF0A0FAC6
:104AB8000D20514601225346CDF800A0FDF71EFEF9
:104AC80006EB061319F8033013F0400F3DD00A4BDC
:104AD8001B7823B9094B1B7813F0010F35D1E37804
:104AE80003F02003DBB283BB054B032283F840208D
:104AF8002BE000BF9F3700207E180020811D00207A
:104B0800DF180020E137002028390020D5380020A0
:104B18005F380020D5370020FD370020DFF8B49338
:104B280006EB061319F8033013F0400F05D08D205B
:104B380001220B460091FDF7E1FD06EB061319F87B
:104B480003206FF3861209F80320059A12F8011F53
:104B58000592002933D02368404643F08043236000
:104B6800FEF7F6FD002841D1DFF868A306EB061929
:104B78001AF8093013F0200F38D14046FEF79AFC96
:104B8800064698BB1AF80930012143F020030AF8B9
:104B9800093004230093033301933BB203220293A9
:104BA8001F200B460CF056FE50200DF021FA19205C
:104BB8003146012233460096FDF7A0FD16E0DFF8E6
:104BC800149306EB061319F8033013F0200F05D0E1
:104BD800992001220B460091FDF790FD06EB061681
:104BE80019F806306FF3451309F8063008F1010883
:104BF800042F5FFA88F87FF423AF4FF000084FF0D6
:104C08005B094FF0A70A4646AB4B08F10108F15C77
:104C1800AA4F002949D02368484643F0806323609F
:104C2800FEF796FD002852D113237343FA5C12F065
:104C3800200F22D148460493FEF73CFC049B834690
:104C4800D8B9FA5C012142F02002FA5404230093F7
:104C5800023301930FFA88F30322029320200B46B4
:104C68000CF0F8FD45200DF0C3F90D20594601223E
:104C78005B46CDF800B0FDF741FD13237343FB5CA1
:104C880013F0200F23D08E4B1B7823B98D4B1B7844
:104C980013F0010F1BD1E37803F02003DBB2B3B9A3
:104CA800894B032283F8402011E013237343FB5CF4
:104CB80013F0200F05D08D2001220B460091FDF73F
:104CC8001DFD13237343FA5C6FF34512FA547F4BAF
:104CD800F15C002933D02368504643F080432360B9
:104CE800FEF736FD00283ED1132303FB06735A78DE
:104CF80012F0200F37D150460493FEF7DBFB049BDC
:104D0800834680BB5A78012142F020025A7004235E
:104D18000093033301930FFA88F3032202934C2084
:104D28000B460CF097FD50200DF062F919205946FA
:104D380001225B46CDF800B0FDF7E0FC13E0132339
:104D480003FB06735B7813F0200F05D0992001222E
:104D58000B460091FDF7D2FC132303FB06735A7828
:104D68006FF345125A705A4B1322F35C002B43D051
:104D780002FB06F317F803B0CBF3801BBBF1000F5F
:104D880022D143F6DE2004930CF0E6FC049BD8B154
:104D9800FA5C012142F04002FA5404230093DB1824
:104DA80001930FFA88F3032202932F200B460CF08D
:104DB80051FD47200DF01CF90920414601225B46B0
:104DC800CDF800B0FDF79AFC13237343FB5C13F096
:104DD800400F22D03A4B1B7823B93A4B1B7813F07B
:104DE800010F1AD1E37803F02003DBB2ABB9364BDD
:104DF800032283F8402010E07243BA5C12F0400F9F
:104E080005D08920414601220093FDF777FC132342
:104E18007343FA5C6FF38612FA5401360AF1010AF9
:104E280009F10109022E5FFA8AFA5FFA89F97FF41B
:104E3800EBAEDFF8A4A04827023E1AF8011FB046DF
:104E4800013600294CD02368384643F0804323605C
:104E5800FEF77EFC00285CD14FF01E0909FB08F91B
:104E6800DFF878B01BF8093013F0200F51D138461D
:104E7800FEF720FB804600284BD11BF809300121A2
:104E880043F020030BF80930042300930333019304
:104E980033B20322029313200B460CF0DBFC5020A4
:104EA8000DF0A6F81920414601224346CDF80080AE
:104EB800FDF724FC2DE000BFEC380020B0370020BF
:104EC8007E180020811D0020DF180020DD3800201A
:104ED800E7370020FD37002056380020B73A002079
:104EE8001E2303FB08F3DFF8749219F8033013F05C
:104EF800200F05D0992001220B460091FDF7FEFBFB
:104F08001E2303FB08F819F808306FF3451309F856
:104F180008300137082EFFB28FD1A67806F00806B0
:104F2800F6B2002E40F01E81DFF80892FBE0814BBC
:104F38003702DB19E2B218462146079205931EF0A4
:104F4800FEFE40B97B484037C01921461EF0F7FEE7
:104F5800002800F0DA80774937028037CF193846C1
:104F680021461EF0ECFE002840F0CF80384621464E
:104F7800F7B21EF0CEFEDFF8E8A10FB9404600E018
:104F880006980CF0E9FB8AF800009AF80000DFF8B0
:104F9800D0B1002800F0B9800138C0B28BF8000009
:104FA8000BF044FD002840F0B0809BF8000000F5AD
:104FB8006A5079300CF0D0FB5F4AC0B2107027B944
:104FC8005E4B434413F86AAC03E009EB040393F81F
:104FD800C0A000EA0A0ABAF1000F00F0968005980E
:104FE80021461EF0ACFEDFF860B1E0B13002514B53
:104FF8004030181821461EF0A2FEA0B95049012FD2
:105008000B784AEA030A8BF800A03ED1079A04F00D
:105018001F0153094FF4D0625A43342303FB012381
:105028004849CB182BE03002424A4030101821463C
:105038001EF085FE38B1059821461EF080FE10B995
:105048003F490B7804E03E4A13781AEA030F04D06C
:1050580023EA0A0A8BF800A017E04AEA030A012F9C
:105068008BF800A011D107994FF4D0624B095A432D
:1050780004F01F01342303FB0123324AD31893F8A9
:10508800302042F0200283F830202F482F49304A40
:10509800FEF742FD2D4B1B781BB1FEF707F80028E1
:1050A80033D12A482B4912F08DFC68B10CF0B4FEBC
:1050B80058BB284808F05EFD38BB0123254826491F
:1050C800224A0093FEF7FEFC002300931A4901339D
:1050D80001930B781C4802931C491D4A1E4B08F08B
:1050E800DDFC012F11D1079A04F01F0153094FF479
:1050F800D0625A43342303FB01231249CB1893F897
:10510800312042F0010283F83120069A0134053239
:10511800402C08F1010806927FF409AF0136022EEF
:1051280009F580791ED047F29773069349F22A3819
:105138000024FCE6C4270020C21C0020CC97FF1FD7
:105148007E180020143D0020281C0020111D00207E
:10515800041D002088180020ED1B0020B73A00200D
:1051680071190020B54C63786FF3C71363702B78FF
:1051780003F08002D2B2002A00F0D780B0490E783E
:10518800002E40F0D28003F02403042B0BD1FEF74D
:10519800F3FBFF2300934020314602223346019659
:1051A80002960CF057FB2B8800266FF3C7136FF39A
:1051B800820366F3451366F3410366F30003A14ACD
:1051C80066F3492366F38A2316702B809E4B1A7860
:1051D80042F0C0021A705A7866F3C3025A70FEF79A
:1051E800ABFC9A481EF050FD99481EF04DFD9948B9
:1051F8001EF04AFD984831464122FBF7CBF81823A8
:105208007343964A0136D15C082E01F0DF016FF333
:105218000411D154F3D10023914903EB0312885CA4
:10522800013300F0DF006FF38610072B8854F3D1A9
:105238008C4B1A786FF345121A709A7F6FF34512E8
:105248009A7793F83C206FF3451283F83C2093F843
:105258005A206FF3451283F85A2093F878206FF399
:10526800451283F8782093F896206FF3451283F857
:10527800962093F8B4206FF3451283F8B42093F87E
:10528800D2206FF3451283F8D220774B1A7802F0B8
:10529800DF026FF386121A705A7C02F0DF026FF396
:1052A80086125A7493F8222002F0DF026FF38612F6
:1052B80083F8222093F8332002F0DF026FF386127E
:1052C80083F83320694B5A786FF345125A701A786D
:1052D80002F0BF026FF345121A701A7D6FF3451280
:1052E8001A75DA7C02F0BF026FF34512DA740023F4
:1052F80011E04FF4D0615943342000FB02115C489F
:10530800013209188878202A6FF382008870F0D15A
:105318000133022B01D00022EBE708225548002177
:10532800FBF738F8544B00221A70544F387800288D
:1053380046D12A78524B02F00202D2B2CAB1424A8E
:10534800517860F3C30151701A88CA3042F0800264
:105358001A801FF0E1FAC6201FF0DEFA1FF02AFBC0
:10536800374A13780BB90CF0CFFEFEF785F8FEF735
:1053780091FD444A2B8811786FF341036FF30001C4
:105388006FF3000311704048002140222B80FBF787
:1053980001F83E481EF078FC3D481EF075FC2D488B
:1053A8001EF072FC3B481EF073FC082231480021B5
:1053B800FAF7F0FF304A00231370374A13709AE067
:1053C8002E7806F00203DBB293B916F001060FD16E
:1053D8002E481EF059FC3B78F0B2334113F0010F10
:1053E80003D0FEF7E5F90CF00DFD0136082EF2D1D9
:1053F8002B78234E13F0010F55D0FEF7DFFC3388CE
:1054080043F002033380FEF775FA1B4B1F78002F19
:1054180046D1CA201FF080FACD201FF07DFA3388CC
:105428001E4867F300033380164B1A7842F00102D6
:105438001A701EF029FCFEF71FF834E0D11800207E
:10544800901100203E1A0020983A0020BC1A002033
:1054580080180020C1180020DF18002028390020FB
:105468005F380020B73A0020FD370020B037002011
:105478001C3D0020B11800207C1800207E18002058
:105488005A1A00207F1800207C1A0020112F0020B3
:10549800351A0020741A0020C41A0020721900203E
:1054A8000120FEF789FB2B7803F00202D2B212B377
:1054B8008B4A12782AB113F0010F02D10220FEF7AD
:1054C8007BFBFEF7ADFE874987481EF0FBFB86494C
:1054D80086481EF0E1FBFEF749FB834984481EF02D
:1054E800DBFB844982481EF0E2FBFEF7D9FA8248CA
:1054F8007D491EF0F2FB7B4980481EF0CDFB8049B8
:105508000B780BB9FEF75AFA637803F08003DBB225
:10551800DBB92B7803F02403042B06D143F6EC20E7
:105528000CF01AF908B106200DE0FEF7A1FC08B14D
:10553800052008E00CF0D2FE08B1032003E001F0DA
:105548008DF810B10420FEF737FB6E4B1B781BB1AA
:1055580063786FF3C71363706B4A137813B16B4B9F
:105568001B78CBB12B786A4C03F04403402B13D142
:105578000021BF3300933F200B4602220191029184
:105588000CF068F9238843F6CE2043F00403238007
:105598000CF0E2F85F4B18705B495F4E0B789BB1DB
:1055A8005A4B197881B92A78594B02F04002D2B285
:1055B80052B11A8861F382021A80337823B943F60C
:1055C800CE200CF0C9F830702A78514F02F0040050
:1055D800C0B2524B002872D002F02000C0B24D4C2D
:1055E80080B11A78002042F0C0021A70FDF772FEEE
:1055F8002378002B69D13A8863F3820263F345125A
:105608003A8062E0D20052B219789211D2B241F0D7
:10561800C00112F0010F197003D0C9B260F3C711AD
:10562800197012F0020F03D01A786FF386121A70ED
:105638001B783A4A03F04003DBB21BB9537843F0B6
:10564800080353700120FDF745FE43F6CD200CF00A
:1056580083F8C0B20128307002D12F4B02221A7091
:105668002478002C31D1FEF787F9FF23022200931A
:10567800402021462346019402940CF0EBF82B8835
:1056880043F6CD2043F020032B800CF065F8214B26
:105698001B4A18701D4B14701A780AB1013A1A7017
:1056A800197891B9184A13787BB1FF2300934120E8
:1056B80002220B46019102910CF0CCF805E01A7811
:1056C80042F0C0021A70FDF705FE0CF0B7FD144851
:1056D8001EF008FB134B38BB1A7860F3820226E0F1
:1056E800C41A0020D4180020351A0020C118002040
:1056F800641A002021190020741A0020B91800200B
:1057080090110020324D0020471A0020C51A0020B1
:105718005A1A00203E1A0020DE180020983A00206D
:10572800291900207F1800201A7842F004021A7004
:105738006A78614812F001011A780CBF61F34102DE
:1057480042F002021A705D491EF0C7FA5C495A48D5
:105758001EF0ADFA58485B491EF0A9FA3378012BC0
:1057680040F0A7802B8800246FF349236FF38A2326
:105778002B80554B21461C7041225448FAF70AFEEB
:1057880053481EF081FAFEF7D7F94D481EF07CFA0F
:105798004C481EF079FA182363434E4A0134D15C11
:1057A800082C01F0DF016FF30411D154F3D1002369
:1057B800494903EB0312885C013300F0DF006FF303
:1057C8008610072B8854F3D1444B1A786FF345128F
:1057D8001A709A7F6FF345129A7793F83C206FF30B
:1057E800451283F83C2093F85A206FF3451283F84A
:1057F8005A2093F878206FF3451283F8782093F8AD
:1058080096206FF3451283F8962093F8B4206FF32F
:10581800451283F8B42093F8D2206FF3451283F829
:10582800D2202F4B1A7802F0DF026FF386121A701B
:105838005A7C02F0DF026FF386125A7493F8222022
:1058480002F0DF026FF3861283F8222093F83320E8
:1058580002F0DF026FF3861283F83320214B5A7867
:105868006FF345125A701A7802F0BF026FF34512AF
:105878001A701A7D6FF345121A75DA7C02F0BF02AE
:105888006FF34512DA74002311E04FF4D0615943E5
:10589800342000FB02111448013209188878202AA4
:1058A8006FF382008870F0D10133022B01D00022FF
:1058B800EBE709B0BDE8F08F8E330020641A0020B2
:1058C80080180020BC1A0020DE180020DF180020F5
:1058D800C1180020283900205F380020B73A00207E
:1058E800FD370020B03700201C3D00202DE9FF4186
:1058F80004460D460CF0CCFC9E4B1A1992F88070A9
:105908009D4A98461278AA2A0AD1A7F14F03DAB21B
:105918000B2A00F2A981994A5BB29A4040F1A4810E
:10592800974B0C2202FB04335A7A0833AA42C0F080
:105938009B81FF2A00F09881FF229A70914808EB1A
:10594800D403214693F888511EF0F9F90646002839
:1059580040F08A8104F007031D41502F05F001052E
:1059680000F0228114D8462F00F0EE8009D8412F8C
:1059780000F09A80452F00F017812D2F40F072819A
:1059880034E0482F00F0C1804F2F40F06B810EE0CB
:10599800542F63D006D8522F00F08680532F40F042
:1059A80061811CE0A7F15903012B00F25B81764865
:1059B80021461EF0C4F90646002840F055815A2FAA
:1059C80001D1724802E0592F04D1714821461EF0D6
:1059D800A0F950E121466D481EF09BF9F5E76D48A6
:1059E80021461EF0ACF9002800F03E816A482146A5
:1059F8001EF0A5F90746002840F036812146664882
:105A08001EF087F9654821461EF08EF9012602220C
:105A18004DB1A419142039463B46009201960294D0
:105A28000BF018FF27E129463346671C0A2000922D
:105A3800019602970BF00EFF2046FCF799FB3946BA
:105A480002462B4613200095FCF758FE12202946E3
:105A58002A4633460095FCF751FE0CE14E48214694
:105A68001EF06DF90746002840F005810126022244
:105A780031463346A5193E200092019602950BF057
:105A8800E9FE2046FCF774FB294602463B461420F3
:105A98000097FCF733FE21463F481EF03AF92146AD
:105AA8003E481EF041F9E6E03A4821461EF047F923
:105AB8000646002800F0DF80374821461EF03FF9EF
:105AC800064628B92046FDF7F5FC002840F0D380AB
:105AD800002D40F08E802046FEF7A4F9002840F003
:105AE800C5802046FEF78CFB2D4BDB7803F02003A6
:105AF800DBB20BB92B4B1855412F00F08880522F81
:105B080040F0B0802046012183E0234821461EF062
:105B180016F928B92046FDF7CDFC002840F0A480EE
:105B2800002D66D12046FEF77DF9002840F09E80C2
:105B38001B4BDB7803F02003DBB2002B67D1194B3A
:105B4800032283F8402062E0134821461EF0F7F84C
:105B5800064628B92046FDF7ADFC002840F08B80AA
:105B68002046FEF75FF900287ED1002D41D120465E
:105B780003214EE0CC2900203D1A0020000030808F
:105B8800A02B0020D418002044280020C42700207F
:105B980004280020351A0020641A00206C1A0020FE
:105BA8009C370020DF180020354821461EF0C7F832
:105BB800064600285FD02046FDF754FE20B1214656
:105BC80030481EF0A6F84FE0502F28D12E4B1B78F6
:105BD8002BBB2046FDF732FE08BB2C4821461EF0A1
:105BE800AEF8064620B92046FDF764FC002842D1ED
:105BF80015B1204602210CE02046FEF701FB244B9C
:105C0800DB7803F02003DBB20BB9224B1855204692
:105C18000021FEF7FDF9061E18BF01262BE02046DD
:105C2800FDF70CFE0546F8B91B4821461EF087F81B
:105C38000646D8B92046FDF73DFC0746D8B91648B0
:105C480021461EF066F8154A135D8BB910494E7847
:105C580006F02006F6B26EB908EB040393F800319B
:105C6800135508E0012606E0002604E02E4602E06F
:105C78003E4600E01E46304604B0BDE8F08100BF55
:105C8800351A002072190020C41A0020641A002056
:105C98009C370020DF180020C11800207C1A002043
:105CA800032210B505490648FAF74AFE0548064991
:105CB8000222BDE81040FAF743BE00BF22250020AB
:105CC80004020020090200202025002070B5844C21
:105CD800237813F0010F0AD00CF0A6F838B1002091
:105CE800804902F09FFE804B8048197849E0804D3A
:105CF8002B78002B4AD00CF09DF8002846D07D4B1D
:105D08001B7873B97C4B5B7813F0010F09D00CF04A
:105D180083F830B9237803F02403042B01D103302E
:105D2800BEE0764C207870B10020754902F07AFE0A
:105D380021780122734802F09BFE00201021621C8A
:105D480007F090FA02E0704902F06CFE6F4C684868
:105D580007F0D6FA2378002B00F018810CF064F8CD
:105D6800002800F013816A496A481022FAF7E8FD12
:105D780068485B21FAF78CFB002800F0078121783E
:105D880001308322BDE8704002F072BE624C237875
:105D980003F00503012B5DD10020604902F042FEAB
:105DA800202110225E48FAF7F5FA601D5D490322AA
:105DB800FAF770FD40BBE01C5B490222FAF76AFD66
:105DC80030B95A48FAF736FD5849024654480BE0AC
:105DD800E01C57490222FAF75DFD40B95548FAF729
:105DE80029FD544902464E48FAF7AAFD0EE0E01C88
:105DF80051490222FAF74EFD30B95048FAF71AFD18
:105E08004E4902464648EFE7FFF74AFF6278303AC4
:105E1800D3B2092B00F2BA803F4B9B78303BDBB200
:105E2800092B00F2B3800A2101FB0231C9B2002913
:105E380000F0AC80374BFF220C291A7740F2A6807D
:105E480010295A7740F2A28013299A7740F29E804F
:105E5800DA7770BD3A4C237803F00203DBB213B152
:105E6800002038498EE0234E3378EBB9224B5B781B
:105E780013F0010F18D00BF0CFFFA8B932481DF06E
:105E880031FF60B12268314B02EA03033BB918F0D5
:105E980003FA20B9E37803F04003DBB223B1002012
:105EA800BDE870400AF0A6B8337863B90BF0B4FFC8
:105EB80048B1274B1B7803F00603042B03D02B783B
:105EC8000BB90120ECE7FDF7D3FF10B10020214901
:105ED80058E0214B1D78002D42D0204952E000BFE8
:105EE8005A1A002029EC02087C1800200002002021
:105EF8007E180020C01C0020811D00200A1C0020E4
:105F080044C202080502002002C20208C41A002086
:105F180023C20208F40100201D2500204BC70208F7
:105F280004020020A4470308A8470308AEC70208D4
:105F3800AB4703088DC70208AE4703086CC70208C1
:105F48009C370020A2D60208291900203000000F33
:105F58007F180020D4D402089511002065C20208D9
:105F68000B4802F00EFD0A4802F002FD094802F053
:105F7800FFFC1CF097FBE37803F02003DBB22BB1A6
:105F880005492846BDE8704002F04CBD70BD00BF11
:105F9800141D0020341C00205DC10208054B1B782D
:105FA800D8019B015BB2DB1140B243EAE070C0B29A
:105FB800704700BF5A1A002070B50E4686B04100DF
:105FC8000122054601F5E97105A80BF0D6FB002171
:105FD800012E8DF815104FF0FF0205F1010305D1D0
:105FE8000092019102930920FB3A04E0009201918A
:105FF80002931E2004220B460BF02CFC05A84249F4
:10600800FAF7CCFA50B105A84049FAF7C7FA28B10F
:1060180005A83F49FAF7C2FA002872D105A83C49F9
:10602800FAF7BCFA3B4B0446F8B95A78214642F0D5
:1060380010025A70FF23022200930190FE3B029047
:106048003D200BF007FC4D200BF0D2FF691C01220C
:10605800234612200094FCF751FB122021462246C9
:1060680001230094FCF74AFB03E05A786FF304120B
:106078005A700024284BE35C552B07D1284621464B
:1060880015F00FFD10B1204615F0FAFC0134112C63
:10609800F0D1002E32D121482149224AFDF73CFD9A
:1060A8001F48214911F08EFCC0B10BF0B5FEA8B90C
:1060B8001D4807F05FFD88B905A81349FAF76EFA7D
:1060C800012320B9009318481849154A04E01648D6
:1060D8001649134A00933346FDF7F4FC144B104954
:1060E8001D700023009305330193124B0D4A1B7852
:1060F8000A4802930D4B07F0D1FC02E00E4B002238
:106108001A7005A806B070BD21480308B1470308F6
:10611800F7490308983A0020ED390020281C002090
:10612800111D0020041D002088180020ED1B0020F0
:10613800A73B0020C21C0020B018002007B5410072
:10614800012201A801F5E9710BF017FB002301A852
:1061580004498DF80530FAF721FAD0F1010038BF6B
:1061680000200EBD2148030807B54100012201A8FF
:1061780001F5E9710BF001FB002301A804498DF832
:106188000530FAF70BFAD0F1010038BF00200EBD38
:10619800B449030870B5154B04461B1893F8805092
:1061A800B1B1134821461DF0CAFD88B911482146EE
:1061B8001DF0AFFDA5F15903DBB2012B0CD94F2D12
:1061C8000AD0542D08D021460B481DF0A2FD07E047
:1061D800084821461DF0A8FD074821461DF0A4FDEA
:1061E80004480649BDE870401DF056BDCC29002082
:1061F800D418002029190020C9180020741A00207A
:10620800024B1878C0F38000704700BF7F18002049
:10621800024B1A8860F308221A8070475A1A002025
:10622800034B5878C00140B2C011C0B2704700BFDC
:106238005A1A0020014B1878704700BF7E180020BA
:1062480030B5457800230021C218917055FA03F142
:1062580011F0010F08D0064959188C7C017804EA1E
:106268000101A14208BF91700133042BEBD130BD6D
:106278000A1C002046F6753104220BF07EBA000095
:1062880070B5104C0546112220460021FAF782F815
:10629800002004F8010C2A78103414F8011FC3B246
:1062A80091420BD152B10849013301F8013B112247
:1062B80046F6C553BDE8704002F000BB0130042823
:1062C800EBD170BD0B1C00200A1C00201FB520B1AB
:1062D800134B1A8842F480521A80124B00245A78C1
:1062E800214642F010025A70FF23022200933D20FB
:1062F800FE3B019402940BF0ADFA4D200BF078FEB2
:1063080040210122234612200094FCF7F7F91220BD
:106318002146224601230094FCF7F0F91FBD00BF77
:106328005A1A0020983A00202DE9F3412D4C0722F3
:10633800E37849F2C02702FB003349F2E120DBB2DF
:1063480018180BF009FA257964795FFA80F80026A5
:1063580048FA06F313F0010F3AD03946042201A88F
:106368000BF00BFA9DF804009DF805309DF8061017
:106378009DF8072000282BD0002929D0002B27D0F2
:10638800002A25D0934204D19C4221D185421FD3B3
:106398000FE09A4210D99C421AD3944218D89C42D2
:1063A80001D994421AD39C4201D1854216D2944213
:1063B8000ED18D420CD811E09C4201D185420DD2FC
:1063C800944201D18D4209D99C4207D8944205D301
:1063D80001360437082EBBD1002000E00120BDE8BB
:1063E800FC8100BFA04A002010B5044649F21930CC
:1063F80000EBD4000BF0B0F904F00704C0B2204160
:1064080000F0010010BD70B5C30849F219355D19D7
:10641800044628460E460BF09FF904F00704C0B264
:10642800012126B9A14040EA0101C9B202E0A14018
:1064380020EA01012846BDE870400BF083B900004E
:10644800F0B57D4B95B0DE78082200EBC606F6B2B3
:10645800F10001F5FE4104A848310BF08EF9774BA5
:10646800774C1A78002304A9C95C312905D1303941
:10647800994041EA0202D2B205E0302903D12F390E
:10648800994022EA01020133082BECD122706C48B2
:106498006C496D4AFDF740FB6A4B1B7813B96A4B90
:1064A8001B78F3B16748694911F08CFA68B10BF0B1
:1064B800B3FC50B9654807F05DFB30B90123634868
:1064C8006349604A0093FDF7FDFA00230093023305
:1064D8000193FD3302935A485A495B4A5C4B07F0D3
:1064E800DDFA06EB0611002501F50041257004A828
:1064F80001F5847111220BF040F92C462F46554BBB
:106508000135E35C542B36D104AB1B5D312B03D131
:10651800204615F0BDF938B104AB1B5D302B2AD1EC
:10652800204615F0B5F930B34FB9FF230093342056
:10653800394604223B46019702970BF08BF904AFCA
:10654800385D2146303815F0B1F93B5D0127312B14
:106558004FF0030305D100932BB201970293352026
:1065680004E000932BB20197029336200021042205
:106578000B460BF06FF90134112CC0D1B10101F5B4
:10658800044104A8C03140220BF0F7F8113C04ADD7
:10659800274615F8013BE6B20134302B03D13046CB
:1065A800FFF722FF38B115F8013C312B2CD13046CA
:1065B800FFF71AFF40B34FB9FF2300933420394641
:1065C80004223B46019702970BF044F915F8011C89
:1065D80030463039C9B2FFF716FF15F8013C0021E3
:1065E800302B4FF0FF0305D1009323B201910293A2
:1065F800372004E0009323B201910293382004224B
:106608000B460BF027F90127402CC2D1124D6B78AD
:1066180003F00403DBB263B1403C2046FFF7E4FE1D
:1066280038B90134E4B2402CF7D16B7860F38203B7
:106638006B7015B0F0BD00BFA04A00207E18002086
:10664800281C0020111D0020041D0020881800208F
:10665800ED1B0020ED390020983A0020014B1878F6
:10666800704700BF951100202DE9F04F4E4B0022D6
:106678001A704E4A85B01678002E40F091804C4B27
:106688004FF4B468DA78997808FB02F24FF03C08C6
:1066980008FB01285A78474F90441FFA88F8BA46F1
:1066A8006CE03AF815303C24DAB2544304EB132476
:1066B8004C44A4B2042CEEB207D842F25A7398455F
:1066C80003D904F51C546034A4B2444511D949F2E5
:1066D800E0200BF041F8C8EB0403834209DC364B99
:1066E8001A787B1993F87030934302D02E4901230E
:1066F8000B702F4AD378B34232D142F26073B4FBA5
:10670800F3F203FB12439BB2434523D12B4B9B78F7
:1067180013F0090F44D12A4B5B7803F08003DBB2F6
:10672800002B3DD1274B5B7803F00203DBB2002B33
:1067380036D1254B1A781BEA020F11D1019900981E
:1067480041EA02021A70FFF7EFFD48B90098FFF717
:1067580077FE05E01C4B02991A7801EA02021A70CA
:10676800013509F5B469072D1FFA89F999D1039EF6
:1067780007370136082E0AF10E0A11D04FF0010B27
:106788000BFA06FB5FFA8BF301936FEA0B03F2B285
:10679800DBB24FF00009009202934D46039680E762
:1067A80005B0BDE8F08F00BF95110020CD1A00207C
:1067B800A04A0020CE1A00207E1800209C37002016
:1067C800A73A002086310020CC1A002073B50C4669
:1067D80001EBC001C9B2C90001F5FE410546082216
:1067E800684648310AF0C9FF104B002003EBC40289
:1067F800121B521982F870001DF80020312A0AD1A4
:106808000121814003EBC402121B521992F87060F7
:10681800314382F8701001300828EDD169463122E1
:1068280030231DF094FAC0B27CBD00BFCE1A002000
:1068380000B501EBC001C9B2890191B001F504416D
:10684800C031402268460AF098FF4020694631224C
:1068580030231DF07CFAC0B211B000BD7FB501EB4A
:10686800C001C9B201EB011101F50041112201A8D3
:1068780001F584710AF081FF112001A9312230232A
:106888001DF065FAC0B207B000BD00002DE9F8435D
:10689800002634462BE021462846FFF797FF21467D
:1068A80081462846FFF7C4FF214640EA09092846E1
:1068B800FFF7D4FF5FFA89F949EA000010F0FF0FEB
:1068C80005D04046394602220AF057FF03E04FF050
:1068D800FF33A8F800300135EDB20237072D08F173
:1068E8000208D8D10134E4B20E3E082C07D0054B7B
:1068F800C6F5FC47C6EB0308D8370025CBE7BDE84B
:10690800F88300BFCE1A002010B51EF087FA4FF4A6
:1069180080301EF0A3FA1EF0BBFB0128044628D1E4
:1069280010201EF09DF902201EF08EF900201EF0A6
:10693800D5FA00201EF0E6FA4FF480601EF0D8FA6F
:106948004FF440401EF0E8FA4FF480304FF4E01165
:106958001EF0A0FA20461EF0A9FA39201EF084FB8A
:106968000028FAD002201EF0A7FA1EF0AFFA082875
:10697800FBD17C2001211EF041FB46F601200121BC
:106988001EF03CFB0C4801211EF044FB0B48012182
:106998001EF040FB042001211EF03CFB7E201EF06F
:1069A80063FB38B11EF08AFB054B04211A7861F3AA
:1069B80044021A7010BD00BF0340060020080818E2
:1069C800154D002010B50C46014620B110220C4888
:1069D800F9F7B6FF04E00A4820211022F9F7DAFC9B
:1069E80034B1084821461022BDE81040F9F7A8BF85
:1069F800044820211022BDE81040F9F7CBBC00BFA5
:106A0800F40100200402002010B5FF2B1446029A5E
:106A180003D0421802F8013C08E06FF07F439A4225
:106A280004D01314437013128370C2701AF03AFD25
:106A380002E07F201EF05EFE1AF020FD0028F8D14B
:106A4800ACB10B4890F82010163001F00F011AF085
:106A580029FD02E07F201EF04DFE1AF00FFD0028F0
:106A6800F8D1044B93F8693013F0010FE9D110BD48
:106A7800580C0020304C002010B50A4B002203EBC4
:106A8800C003013B1046084951184C7813F8011F00
:106A98008C4205D10130C0B20C320828F3D1F7304E
:106AA80010BD00BFC6570208A02B002070B50D4CC2
:106AB80005460E464FF4007200212046F9F76AFC9D
:106AC8002A46314604F50070F9F7BCFB642024F827
:106AD800035C1CF0B9F80023A4F82D33024B6422A0
:106AE8001A6070BD994D00202825002010B5054C6E
:106AF800002120464FF40072F9F74CFC0023A4F85B
:106B08002D3310BD994D0020164B2DE9F0415D8ABB
:106B180007462846FBF704F81349FBF70DF9134B12
:106B2800134E1860D723B5FBF3F5EDB28222294640
:106B38000446F01901F09CFF2846FAF7F5FF0146D4
:106B48002046FAF73BFF0B49FBF742F8FBF706FA3A
:106B58000337BE19C1B281223046BDE8F04101F0C9
:106B680087BF00BFDC2E002000005743781B0020A1
:106B7800F40100200000204170B54B4D2868FAF759
:106B8800DBFB45A3D3E90023FAF776FAFAF7C2FE4E
:106B9800FAF7D2FB42A3D3E90023FAF721FC3EA37C
:106BA800D3E90023FAF746FDFAF7B4FEFAF7C4FB77
:106BB800FAF7CEF9FAF7AEFE3C4906462860FBF72D
:106BC800AFF920B13046FBF7C9F9C4B25EE03046F0
:106BD8003649FBF7B9F950B130463549FBF7A0F90A
:106BE80028B13046FBF7BAF9C0B2441C4EE0304633
:106BF8002F49FBF7A9F950B130462E49FBF790F918
:106C080028B13046FBF7AAF9C0B2841C3EE03046F2
:106C18002849FBF799F950B130462749FBF780F925
:106C280028B13046FBF79AF9C0B2C41C2EE03046B2
:106C38002149FBF789F950B130462049FBF770F933
:106C480028B13046FBF78AF9C0B2041D1EE0304671
:106C58001A49FBF779F950B130461949FBF760F941
:106C680028B13046FBF77AF9C0B2441D0EE0304631
:106C78001349FBF769F948B130461249FBF750F957
:106C880020B13046FBF76AF9C0B2841D0A202146BC
:106C9800BDE870400AF056BD736891ED7CFF7F40F7
:106CA8000000000080842E417C1B00200000104161
:106CB8000000F0410000484200008E420000B84247
:106CC8000000E0420000F2422DE9F04F9DB01AF0BA
:106CD8007FFB09201CF054F91BF03AFF4FF4614088
:106CE8001CF08AF909201CF007FA0022A3484FF487
:106CF80080411EF01AF8A24800211EF0E3FBA149CA
:106D080004224B78DFF8A0E26FF300034B709E4B30
:106D18009E4C1A705A715A709A70DA701A719A7178
:106D2800DA719B4B033A1A709A4B00201F328EF887
:106D3800000020705A7105900546069006467F208F
:106D48001EF0D8FC23780E2B01F2B681DFE813F091
:106D58000F004F009500E0007902DE03300485043F
:106D6800EA06DC07EF075808B108D00882098A4EFE
:106D78008A48317801F00F01013149014118FFF7C4
:106D880021FE337813F00F0308D1854A92F80123C6
:106D9800012A41F09181834A138024E0012B03D119
:106DA8007F4B93F819330BE0022B04D17C4B93F8FB
:106DB8000D33032B05E0032B06D1794B93F80D33E4
:106DC800012B41F079810EE0774901220A7077485A
:106DD8004FF400711DF0A9FF754BC8221A60337873
:106DE8006FF30303BFE333785A1C01F05FB8704BAD
:106DF8001A6822B96D484FF400711DF096FFDFF84C
:106E080098816C4898F8001001F00F010131490190
:106E18004118FFF7D7FD36B198F800305A1C62F3D5
:106E2800030388F800305F4B00221A8098F800109E
:106E380001F00F02022A03D11A7842F010020AE088
:106E4800042A03D11A7842F0040204E0052A05D185
:106E58001A7842F040021A7001F02EB9062A04D1BD
:106E68004D4B6FF3030119707EE301F00F0101220E
:106E780012FA01F1198001F01FB9474E4E483178D6
:106E880001F00F01013149014118FFF79BFD96F808
:106E9800008008F00F08B8F1070F27DC18F0010F81
:106EA800464B02D00020588002E04FF0FF31598055
:106EB8004FEA6809062209F1010902FB09394FF076
:106EC800FF32A9F802204046FFF7D6FDFF2806D07A
:106ED8003B4B03EB40005823437401F0EDB800230B
:106EE800A9F8023008F1010801F08AB8002110223F
:106EF80013A8F9F74FFA0FA800211022F9F74AFA58
:106F080023780133237033786FF3030301F07BB8E0
:106F1800DFF884A09AF8008018F00F0840F03F814D
:106F2800284E337803F04003DBB2F3B926486FF0FC
:106F38007F43817A0122009301F00F01FF23FFF7BD
:106F480063FD224B93F8692012F0400F08D093F8A4
:106F58006C3013F0040F03D0337843F040033370E0
:106F68007378142262F3C7037370737813F0F80F01
:106F780030D0174800F12001A7E300BF00180140F6
:106F8800002C0140FE2E0020CC290020821B00206E
:106F98009311002028390020811B00200658020880
:106FA800A02B0020983A002058250020000C014012
:106FB80028250020A6580208865902081E3A0020F3
:106FC800F401002087370020580C0020304C0020A6
:106FD800A65A0208BC4B1B7803F04003DBB2002B17
:106FE80000F0D980DFF80483DFF8049398F80030C4
:106FF80013F00C0B30D1B54E6FF07F4396F82B1081
:1070080006F12100009301F00F0101220523FFF78B
:10701800FBFC96F84C104FF4860A06F1420001F08A
:107028000F010122FF23CDF800A0FFF7EDFC96F831
:107038004110FF2306F1370001F00F015A46CDF841
:1070480000A0FFF7E1FC042389F8003098F800302D
:1070580043F0080301F02EB803F00803DBB2002B5D
:1070680039D099F800A0BAF1000F03D0984800F180
:10707800400138E0954E6FF07F4B717D06F10B00B3
:1070880001F00F010122FF23CDF800B0FFF7BCFC8F
:1070980096F82B1006F1210001F00F0101220723B9
:1070A800CDF800B0FFF7B0FC96F836104FF4860321
:1070B800009306F12C00FF2301F00F015246FFF761
:1070C800A3FC98F800306AF3C303DBB243F004036F
:1070D80088F800305AE099F800C0BCF1000F08D0D9
:1070E8007B4800F16001FFF76DFC99F80020303211
:1070F80008E2764E6FF07F40717DFF23009001F02B
:107108000F0106F10B000122CDF80CC0FFF77CFC43
:107118009AF80030DFF8C4B103F0100A5FFA8AFA6F
:10712800DDF80CC0BAF1000F0CD098F800206CF311
:10713800820288F800205A1C62F303038BF800309F
:1071480000F0BABF96F82B106FF07F42009206F15C
:10715800210001F00F0101220C23FFF755FC96F8DE
:1071680036104FF4860300935246FF2306F12C0095
:1071780001F00F01FFF748FC9BF8003083F0100284
:10718800C2F3001262F304138BF80030042389F869
:10719800003000F091BF4E4800F1800195E2B8F14F
:1071A800010F3CD14A4800F1A001FFF70BFC002E6B
:1071B80000F082879AF80030444E5A1C62F30303A9
:1071C8008AF8003096F82B106FF07F4906F12100FD
:1071D80042460F2301F00F01CDF80090FFF714FC91
:1071E80096F82B1006F1210042460E2301F00F01FC
:1071F800CDF80090FFF708FC96F82B1006F1210057
:10720800424601F00F010F23CDF80090FFF7FCFB79
:107218003048802142461DF088FD00F04DBF2C48C3
:1072280000F1C001FFF7CEFB002E00F045872A4B86
:1072380096221A609AF800306FF303038AF8003038
:1072480092E1264E317811F00F0A16D1244800F148
:107258002001FFF7B7FB204B1B68002B40F02C8761
:1072680013A8F9F7E7FA40221346014613A801F0DC
:1072780023FA3378012200F019BEBAF1010F39D18F
:1072880012486FF07F4390F82010002200931630C8
:1072980001F00F01FF23FFF7B7FB01F077FA002891
:1072A80000F00A873378022262F3030333700D4B30
:1072B8001A7842F080021A700B4B5A7842F0020298
:1072C8005A7000F0F9BE00BF87370020580C002024
:1072D800A65A02080010014028250020811B002022
:1072E800865B02088C370020363C0020B45300200F
:1072F8003B55002001F00F0101F10E0303F00F03CD
:10730800012B44D89B4849014118FFF75BFB9A4879
:107318006FF07F4390F8201000221630009301F0A0
:107328000F01FF23FFF770FB1BF05AFA337803F0C5
:107338000F03022B13D116F07BFF002800F0BC8648
:107348008E4B1A7842F040026FF304121A705A7882
:107358006FF345125A703378032200F0A7BD16F078
:1073680051FF78B116F0F0FF16F0A8FE844B00200C
:107378001A7858816FF3C7121A703378042262F3AF
:10738800030333707F4B1A786FF3000263E5BAF199
:10739800040F4DD1DFF8DC914901DFF81082494430
:1073A8004846FFF70FFB98F80010774B01F00402EE
:1073B800D2B27AB941F004016F4883F800A088F886
:1073C800001090F836104FF4860300932C3001F02B
:1073D8000F01EEE293F800A0BAF1000F40F06C86BE
:1073E80065486FF07F45417D01220B3001F00F01A8
:1073F800FF230095FFF708FB64480122817AFF23E9
:1074080001F00F010095FFF7FFFA98F80030052208
:107418006AF3820388F800303378484662F303033E
:10742800337009F1A001FFF7CDFA554600F044BECC
:10743800DFF84481FF2398F8201000226FF07F497D
:1074480008F1160001F00F01CDF80090FFF7DCFA03
:107458002BB2072B18D1337808F121006FF30303FF
:107468003370237801220133237098F82B100E23F0
:1074780001F00F01CDF80090FFF7C6FA44488021CB
:1074880000221DF052FC0025424E96F86B3013F096
:10749800040F00F0118698F857106FF07F43002210
:1074A80000933D48FF2301F00F01FFF7ADFA96F86E
:1074B8006B303A4A03F00F03012B137003D1002DF0
:1074C80008BF01250CE0022B04D12BB2012B08BF09
:1074D800032505E0032B03D12BB2032B08BF072597
:1074E800ABB213F0010F02D02D4A3121517713F0BE
:1074F800020F02D02A4A3221917713F0040F00F0CC
:10750800DB853322264BDA7700F0D6BD1948254EA5
:1075180000F1C001FFF756FA96F80090DFF85C809A
:1075280019F00F090CD116F0E3FC98F8003069F354
:10753800000388F8003033785A1C62F30303337071
:1075480016F068FD98F8003013F0010F00F0B485CC
:107558000022154880211DF0E8FB0A4B00225A70D2
:10756800337862F30303337023780133237000F018
:10757800A3BD00BF865B0208580C0020363C0020E3
:107588008C370020AE3B00203B5500200100002036
:1075980000100140304C0020A50C00208637002048
:1075A800F4010020811B002000180140B453002082
:1075B8008648874E00F1E001FFF704FA0FA8F9F7B3
:1075C80039F90FA902468348F9F7BAF90021824828
:1075D800B18090F8C5106FF07F4300220093BB3054
:1075E800FF2301F00F01FFF70FFA7C4A92F86B10A6
:1075F80092F86C30327843EA012312F0010FB3801D
:1076080010D0A3F1EB0292B20A2A04D9A3F5E673CB
:107618009BB2282B02D8F3880133F38033786FF3B9
:10762800000333707378002B40F04685684AD2888F
:107638007AB16B4A1BA8117863F3030111702278A1
:107648008DF86F300132227028228DF86C201DF0E1
:107658008BFB0022F28000F02FBD624EDFF8ACA158
:10766800337803F004085FFA88F8B8F1000F15D1F1
:1076780009A841461522F8F78DFE5B4BCAF8008031
:107688001B684546CDF827303368474643F0040366
:107698003360564BA3F8368300F00EBD03F0800329
:1076A800DBB2002B67D1DAF80010002940F004851E
:1076B8004F48FFF787F94F484FF480511DF02BFBD7
:1076C800012806D04A4800F1A001FFF77BF900F035
:1076D800F3BC4649B1F83623002A43D0093146485D
:1076E800013AF9F72DF9444B03F1100113F8012B76
:1076F8000D2A01D00A2A02D1202203F8012C8B423C
:10770800F4D13E4B4FF03C0808FB073808F11E083F
:107718004046F9F78FF8414602463948F9F7BAF872
:10772800D8B9022F03D1336843F0100304E0032FC4
:1077380003D1336843F040033360327853005BB2BF
:1077480003EAC263DB173268DBB263F3C712326045
:107758001BB1FFF7CBF900F0AFBC0137FFB2042F24
:1077680008BF0227254B3C2606FB07363046F9F7AB
:1077780061F8314626E0DAF80080B8F1000F40F0F1
:107788009B84737803F02002D2B2002A40D11D4BAB
:1077980009A81A889B781C498DF82630ADF8242052
:1077A800F8F752FE114B5B7A302B07D1FFF79EF9A1
:1077B800336843F40053336000F07EBC09A8F9F73E
:1077C80039F809A9FFF772F900F076BC865B020860
:1077D800AE3B002008020020580C0020304C00204E
:1077E800811B00202C250020B3470308904D002062
:1077F800865C020800080140040200200C000020FA
:10780800994D0020B8470308BC47030828250020E5
:1078180003F04003DBB2002B40F08980B14800F14F
:107828006001FFF7CFF8B048F9F704F88046AE4991
:10783800AE484246F9F72EF8002873D1AC4B4344C2
:107848005B7A302B6ED1FFF751F93368DFF8D092AD
:1078580043F48043336099F82B106FF07F43009313
:1078680009F12100082301F00F010122FFF7CCF8EC
:107878006423CAF800307F201DF03CFFDAF800309E
:10788800002BF8D1984699F88E10D633994E89F87E
:1078980086304B3B6FF07F4A89F88730964801F075
:1078A8000F0142467433CDF800A0FFF7ADF896F803
:1078B800B91106F5D670033001F00F014246FF23D7
:1078C800CDF800A0FFF7A0F896F8C41106F5DD7012
:1078D80001F00F014246FF23CDF800A0FFF794F80E
:1078E80096F8CF1106F5E270013001F00F0142461B
:1078F800FF23CDF800A0FFF787F896F8DA1106F510
:10790800E87001F00F014246FF23CDF800A0FFF711
:107918007BF899F899107948CDF800A001F00F018B
:10792800424646E07648F8F785FF75494AE796F8F3
:1079380002B0DFF8EC910BF0020B5FFA8BFBBBF1A6
:10794800000F3AD199F82010FF236FF07F4809F112
:10795800160001F00F015A46CDF80080FFF754F8E1
:10796800684B93F86B3003F00803DBB2002B00F090
:10797800A38399F82B10012209F1210001F00F01CE
:107988000323CDF80080FFF73FF83368554843F4E8
:10799800003300F180013360FFF714F855485A4668
:1079A80090F8E51100F5EC70CDF80080033001F097
:1079B8000F01FF23FFF728F87EE3CAF8008099F843
:1079C80020106FF07F4300934246FF2309F1160011
:1079D80001F00F01FFF718F82AB241F211139A4289
:1079E8001DD1434B5B7A302B13D1FFF77FF83368F7
:1079F800454668F3514368F38E3368F34D3333607B
:107A0800414B1A7868F303021A7023780133237004
:107A180052E33E48F8F70EFF3C49FFF747F8394E66
:107A280096F86B3013F0040F00F0468325B93848F8
:107A380020211022F8F7AEFC7F201DF05BFE99F89C
:107A480057106FF07F43002200933248FF2301F064
:107A58000F01FEF7D9FF96F86B202F4B02F00F02AB
:107A68000D2A1A7005D125B92C4A412191754FF478
:107A780080551A78062A08D12AB2B2F5805F04D157
:107A8800264A3621D1754FF488551A78082A08D124
:107A98002AB2B2F5885F04D1204A3821117641F222
:107AA80010151B780B2B09D12AB241F210139A42F8
:107AB80004D11A4B2A225A7641F211150D486FF05B
:107AC8007F4390F8F0110022009300F5F370FF2334
:107AD80001F00F01FEF798FF96F86B3013F0010FD5
:107AE800AAD0E9E2865C02081A010020994D00201C
:107AF800904D002001000020DC0C0020E70C002045
:107B0800FC000020304C0020811B002038010020A0
:107B180004020020A50C002086370020F401002074
:107B2800580C0020A34B1A7842B300221A700F2079
:107B3800FAF78AFA06460A20FAF786FA9E4B9F4910
:107B480058824A7812F0010F18D06436301A5883D8
:107B58009B4B1A78642A01D19B321A701B78984E75
:107B6800FF2B0BD00A21B3FBF1F1964B1931198089
:107B780095481DF0A7FC337801333370DFF8648231
:107B880098F8003013F00F0612D18E4B19228B484B
:107B98001A804378192143F0010343708A481DF085
:107BA80091FC8A4800F12001FEF70CFF04967CE264
:107BB800012E68D1804B5A8BA2F1690189B2112933
:107BC80008D8049911F0010F04D141F00101C9B29C
:107BD80004910592049A12F0020F0DD15B8A7C4A37
:107BE8001380A3F5C263023B9BB2D72B04D8049839
:107BF80040F00203DBB204931B20FEF785FF0599D2
:107C0800744B0AB2632A05DD642192FBF1F230322B
:107C18001A7401E0092A0CDD059A11B2642291FB5D
:107C2800F2F002FB10120A2012B292FBF0F230328C
:107C38005A74059802B2642092FBF0F100FB1121FE
:107C48000A2209B291FBF2F002FB101230329A7448
:107C58005B4B1B78FF2B08D158495B484B786FF377
:107C680000034B7000211DF02DFC049A032A40F0FC
:107C780023825248002143786FF30003437052482F
:107C88001DF020FC11E2022E03D1534BC8221A60CA
:107C98000BE2032E16D1504B1B68002B40F00C82D0
:107CA8004A4800F14001FEF78DFE1B20FEF72CFF2D
:107CB800414B5B8AA3F51E630F3B9BB2542B00F22A
:107CC800FB81F2E1042E0CD13B4B988A0FF07EFA2F
:107CD800002840F0F1813D4800F16001FEF772FE96
:107CE800E3E1052E07D1344B988A0FF06FFA032889
:107CF80040F0E281D9E1062E40F0D78122786FF377
:107D0800030301322270D5E1344800F12001FEF767
:107D180059FE334B1B78002B00F0CE8123780133BA
:107D28002370304B1A786FF30302FFF794B82D4E87
:107D3800DFF8A480337813F00F021AD12A4800F133
:107D48002001FEF73FFE2948F8F774FD274902464F
:107D58002748F8F777FA2548F8F76CFD254BA3F87C
:107D6800160233785A1C62F3030333701BF0EEF9E2
:107D780091E0012A16D1D8F80030002B40F09C8100
:107D88001BF010FA012840F097811B48F8F752FDC4
:107D9800194902461948F8F77DFD002840F08C8102
:107DA80011486FE0D8F80020002A40F085810B21A7
:107DB8007BE000BF96110020DC2E0020FE2E002064
:107DC800901B0020540C0020002C0140465D020846
:107DD800841B0020F401002028250020C65D02082D
:107DE800801B0020811B0020065E02087401002011
:107DF80074350020345100209201002035510020B4
:107E0800874E337813F00F080CD186484146FEF7A9
:107E1800D9FD33785A1C62F303033370824BA3F8FD
:107E2800028049E1B8F1010F18D1804804211CF003
:107E380072FF002800F040817A4800F12001FEF727
:107E4800C1FD33784FF0FF315A1C62F303033370DE
:107E5800774B64221A60744B59802DE1B8F1020FF8
:107E6800DFF8CC811BD1D8F80030002B40F02481FA
:107E78006E4804211CF04FFF002840F01D816A4B1A
:107E88005880684800F14001FEF79CFD33785A1C81
:107E980062F3030333706423C8F800300CE1D8F8A8
:107EA8000020002A40F008810C21217062F30303AE
:107EB800A9E0604910234FF40052CB700D3B8B7042
:107EC8000A805D481CF0D8FE0A2200215B48F8F7BA
:107ED80061FA80201CF034FE237801332370504B64
:107EE8001A786FF303021A70514BC8221A60E3E044
:107EF8005348DFF848A100F12001FEF763FD9AF826
:107F08000030002B00F0D8804E48DAF80020444EAC
:107F18000260BAF8042082809AF8062082713178CB
:107F280011F00F0159D1DFF80881D8F800100029A5
:107F380040F0C2809AF80410A2F5A6524FF0640BE4
:107F4800103A0BFB01229AF805004FF00A0909FBC9
:107F580000200393F9F7E4FD3B49F9F7EDFE0246EB
:107F68009AF80200039BA0F5A65010380BFB030BF0
:107F78009AF80100354B09FB00B018600392F9F735
:107F8800CFFD039A01461046F9F71AFD304B1860E9
:107F9800F9F7D2F91EA3D3E9002382468B46F9F7F5
:107FA800A5FC002800F08880504659461AA3D3E95A
:107FB8000023F9F791FC00287ED0FEF7DDFD337829
:107FC80048465A1C62F303033370C823C8F80030CC
:107FD80009F0C2FBC0B207906EE001296CD10D30E8
:107FE8000799832200F044FD114BD3F80080B8F1C3
:107FF800000F61D140461CF0A3FD237801332370A4
:10800800337868F30303337056E000BFAFF30080A2
:10801800736891ED7CFF7F400AD7A3703D008040D4
:10802800811B0020665E02081E3A0020000C0140F9
:1080380028250020FA2E002000100140981B00205F
:10804800C65E02080402002000007A44941B002047
:108058007C1B00208448854E00F12001FEF7B2FC0D
:10806800F37913F0010F27D0DFF8488298F80090D1
:1080780019F00F0920D17E4B0A2259781878103947
:1080880002FB0011B1701979D878103902FB001180
:108098007170D9799B79103902FB0312327018F08C
:1080A800A7F9F37969F30003F37198F800305A1CC3
:1080B80062F3030388F80030DFF8FC9199F8006058
:1080C80016F001063EF43BAE6A4B01221A7019F015
:1080D800E1FF2378092B01D00D2B28D10120664917
:1080E80011F0C6FF654B664A5B7803F01F03D35C4B
:1080F800644A522B137002D1634B01221A70634BEE
:10810800634A03F1200153F8040B8B4242F8040B35
:10811800F9D1002117A811F0D5FF17A80D211AF0E1
:10812800B1FF5C4B1A78013202F003021A7099F819
:10813800006006F00206F6B2002E00F08B800FF009
:10814800A1FA13F03DFB06980322431C93FBF2F2BD
:1081580002EB42029B1ADBB20693002B79D1DFF8BF
:10816800488198F84960C246002E4DD0022E03D1AE
:1081780098F80130312B49D023780E2B13D146487B
:1081880046490522F8F786FB8246002840D1B21FEF
:1081980037484349F8F7D4FB344B5646DA7942F06E
:1081A8000102DA7135E00D2B03D13E483A49072226
:1081B80027E0032B22D13C4B002713F8012F2C2A50
:1081C80003D00137FFB2B742F7D113A832493A4674
:1081D800F8F7B6FB7B1C07E00AEB03025278303A4B
:1081E800D2B2092A03D80133DBB2B342F4D30AEB83
:1081F8000701FA430FA80231D21802E0264909A85C
:10820800721EF8F79DFB03E0069E02E0012600E0DF
:1082180000261E4B204A03F1100153F8040B8B4231
:1082280042F8040BF9D1214B214A03F1100153F80C
:10823800040B8B4242F8040BF9D1402388F8113023
:108248001C3B88F82230023B88F84B301AF0A2FC1D
:1082580000E0002699F8003003F0F5036FF30003FF
:1082680089F80030FEF76BBD065F0208A04A0020BF
:10827800861B002096110020D1500020D0500020ED
:108288005095020849380020801B0020F401002086
:10829800FB380020A73700203F4D0020BF470308C8
:1082A800444D0020981B00203E4D00200402002071
:1082B800504D0020811B0020184D0020AFF3008096
:1082C80010B5044640181146F8F756FA2046F8F754
:1082D800B1FAC0B210BD42540131C8B270470000B3
:1082E80010B50D4B0D4A1B780C460E2101FB0323DC
:1082F800997A39B101390523594301F56E51413154
:1083080089B201E043F6C1310019042209F035FAB7
:10831800201DC0B210BD00BF5553002020160020FC
:1083280010B5054B0C46197800190131042200F0EC
:108338009FFB201DC0B210BD5553002000F52A40F8
:1083480008B5D73009F008FA10F0FF0F14BF002065
:10835800012008BD10B50A4600210446FFF7B0FF0A
:1083680001462046FFF7DCFF114A01462046FFF789
:10837800A7FF232201462046FFF7ADFF014620460E
:10838800FFF7AEFF5B2201462046FFF7A4FF23223A
:1083980001462046FFF79FFF01462046FFF7A0FF52
:1083A8007C2201462046BDE81040FFF794BF00BF7D
:1083B800C547030810B55D220446FFF78CFF0D2260
:1083C80001462046FFF787FF0023235410BD38B528
:1083D8001D460C4640182C1911461A4600F048FB59
:1083E800E0B238BD2DE9F04118490446FFF7B2FF65
:1083F800174F0E263B78174D73430146EA5A20461D
:108408000423FFF7E4FF202201462046FFF763FF1D
:108418003B78014606FB035320469A7A0223FFF76E
:10842800D6FF202201462046FFF755FF3B7801463C
:1084380006FB035520466A7A0323FFF7C8FF014667
:108448002046BDE8F041FFF7B5BF00BFC8470308A5
:1084580055530020201600202DE9F047264E0E2205
:108468003378264F534337F90380FA1824494FF4D9
:108478007A73044698FBF3F8157AFFF76BFF4E22E0
:1084880001462046FFF727FF1E4B1C2202FB05353D
:108498005FFA88F8B8F1030F01460CBF05F1120224
:1084A80005F108022046FFF70BFFA146804600258C
:1084B80019E019F8013BA32B07D133780E2202FBF0
:1084C8000373204629465A7A08E0242B09D13378C9
:1084D8000E2202FB03739A7A204629460223FFF7ED
:1084E80076FF0135EDB24545E3D120462946BDE882
:1084F800F047FFF75FBF00BF55530020201600204C
:10850800D247030870950208074B187800F004005A
:10851800C0B240B11A686FF382021A60034B00229E
:108528001A70034B187870479C370020BC1B00203A
:10853800A41B0020054B00211970054B05481A683B
:1085480061F382021A601222F7F724BFBC1B0020D5
:108558009C370020A41B002038B5084C0849227815
:108568000546F7F76FFE23780021E954054B1A6892
:1085780061F382021A60207838BD00BFBC1B00205E
:10858800A41B00209C370020064A07491378112BAA
:10859800C85401D801331370044A136843F0040324
:1085A80013607047BC1B0020A41B00209C370020D0
:1085B800054B1B7813F0010F05D1044B181810F860
:1085C800010CFFF7E1BF7047BD1B0020465F0208A2
:1085D8002DE9F041334C002314F8101094F82A20A8
:1085E80001F00F0161F3030284F82A2004EB400034
:1085F80084F8293084F828304378DFF8B88063F3AA
:108608000712638C4FF4D277E38498F800302A2657
:108618007B4306FB0133244D2448E95A84F82A2079
:108628001CF04EFF98F8003094F82A207B4302F0A3
:108638000F0206FB0233EB1859881C48013989B22E
:108648001CF042FF01210A4618481CF009FF0121CD
:1086580016481CF0F6FE98F8003094F82A207B4360
:10866800120906FB02331248E95A1CF029FF98F850
:10867800002094F82A3057431B0906FB0376AD19EE
:1086880069880B48013989B21CF01CFF01210A4690
:1086980007481CF0E5FE06480121BDE8F0411CF042
:1086A800D0BE00BFBE1B0020525F02080008004079
:1086B80000340140EA1B002030B5164C94F82B50CA
:1086C800A38445F00105002384F82B50628484F8C4
:1086D800211084F8203019E0C55CA5F13002D2B22F
:1086E800092A08D9A5F14102D2B2052A9ABFA5F1F3
:1086F8003702D2B22A46084D013305EB420292F8FE
:10870800495392F84823257062700234DAB28A42DB
:10871800E2D330BDBE1B0020525F0208124B10B5D9
:108728009A8C0024DA8483F8294083F8284022466A
:1087380001210E481CF094FE64210C481CF0C0FE78
:1087480032210A481CF0C0FE0121224608481CF0CC
:1087580087FE642106481CF0B3FE05483221BDE8B7
:1087680010401CF0AFBE00BFBE1B00200008004038
:108778000034014010B500212C220348F7F70AFE07
:10878800BDE81040FFF7CABFBE1B002070B5214CE2
:108798002378042B39D8DFE803F0030D152A3000BD
:1087A8001D4B012093F82B3013F0010F30D02070AF
:1087B800013870BD184B93F82000FFF709FF02231A
:1087C800237022E0144DEE8CFEB9FFF7A7FF95F851
:1087D800203095F821200133DBB29A4285F8203009
:1087E80001D8042300E003232370304670BD0A4BF0
:1087F800D88C50B90123237070BD074BDD8C35B977
:10880800FFF7B8FF2570012070BD002070BD002063
:1088180070BD00BFEB1B0020BE1B0020044B0022D4
:108828005A701A709A7842F001029A70704700BF25
:10883800141D0020202102480A46F7F7ABBD00BFEF
:10884800F401002038B5044608460D46F7F7F2FF54
:1088580098B10319202B094BC8BFC4F120001C197B
:10886800002308E014F8012BE02A14BFEA5C202258
:1088780004F8012C01338342F4DB38BDF4010020F5
:108888000D4B46F635321B689B6893420FD043F672
:10889800F92293420BD0122B09D0B3F5E97F08D007
:1088A80046F6D9301B1A584240EB030070470120A6
:1088B80070470120704700BF241C0020F0B51F46F8
:1088C80087B006460C46084600211546F7F762FDB4
:1088D800244B07B19F80B3F9041005A801EB86016A
:1088E800042208F04AFF002605AB9B5D013BDBB282
:1088F800B92B35D81D2B4FEA031209D8D31803F525
:108908001C41684601F5C571112208F036FF0BE0DD
:108918001549D3185B186A4603F110071868596897
:108928000833BB4203C2F9D12046F7F783FFC7B229
:108938006846F7F77FFF3818A84203D8E019694658
:10894800F7F71AFF6846F7F775FF7B1C1B18AB4251
:1089580003D2E0190549F7F777FD0136042EC3D194
:1089680007B0F0BD141D0020D9290308EA47030801
:1089780010B500216C220446F7F70CFD0123A37003
:1089880010BD002343700370837843F001038370A4
:10899800704700002DE9F0419378804613F0010FED
:1089A8000D4614463AD06FF3000393701AF0CAF8D4
:1089B8006378002B32D123780BB90A336370A3781C
:1089C800174F6FF30003A3701AF0BCF8217807EB78
:1089D80008066118073130462A46F7F7B1FF3046D6
:1089E800F7F728FFC6B2AE420DD80AD2002323708B
:1089F80006EB08000A33637038182021AA1BF7F722
:108A0800C9FCAE420AD12278A3181B7A1BB10132E5
:108A18002270BDE8F08123700A236370BDE8F081FD
:108A2800F4010020054B1A780AB100221A701B784D
:108A380046F69B2202FB0311FFF704BF071C002028
:108A4800F8B505460C460818002108F07BFE013CE5
:108A5800E4B26719384608F07FFEC6B2202E03D864
:108A68003846002108F06EFE0CB1202EEFD9F8BD73
:108A780002F00F03032B22F07F0230B5D2B20CD9DB
:108A88004FF47A7491FBF4F42025E4B2057002B136
:108A980014B13034047000220130B1F57A7F05DB5F
:108AA8004FF47A7491FBF4F504FB1511022B0BD9E2
:108AB800642491FBF4F42025E4B2057002B114B1EA
:108AC8003034047000220130632904DD642491FBF2
:108AD800F4F504FB1511012B0AD90A2391FBF3F3D2
:108AE8002024DBB2047002B10BB1303303700130C3
:108AF800092904DD0A2391FBF3F203FB121130313B
:108B0800017030BD13B5104B01461B689A899C7BD8
:108B180012F0100214BF0220012034B10B4C9B7CD0
:108B28002478634303FB001109B23AB10DF1060042
:108B3800022208F022FEBDF8060002E0084608F00E
:108B48000BFE00B21CBD00BF241C0020B31C00207B
:108B580010B50F4B1B689A899C7B12F0100214BF4A
:108B68000221012134B10B4C9B7C2478634303FB25
:108B7800010000B22AB108490222BDE8104008F0FD
:108B8800F6BD054B1968BDE8104008F0DBBD00BF15
:108B9800241C0020B31C0020CC1C00203038C0B29C
:108BA800092894BFFF20002070470000024B1A7864
:108BB8006FF300021A707047031D002070B58F4CC8
:108BC800FFF7F4FF2678254606F0F006202E72D12E
:108BD80009F022F900286ED1894B1B7833B9237824
:108BE800C3F30312013262F307135EE0854B1B786F
:108BF80003F08003DBB2002B59D08348F7F71AFE45
:108C0800C5B2824CBDB1204681493246F7F798FE7D
:108C18000A2D0BD82A4620467B49F7F791FE6019A2
:108C28003146C5F10A02F7F7B5FB04E0204676495C
:108C38000A22F7F785FE774B1B7813F0010F01D056
:108C4800472300E02023E372704C042204F10C0057
:108C5800A521F7F79FFB704B1A7852B1FF23012A21
:108C6800237306D9022A637303D0032AA37318BF98
:108C7800E3736A4C257815F0600502D194F8A330A7
:108C880013B96748674902E0654804F1A301062261
:108C9800F7F756FE644B1B78452B40F09D81002D5D
:108CA80040F09A81237843F08003237070BD5748C1
:108CB8005E49324685E12C7804F0F004102C3FD14F
:108CC80009F0AAF800283BD1202259494F48F7F764
:108CD80037FE4E4856492246F7F732FE554B1B7869
:108CE80013F0010F06D05448F7F7A4FD5249024685
:108CF800524805E05248F7F79DFD514902464F4852
:108D0800F7F71EFE3E4B1B781BB94E484E49102202
:108D180057E14C484D491022F7F712FE394B1B78A2
:108D280003F08003DBB22BB14348F7F783FD02461B
:108D380047484FE04248F7F77DFD0246444842E085
:108D48002B7803F0F003302B46D109F065F80028A2
:108D580042D12E4C20223F492046F7F7F1FDA521AC
:108D6800052204F10B00F7F715FB3B4B1B78042B8E
:108D780002D9FF23E37300E002D1FF23A37301E0CC
:108D8800032B02D1FF23637301E0022B02D1FF23DF
:108D9800237300E00BB1FF23E372304B5B7813F0D1
:108DA800600F05D03F23E37223736373A373E373E8
:108DB8002B4B1B7803F02003DBB233B12048F7F7C5
:108DC80039FD024627481E49FBE01B48F7F732FDEC
:108DD800024624481849F4E02B7813F0F00347D1F1
:108DE800202221490948F7F7ABFD204B074819888D
:108DF8008322BDE87040FFF73BBE00BF031D002083
:108E0800582500202C25002030250020F4010020C2
:108E1800E6EF02084C53002025260020602500209C
:108E28000E020020CFC70208EC1B0020A4EF0208A6
:108E3800C8250308363C0020122703080102002039
:108E48003327030804020020952B0308E9250308AB
:108E58001102002074C80208CB290020042F00202A
:108E68009C3700200F02002011C80208021C0020B5
:108E7800602B1ED108F0D0FFD8B958492022584895
:108E8800F7F75EFD5748F7F7D5FC564902465648AE
:108E9800F7F756FD5548F7F7CDFC544902465448B4
:108EA800F7F74EFD5348F7F7C5FC524902465248BA
:108EB80087E02B7803F0F003102B06D108F0ACFF05
:108EC80018B147484D4920227BE02B7803F0F00485
:108ED800402C02D0502C78D108E041484849202243
:108EE800F7F72EFD474B1B784BB94CE03C484649F9
:108EF8002022F7F725FD454B1B783BB943E0444B4F
:108F08005A7882B11B78022B14D105E0414B1B78AB
:108F180013F0010F07D00DE03F48F7F78BFC3E49EF
:108F280002463E4835E03E48F7F784FC3C49024695
:108F38003A482EE03B48F7F77DFC3A490246374865
:108F4800F7F7FEFC402C0BBF314B374B5B78DB78D7
:108F5800022B0AD0042B0FD0012B1CD13348F7F772
:108F680069FC3249024632481BE03248F7F762FC96
:108F7800304902462E4814E02F48F7F75BFC2E498B
:108F880002462B480DE02D48F7F754FC2B490246C2
:108F98002248F7F7D5FC2A48F7F74CFC284902463F
:108FA8002348F7F7CDFC274B1B78ABB920210722C4
:108FB8001F48F7F7EFF92148F7F73CFC1F4902462D
:108FC8001B48BDE87040F7F7BBBC1F4A6FF3071397
:108FD80013701E4B00221A6070BD00BFF0C7020854
:108FE800F4010020F0C00208F8010020FAC00208CD
:108FF80008020020F5C002080F02002053C802082A
:109008000A260308843700202B2603085825002049
:10901800963300204C530020D0260308FD01002081
:109028007527030812270308002500204C2603088B
:109038000D0200206D2603088E2603085427030816
:10904800AF2603087C310020031D0020241C0020CB
:10905800204B70B5F022204D1A702B7813F0010FB9
:109068000BD01E4C207810F0010006D11C49FFF7E8
:10907800D9FC237843F0010323701A4E3378532B1D
:109088000ED1164C237813F0010F07D00020164993
:10909800FFF7C8FC23786FF300032370FFF786FD02
:1090A8003378232B14D10D4B1B7813F0010F0FD1FC
:1090B800FFF77CFD2B780D4A43F006032B701378DD
:1090C800013BDBB213700A4A52F82320094B1A609D
:1090D80070BD00BF0F1D0020031D0020291C0020AB
:1090E800991B0308EC1B0020781B0308E31C0020D5
:1090F800F01C0020241C00202DE9F0415E4BF022DA
:109108005E4D1A702A7802F01003DBB2002B2DD1C5
:109118005B4963F347120B601C462A70594A9A5CF4
:109128002D2A01D00134E4B20133112BF6D1564E69
:109138003A213046F7F7ACF938B1801BC0B201309C
:10914800301821460222FFF793FC504B1B78452B21
:1091580040F08F8000242046013412F089FB112C46
:10916800F9D12B7843F010032B703CE0484C23785E
:1091780013F0010F17D1424E4648FFF7F9FB424F53
:109188003168384601310222FFF772FC2D23BB708B
:10919800307846F6615340496522FFF78FFB237804
:1091A80043F00103237003200D213A4AFFF7F2FB35
:1091B8002D78324E15F0E00545D110203749FFF7DC
:1091C80031FC324B1B78442B11D12D4A13680133E3
:1091D8001121B3FBF1F101EB01115B1A2949C95CBB
:1091E8002D29F4D01360BDE8F041FFF7DFBC532B05
:1091F8000DD132784E3B63F347123270204A28492A
:109208001268062000FB02125380BDE8F081232B70
:109218002FD11B4B1D60337803F0EF0365F3471321
:109228003370FFF7C3FC23781E4A43F0060323700C
:109238001378013BDBB213701B4A52F823201B4BF7
:109248001A60BDE8F081104C10201949FFF7EAFBBD
:1092580004F110002821F7F71BF950B1001B3178F1
:10926800C0B20130201849098022BDE8F041FFF75B
:10927800FFBBBDE8F08100BF0F1D0020291C0020A6
:10928800CC1C0020ED390020F4010020EC1B00204C
:10929800031D0020141D00201B1D0020151B0308A2
:1092A8001E3A0020E31C0020F01C0020241C002093
:1092B800361B0308454B2DE9F041F022444E1A7045
:1092C8003378444D43F0010333702B68424C9B7C48
:1092D800022B06D1414B1B7803F04003DBB23BB1B4
:1092E8000FE0012B0DD13E4B1B7813F0010F08D175
:1092F80008F00AFF236800206FF3555323603949AB
:1093080044E0A378344F03F02003DBB2C3B908F07C
:10931800FBFEF87800F02000C0B288B92968324B0B
:10932800897C1A7861F301021A703B682D4943F46D
:1093380000133B60FFF776FB2C4B802283F8432019
:109348000DF0F4FA804678B12B689B7C012B08D18C
:10935800234B5B7803F01003DBB213B100202449E0
:1093680014E00020234911E00DF010FB074610B16E
:10937800404621490AE00DF051FB10B138461F491B
:1093880004E01A4B93F8433013B91D49FFF74AFB21
:109398001C4B1B78232B16D1FFF708FC337843F0BE
:1093A8000603337008F0B0FE23686FF3555323604B
:1093B8000CF028FA144A1378013BDBB21370134AF5
:1093C80052F823302B60BDE8F08100BF0F1D00204C
:1093D800031D0020241C00209C3700202C25002081
:1093E800363C0020BA1B03083B3C0020AD2000207F
:1093F800FC1B0308DB1B03083E1C03081D1C030899
:109408005F1C0308EC1B0020E31C0020F01C00205C
:109418002DE9F3416E4B6F4DF0221A702B686E4C9C
:109428009B7C1BB9637843F0100302E0637843F038
:1094380008036A4E6370337843F00103337023885E
:1094480023F47E6323F01E03DB04DB0CB3F5805F9B
:1094580008D0634B1B7883B15F4B5B7803F008033C
:10946800DBB253B1637800206FF341035D49637049
:10947800FFF7D8FAF8F724FE84E06378564F03F034
:109488000203DBB2FBB9BB78EBB9574B93F800800A
:1094980018F0010817D1F8F713FE7B7843F00203A0
:1094A8007B702B68B3F91030022B7B780CBF43F02C
:1094B800040368F3820300217B70082001220B4615
:1094C8000091F9F71BF9A378434A032B28D003D856
:1094D800012B0BD00DD806E0052B2DD0517825D3C4
:1094E800FF2B32D12BE000203E4949E000203F49C4
:1094F80046E03F48F7F79EF9DFF82C81C7B23C49B0
:1095080008F110003A46F7F71BFA0F2F3AD807F17F
:10951800100040442021C7F11002F6F73BFF31E06C
:10952800344B187800282DD1334929E06FF34101D5
:1095380051700020314923E00020314920E06FF3C9
:109548004101517000202F491AE0053BDBB26FF34F
:109558004101022B517002D100202B4910E0012B50
:1095680002D1002029490BE0032B02D10020284911
:1095780006E0052B02D10020264901E026490020FB
:10958800FFF750FA637803F00203DBB20BB9F8F780
:1095980097FD224B1B78232B18D1FFF707FB337855
:1095A800002243F0060333706378A27003F0E503EA
:1095B80062F382036370F8F783FD194A1378013B5D
:1095C800DBB21370174A52F823302B60BDE8FC81D8
:1095D8000F1D0020241C00204C530020031D0020D8
:1095E80096330020BA1B030852530020FD170308C6
:1095F8005B530020505300201E180308C21C0308A8
:10960800A2180308051903083F180308601803087F
:1096180081180308C3180308E4180308EC1B00208A
:10962800E31C0020F01C0020F40100207B4B2DE9F6
:10963800F341F0227A4E1A7033787A4D43F00103E1
:1096480033702B68784C9B7C022B11D1774B1B789D
:1096580003F04003DBB293B1754B1B7803F0200392
:10966800DBB2BBB1A37803F04003DBB23BB111E03E
:10967800012B0FD16F4B1B7813F0010F0AD1F8F7AC
:109688001FFD2368002023F480036FF3D753236062
:1096980069498FE0A778DFF8908107F04003DFB2CF
:1096A800002F34D1F8F70CFD2968644B897C1A78AF
:1096B800384661F301021A70D8F800305E4943F465
:1096C800800367F3D753C8F80030FFF7ABF92B686E
:1096D800198A21B90091082001220B4615E00BB226
:1096E800022B0CD101223B46082039460097F9F796
:1096F80005F8534B1A7842F008021A7007E0012B5C
:1097080005D100970E2039463A46F8F7F7FF0DF0D5
:109718000DF9074678B12B689B7C012B08D1454B86
:109728005B7803F01003DBB213B10020454941E038
:10973800002045493EE0414B3946187800F00300C7
:10974800F8F7F6FDFF280FD13D4B1B7803F01803FF
:10975800182B31D0A07800F08000C0B210B1384684
:109768003A4927E03A4925E00DF010F98046E0B182
:10977800334B187800F008085FFA88F8B8F1000F42
:109788000AD1F8F72BFFC0B2022801D840460AE0F8
:10979800062811D8404604E000F01000C0B210B10D
:1097A80038462C4906E02C4904E00DF037F918B189
:1097B8002A494046FFF736F9294B1B78232B29D134
:1097C800FFF7F4F9337843F006033370F8F778FCC1
:1097D800236823F480036FF3D7532360184B1A7858
:1097E8006FF3C3021A701F4A1378013BDBB2137080
:1097F8001D4A52F823302B60104B1B7803F00303EB
:10980800022B02D10DF068F820B102B0BDE8F0419A
:109818000BF0F8BF02B0BDE8F08100BF0F1D0020BB
:10982800031D0020241C00209C3700202C2500202C
:1098380060250020363C0020BA1B03083B3C002072
:109848003C1E0020FC1B0308DB1B0308C21C03088A
:10985800E31C0308A11C0308801C03081D1C030843
:10986800EC1B0020E31C0020F01C002010B5FFF7C3
:109878009DF90A482523C377094B0A4A1B68132117
:109888009B7C1C3001FB03235B78093903F00F0331
:1098980059438322BDE81040FFF7EAB8F4010020DD
:1098A800241C0020B03700202DE9F0474E4C4F4EC5
:1098B8002378F02243F0010323704D4BDFF86881D1
:1098C8001A7033689A6847F23753D21AD2F10009EE
:1098D80049EB0209132101FB09F1464A555C53186B
:1098E800C5F30005EFB2924617BB38464249FFF769
:1098F80099F898F80030232B74D1FFF757F923789B
:109908003E4A43F0060323701378013BDBB2137021
:109918003B4A52F8233033603A4B1D703A4B1D7066
:109928003A4B1D703A4B1F603A4B1D70BDE8F087EB
:1099380098F80020232A21D19A786FF300029A70B0
:109948000DF04CFFFFF732F923782C4A43F0060359
:1099580023701378013BDBB21370294A52F8233085
:10996800284A336000231370274A1370274A13705C
:10997800274A1360274A1370BDE8F087532A14D189
:109988009A7812F0010110D1422000FB09F0224C14
:1099980042F00102255C61F3000525549A701C4BC6
:1099A80001221A60484615F07BFF132303FB09A325
:1099B8009B7813F0010F02D0002018490EE0144BD9
:1099C8001B684BB9484615F0D7FA014614480222DD
:1099D800BDE8F047FFF74CB812490020BDE8F04752
:1099E800FFF720B8BDE8F087031D0020241C0020E5
:1099F8000F1D0020B03700203FD60208E31C0020CE
:109A0800F01C0020091C0020321C0020B31C002080
:109A1800CC1C0020BE1C0020144A0020F31E0308A2
:109A28000D020020D21E0308EC1B00202DE9F04196
:109A38002D4E2E4F307800F5E240BD3007F08CFEF9
:109A48003B78C4B213F0010F26D0294D2B78552B43
:109A58000AD1EC2C01D0013CE4B23078214600F563
:109A6800E240BD3007F06EFE2B78442B0DD1A4F1F7
:109A78001403DBB2D72B01D90134E4B23078214684
:109A880000F5E240BD3007F05DFE2B78532B03D183
:109A9800FFF78CF80DF0A2FE164B1B7803F080033D
:109AA800DBB253B13B7813F0010F06D012482021E6
:109AB8000422BDE8F041F6F76DBC14F0800F0F48A2
:109AC80005D12B230A2103746143113006E02D23AD
:109AD8000374373B5C43113004F520610322BDE871
:109AE800F041FEF7C5BF00BFB31C0020031D0020D6
:109AF800EC1B00209C37002004020020F401002009
:109B08001FB5204B20491A781AB1087840F0010097
:109B1800087009781C4C11F0010F31D01B490978E5
:109B2800532901D00AB103E082B901221A700DE06D
:109B380023290BD1002018701549FEF773FFFFF792
:109B480035F8237843F00603237019E01B78012BBE
:109B580016D120210A460F48F6F71CFC0E4B684622
:109B68001B681022996807F008FE002409491DF8AF
:109B7800040001EB440101341AF0FCF8102CF5D173
:109B88001FBD00BFB31C0020031D0020EC1B0020DC
:109B98000B220308F4010020241C0020034B1B782F
:109BA800532B01D1FFF702B8704700BFEC1B002010
:109BB800084BFF281A68936807D1917B41B1064981
:109BC800927C097801FB023302E0927C02FB0033AD
:109BD80018467047241C0020B31C00204328F8B501
:109BE80004460D46174608D1114B0A261A7891FBF0
:109BF800F6F66FF3C3021A7000E00E462046FEF731
:109C0800CDFF90B10A4B303C1A780A2602F00801C1
:109C1800C9B2002918BF002506FB05466FF3C30229
:109C280036B21A70BE42A8BF3E4630B2F8BD00BF79
:109C3800031D0020624B2DE9F3411A689846157CF4
:109C4800977C604C2DB1604821780222FEF710FF06
:109C580000E02570FF01237807F5124707F5BA776A
:109C680007EB4307594E0BB90DB10FE015B901A821
:109C7800394601E001A8B91E022207F07EFD9DF8D1
:109C88000430F3759DF80530337605E006F11700CA
:109C98003F210222F6F77EFB5B23B375023373760E
:109CA8004B4B1B7813F0010F5DD04A4B1B78A3F187
:109CB8003002D2B2092A31D822780AB9002D3CD113
:109CC800454A117896469942444A01D000211170BC
:109CD80043481178A3F1300490F800C004EB8404E1
:109CE80004EB010802A801318444C9B23D48641854
:109CF80010F80880005D0CF8048C117008B1032975
:109D080001D9002111708EF800300DB9384600E0F5
:109D1800B81E01A9022207F02AFD17E0232B04D15F
:109D28002F4B1A7892B9013205E02A2B05D12C4B1A
:109D38001A785AB1013A1A7008E0532B06D12A4A08
:109D4800533B1370264A1370FFF728FF274B1B78E5
:109D580003F08003DBB2002B2FD0214B1B78F618C1
:109D68002023F37529E045B31A4B1878A0F1300386
:109D7800DBB2092B10D81C4A137803B923700133BE
:109D880003F001031370D8F800302178B3F91020DC
:109D9800FFF724FF207005E0432803D1124B1B78FE
:109DA80003B92370114B1B7803F08003DBB223B196
:109DB800054820210222F6F7EDFABDE8FC8100BF34
:109DC800241C0020331C002002020020F401002083
:109DD800031D0020EC1B0020061C0020321C002064
:109DE800041C0020C0620208BE1C00209C37002012
:109DF800F7B5384E384D3378384C6FF3410333702C
:109E080018F092FCFFF7CAFE02238DF807302B7872
:109E180083B1334AD17941F00101D171314A2078B7
:109E280002EBC3035F6B93F839203978FFF7D6FE4E
:109E380038700DE0337813F0010F06D02378303BEB
:109E4800DBB2062B9CBF264AD37003238DF807305C
:109E5800337813F0010F12D0234B1B7803F08003E3
:109E6800DBB263B129781F4B204803EBC10393F899
:109E780038309DF80720C0182021F6F78BFA237890
:109E8800232B09D11A4A2B781268927C013A934203
:109E980002DA114A0133137023782A2B04D12B7864
:109EA80013B10D4A013B13702378532B0FD116F0D1
:109EB8009FFA0B4B00212970DA7961F30002DA71FD
:109EC800FFF76CFE0B4B9A7942F004029A7100235B
:109ED8002370FEBD031D0020BE1C0020EC1B0020CB
:109EE800A04A0020C06202089C370020F40100202C
:109EF800241C0020301E00202DE9F74F924E934C71
:109F08003378934D232B934F25D12368986843F6D4
:109F1800F123984217D1DFF86082296898F8000089
:109F280000F56A50713007F00DFC98F80000013018
:109F380000F0010088F8000000F56A50713007F061
:109F48000BFC286007E000B2FEF7DCFD28603B78D8
:109F580043F008033B703378532B40F06781236844
:109F680049F221329B68934202D12A687A4B15E064
:109F78004AF6C222934202D12A68784B0EE04AF68A
:109F88003F22934202D12A68754B07E049F27232A8
:109F9800934204D12A68734B02B101221A702368D4
:109FA8009A6843F6DD239A420AD16F4B29681A78DA
:109FB80061F300021A7007F02FFF08B107F04AFF9B
:109FC800236843F6E0229B68934206D1664B2968D2
:109FD8001A7861F3C7121A7019E043F6EA2293421D
:109FE80006D1614B29685A7861F300025A700EE075
:109FF80043F6E72293420AD129685C4B19B11A68E3
:10A0080042F0005202E01A6861F35D721A60236838
:10A018009A684AF658339A420AD12968544B19B1BA
:10A028001A7842F0200202E01A7861F345121A7099
:10A0380023689A684AF6E5339A4202D1287819F0DB
:10A04800DBF8236843F6DA229B68934203D12A6837
:10A05800484B1A7008E049F22A32934204D12B681F
:10A0680013B93B4B01221A6023689A684AF6E63313
:10A078009A420BD1404A2B6812784049032B8B54E3
:10A0880004D13F4B5A7942F010025A71236849F2C1
:10A098006A329B68934202D129683A4A05E049F23C
:10A0A8006D32934203D12968374A117016E049F29C
:10A0B8006E32934203D12968344A117015E049F28F
:10A0C8007032934203D12968314A11701CE049F279
:10A0D8007132934202D12A682E4B13E043F605529F
:10A0E800934202D12A682C4B0CE049F678529342ED
:10A0F80002D12A68294B05E04AF6D622934203D1B9
:10A108002A68274B1A700AE049F22232934206D194
:10A118002A68244B01201A7001460EF041F9236881
:10A12800986843F6F12398423ED1DFF84C802968BD
:10A1380098F8000000F56A50713007F003FB00231F
:10A1480088F8003033E000BFEC1B0020241C0020FE
:10A15800CC1C0020031D0020582500208437002037
:10A168007C310020EA1B0020811D00209C37002044
:10A178004C5300202E4D0020B31C00201816002040
:10A1880000250020083D0020063D0020393C002025
:10A19800AD3B0020B01E002056140020CD1A002030
:10A1A800A21B0020A63A002000B2FEF7D1FC2368CB
:10A1B8009A6843F698139A4236D12968DFF8A8B20C
:10A1C800DFF8D0A20BEBC1031B79DFF8A082C3F341
:10A1D8004113012BDFF8C09221DD98F8000000F54B
:10A1E8006650203007F0AEFA98F80030DAF8001020
:10A1F80009EB030211720BEBC1021279C2F341128F
:10A20800032A0CD1974A126890681030C01807F0DA
:10A2180099FA98F80030DAF800204B441A7498F844
:10A2280000302A6809F80320FFF7B8FC3B78DFF80C
:10A238006C8213F0010F00F0DC80216843F698125D
:10A248008B6893427FD1884A2B68914602EBC30101
:10A258000979C1F34111012906DD844A1278072AD8
:10A2680002D9FEF7A3FCD0E03278442A36D15FFA4F
:10A2780083F82DE008F101087B4B5FFA88F803EBBF
:10A28800C8031B79C3F34113012B06DD784B1B78F8
:10A2980023BB764B1B78072B20D8DFF8D0A19AF880
:10A2A80000303F2B08D807F0B7FD70B109EBC803A1
:10A2B8001B7913F0100F08D19AF800303F2B07D9FB
:10A2C80009EBC8031B79DB0902D0C5F8008005E05B
:10A2D80009EBC8031B7913F0080FCBD03378552B43
:10A2E80040F093802E782BE0013EF6B209EBC603CE
:10A2F8001B79C3F34113012B08DD5D4B1B78002B41
:10A3080040F08380594B1B78082B7ED8DFF85C819E
:10A3180098F800303F2B08D807F07EFD70B109EBA4
:10A32800C6031B7913F0100F08D198F800303F2BA3
:10A3380006D909EBC6031B79DB0901D02E6064E05E
:10A34800002ED1D161E04AF6E63293420AD005DC0C
:10A35800A3F52A42D63A012A0ED803E04AF6434228
:10A36800934209D133782F2B4FD9B1F910203032CD
:10A3780093424ADC303B30E043F6F122934207D166
:10A388003A4B1B7823B13078B5F900103B222CE00A
:10A3980007F042FD18B3236843F6C4219A688A423D
:10A3A80003D047F2CD018A4204D13078B5F90010C4
:10A3B8002D221AE0A2F56A516139052903D943F61D
:10A3C800E9218A4201D1012307E043F6E0218A42CC
:10A3D80002D00A318A4203D100232B6015E023689A
:10A3E8003078B5F90010B3F91020FFF7F7FB2860B3
:10A3F8000BE02368B3F90800FEF784FB286098F89F
:10A40800003043F0080388F80030FFF7C7FB2368E3
:10A4180043F6D222986890420BD12B6813B915489D
:10A42800154901E0134815490222F6F789FA022670
:10A43800C8E14AF6434290420AD12B6813B9104842
:10A44800104931E0012B0E480CBF0F490F492BE092
:10A458004AF6E632904236D12B68012B20D10848C3
:10A468000B4921E0241C002014040020B31C002008
:10A478004A0D002012020020246302082663020805
:10A4880004020020EF0D0308310E0308100E030824
:10A49800C60C0308CC1C0020CC290020031D00207A
:10A4A800022B05D1A548A6491022F6F749FA88E1FA
:10A4B800032B02D1A148A349F6E7042B9F480CBF00
:10A4C800A149A249F0E74AF6D62290420AD12B6860
:10A4D80013B99A489E49E7E7022B98480CBF9D4953
:10A4E8009D49E1E74AF6D72290420AD12B6813B971
:10A4F80092489A49D8E7012B40F063818F489849E0
:10A50800D2E749F26F32904203D043F6EE229042EE
:10A518000ED128680A21B0FBF1F201FB1201914B20
:10A528003031D97730322E2199775A77032649E18D
:10A5380043F6F12290423ED18B4B1B78E3B90222BD
:10A5480029688A48FEF794FA43F6F220FEF7DAFA09
:10A55800022201468648FEF78BFA3B7813F0010F7A
:10A5680000F08081834B1B7803F08003DBB2002B63
:10A5780000F078817D4819E0FEF7C4FA022201460E
:10A588007A48FEF775FA022279482968FEF770FAC8
:10A598003B7813F0010F00F06581764B1B7803F0D0
:10A5A8008003DBB2002B00F05D817148202102227C
:10A5B800F5F7F0FE56E143F69812904240F0B58068
:10A5C8002B686D4EDFF8A08156F8331010225B48D7
:10A5D800F6F7B6F90DF1060298F800000DF107013B
:10A5E8000FF0CAFE4246334620B316786349895DA8
:10A5F80003291FD0296803EBC1010979C1F341116F
:10A60800012917D1072E15D95D490B225D48F6F7A8
:10A6180097F95D48711C0222FEF72AFA9DF8071087
:10A628005A4801310222FEF723FA9DF806105848CD
:10A63800013118E02E68157803EBC601097903EBA0
:10A64800C6063679C1F34111012906F00706C8BFCD
:10A6580005F00705012E0ADC4E494A480B22F6F799
:10A668006FF94948691C0222FEF702FAA9E0022E96
:10A678000BD149490B224348F6F762F93246424862
:10A68800691CFEF7F5F90E369CE0032E0BD1434901
:10A698000B223C48F6F754F93B48691C0222FEF7A6
:10A6A800E7F90D368EE0042E11D13D490B223548CD
:10A6B800F6F746F93448691C0222FEF7D9F93348FF
:10A6C80005F109010222FEF7D3F90C367AE0052ECE
:10A6D80011D134490B222B48F6F732F92A48691C64
:10A6E8000222FEF7C5F9294805F109010222FEF701
:10A6F800BFF90B3666E0062E63D12B490B222148A1
:10A70800F6F71EF92048691C0222FEF7B1F91F4826
:10A7180005F109010222FEF7ABF9244805F1110100
:10A728000222FEF7A5F90A364CE0B3F91060092EAB
:10A738003EDD632ECCBF032602263AE00402002049
:10A74800E70C0308080D0308290D0308A50C0308E6
:10A75800940E0308D60E0308B50E0308180F030855
:10A76800390F0308F4010020B31C00200F02002059
:10A77800120200209C37002014040020CC2900205D
:10A788007D280308F9010020FA010020FE010020BD
:10A79800010200203B280308962703081A2803080B
:10A7A800D8270308B7270308F9270308020200205F
:10A7B80001262D482968801B46F08002FEF758F9CB
:10A7C80000E010263B7813F0010F0BD0274B1B78C5
:10A7D80003F08003DBB22BB123482021801B3246D3
:10A7E800F5F7D8FD224EB37803F00203DBB2002B55
:10A7F80038D0FEF745F81F4D034628B92878F11DD3
:10A808006522FEF75BF808E0B2792978B388F01D75
:10A8180001FB023109B206F0B0FF236847F2CD020E
:10A828009B68934213D006DC43F6C42293420ED0B1
:10A8380043F69A5209E047F24D12934207D049F283
:10A848002A32934203D047F20D1293420AD10520CF
:10A858000B21074AFEF79EF82978074801310222A2
:10A86800FEF706F9BDE8FE8F140200209C37002091
:10A87800141D0020B31C0020F5010020F0B5114B79
:10A888001F78114B303F1E680DE0D6F814C01CF835
:10A8980003C00133644501D112E00023DAB28242D9
:10A8A800F3D301350D70094B0622094902FB073322
:10A8B8000D785B1993F86840002CEED10C70F932D2
:10A8C8001046F0BDEC1B0020241C0020C0620208CA
:10A8D800321C00202DE9F74F964C974E23689A6852
:10A8E80043F606539A4203D133780BB901333370D8
:10A8F8002368924F99689B7C3A78B3F1010848BF66
:10A9080003F106084FEAE808337808F1010812F065
:10A91800010F03FB08188A4D00F0AD80894B1A78A7
:10A928009946432A4DD128780FFA88FA0AEBD000C5
:10A9380006F012FF2268844B916846F2C462914285
:10A94800186001D12A783AB12A78012102F0070269
:10A9580011FA02F250401860287819780AEBD000F2
:10A9680006F0F0FE236847F2AD129B68934209D1C6
:10A97800734B1A78754B03EBD203734A126883F84A
:10A98800A0211EE046F67532934205D131780020A9
:10A9980001310EF023F814E046F28B7A4FF0000BE9
:10A9A80023689B68534504D101200BEB00010EF08E
:10A9B80015F80AF1080A46F2CB739A450BF1010B18
:10A9C800EED199F80030232B10D122682B78927C95
:10A9D800013A93420ADA5A4A013313705C4B9B7866
:10A9E80003F00203DBB20BB1FDF718FF99F8003052
:10A9F8002A2B0CD12B7853B1514A013B1370544B7D
:10AA08009B7803F00203DBB20BB1FDF707FF99F85F
:10AA18000030552B14D12368997C0F2910D92A7836
:10AA280008398A42464B01DA083200E000221A70DF
:10AA3800474B9B7803F00203DBB20BB1FDF7EEFE48
:10AA480099F80030442B42D123689A7C0F2A3ED9CA
:10AA580029783B4B072902D90839197001E0083ACF
:10AA68001A703B4B9B7803F00203DBB2002B2ED00D
:10AA7800FDF7D4FE2BE049F2E12399420ED1314B88
:10AA88001B78A3F13101C9B2072907D842F00602A1
:10AA98003A7007225343284A573B137023689A6831
:10AAA80043F606539A4212D133781B2B08D9284B08
:10AAB80046F661429A809A7842F002029A7006E05D
:10AAC8005901C918234B0020C918FDF7ABFFFFF740
:10AAD80065F8214A2B7811789346994288BF1370FC
:10AAE80012780F32934202DD1B4A0F3B1370236822
:10AAF8004FF0000A93F81290B9F10F0F9ABFC9F1FD
:10AB080020095FFA89F94FF010099BF800004FFA05
:10AB18008AF318180FFA88F202EBE000019306F0A6
:10AB28001BFE9BF80020019B5FFA80FC9B1803F03A
:10AB380007032AE0241C0020B31C0020031D00206A
:10AB4800BE1C0020EC1B0020CC1C0020CC290020BF
:10AB5800141D002049110308B51C00204CFA03F00D
:10AB68006549013300F0010000280CBFA520DB2057
:10AB7800DBB201F809000AF1010A09F10109082B01
:10AB88005FFA8AFA5FFA89F903D0B9F1200FE5D1A3
:10AB980009E0B9F1200F06D023684FFA8AF19B7CAF
:10ABA80089189942B1DB3B7813F0010F15D023685F
:10ABB80052499B7C09780F2B01F0800198BFC3F1A3
:10ABC8001003C9B294BFDBB2002331B12978103128
:10ABD8008A1A4949CB185F219954DFF8288198F8D7
:10ABE8000230474603F00203DBB2002B64D0FDF7C6
:10ABF80047FE034600BB226846F6753192688A42D2
:10AC080006D024318A4203D043F6E5118A4204D1A2
:10AC180030783B496522002309E043F606518A4211
:10AC280008D130781C38C0B208F107016522FDF759
:10AC380045FE18E02878F7E7236846F635329B6822
:10AC4800934203D043F6F922934202D1BA7931787C
:10AC580001E0BA792978BB88294801FB0231BA7921
:10AC680009B206F08AFD23689A7C102A02D90520C9
:10AC78000B211EE09B6846F6353293420ED006DC67
:10AC880043F6E512934209D043F6F92204E046F66A
:10AC98007532934202D02432934201D1102007E04A
:10ACA80043F60652934202D10020102101E0002011
:10ACB8000721144AFDF76EFE226846F6D9319368DB
:10ACC8008B4216D046F693218B4212D043F6ED21E3
:10ACD8008B4202D1084BDB219977937C102B08D942
:10ACE800297809480131022203B0BDE8F04FFDF789
:10ACF800BFBE03B0BDE8F08FF40100209C370020F0
:10AD08001B1D0020141D0020F5010020114B0022FE
:10AD180070B50D461A7118B11B7803B9202343701A
:10AD2800BDB10D48F5F786FD0446681C5CB10A49BB
:10AD38002246F5F787FA022C0BDC601C2818202124
:10AD4800C4F1030201E020210322BDE87040F5F7B9
:10AD580021BB70BDA01C0020A11C002038B50546F1
:10AD6800002408E0601906F0F7FC3038C0B2092862
:10AD780008D80134E4B2044B1B78303B9C42F1DB29
:10AD8800012038BD002038BD081C002008B506F099
:10AD9800E3FC0023C0B2064AD25C824201D12028DB
:10ADA80004D10133082BF6D1002008BD012008BDCD
:10ADB8006463020870B506460D4600240DB12D23C4
:10ADC8002B55A0190021013406F0BCFC062CF5D146
:10ADD80070BD00002DE9F04F944C954E226896F80E
:10ADE8000090936892F8128099B208FB091847F608
:10ADF8004870834287B01FFA88F80BD18D490878CC
:10AE0800497800F00700C1F3420101EBC00108EBEB
:10AE1800C10825E048F2081083420CD1854908781A
:10AE28004D7800F0070088214843C5F3420577397B
:10AE380001FB05010DE048F2C04083420BD17D497A
:10AE48000878497800F00700C1F3420101EBC0011E
:10AE58008901884404E0B3F5E97F08BF01EB49089C
:10AE6800754F764D397811F0010F51D146F6D572EC
:10AE7800934204D046F6D552934240F04481704A3A
:10AE880012782A2A3BD16F4A92F800A00AF1010AE7
:10AE98000AF0010A82F800A0BAF1000F1AD046F6AB
:10AEA800D552934208D1684B46F661429A809A7807
:10AEB80042F002029A7026E1202110226348F5F739
:10AEC80069FA4FEA49136249994400204944FDF759
:10AED800A9FD18E15C48FDF74BFD236850469A68C8
:10AEE80046F6D5539A420CBF5A495B49FDF79AFD7D
:10AEF80031785A4801310222FDF7BAFD03E1552A9B
:10AF080002D0442A40F0FF804E4B00221A70FAE02B
:10AF18005069F5F78FFC4A4B834693F800A0994691
:10AF2800BAF1450F02D14E4B00221A705046FDF778
:10AF380035FE00284FD04B4B5FFA8BFB1A785245F1
:10AF48000ED15846FFF79AFCFF2804D15846FFF760
:10AF580095FCFF283FD0444B1A7801321A7015E04F
:10AF6800DFF804A100228AF8002058460593FFF76D
:10AF780085FCFF28059B04D09AF8002001328AF846
:10AF8800002099F80020FF281A7024D02168374A39
:10AF98004B6910601B5C886846F6D571884213605F
:10AFA800924610D1562B01D0542B0CD13378123B3A
:10AFB800DBB2022B07D82B780FFA88F0C01806F0FE
:10AFC800CBFBCAF800002B780FFA88F0C018DAF823
:10AFD800001006F0B7FB99F80030552B17D12368FD
:10AFE800997C0F2913D92A7808398A42134B01DA38
:10AFF800083200E000221A70134B9B7803F002031A
:10B00800DBB20BB1FDF70AFC174B00221A7099F856
:10B018000030442B39D123689A7C0F2A35D92978F6
:10B02800064B072924D90839197023E0241C00206D
:10B03800B31C0020B91C0020031D0020BE1C0020EA
:10B04800EC1B00200E1D0020141D0020F401002020
:10B058006C0903087D070308BF070308F5010020F2
:10B06800041C0020061C0020321C0020CC1C0020E0
:10B07800083A1A70964B9B7803F00203DBB20BB1C7
:10B08800FDF7CCFB934B00221A7099F80030432B44
:10B098000DD123680FFA88F05B6919788E4B196017
:10B0A8002B78C01806F04EFB8A4B00221A7099F8CC
:10B0B8000030232B13D122682B78927C013A9342DB
:10B0C8000DDA864A01331370824B00221A70804BC6
:10B0D8009B7803F00203DBB20BB1FDF79FFB99F8F5
:10B0E80000302A2B0FD12B786BB17C4A013B1370AF
:10B0F800784B00221A70764B9B7803F00203DBB280
:10B108000BB1FDF78BFBFEF749FD754A2B781178DB
:10B118009246994288BF137012780F32934202DD2B
:10B128006F4A0F3B137023684FF0000B93F812908F
:10B13800B9F10F0F9ABFC9F120095FFA89F94FF0E9
:10B1480010099AF800000FFA88F318185844059364
:10B1580006F002FB634A02F8090009F101095FFAE7
:10B1680089F9B9F11F0F059B05D821680BF1010B6F
:10B17800897C8B45E5DB397811F0010F17D0216800
:10B188005948897C00780F2900F0800098BFC1F1E8
:10B198001001C0B294BFC9B2002140B128789AF812
:10B1A80000C010305218CCEB00005F211154226807
:10B1B800906849F6765290420AD14C4B1B78532B33
:10B1C80030D106F0C9FA4A4B187006F0BFFB29E0E7
:10B1D800B0F5E97F26D1454A1278532A22D118467C
:10B1E800FFF7D4FD8046E8B93378DA00D31A03F1C3
:10B1F8001200FFF7B3FD68B1FF2300933D4BCDF874
:10B2080004801B7879200133029341460422434687
:10B2180006F020FB33780021DA00D31A03F112007C
:10B22800FFF7C8FDDFF8A89099F80230C84603F088
:10B238000203DBB2002B68D0FDF722FB034688B976
:10B24800226848F2C04192688A420BD046F6D5512E
:10B258008A4214BF2878307809F107016522FDF782
:10B268002DFB12E0236898F806209B682248B3F566
:10B27800E97F0CBF31782978B8F8043001FB023136
:10B2880098F8062009B206F078FA23689A7C102A02
:10B2980013D89B6847F6487293420BD13B7813F05A
:10B2A800010F01D010202CE0202107221348F5F7C8
:10B2B80071F82AE0B3F5E97F02D105200B2121E0DE
:10B2C80046F6D55293421BD1002010211AE000BF48
:10B2D800141D0020321C0020CC1C0020BE1C0020A5
:10B2E800B51C0020F40100209C370020EC1B002036
:10B2F800081C0020B31C00201B1D00200402002095
:10B3080000200721094AFDF745FB23689B7C102B89
:10B3180008D9297806480131022207B0BDE8F04F64
:10B32800FDF7A6BB07B0BDE8F08F00BF141D0020D5
:10B33800F50100202DE9F04F794E8BB033689D68F8
:10B3480093F81290122D01D00B2D09D1754A122DA8
:10B3580092F80090A9F130095FFA89F915D01DE03B
:10B368004AF6F3339D4203D028339D4240F053837D
:10B378006D482821F5F78CF88046002800F04E83A8
:10B3880001302821F5F784F848E39F7B37B9674BEC
:10B39800B846D879FEF70CFC044615E00027B846F5
:10B3A800FF20FEF705FC4AF6E4139D4204460BD144
:10B3B8004AF6C32006F0D0F9C0B2099020B15B4B21
:10B3C8009B790BB1FDF7F2FB3368594D9A68122A45
:10B3D8001AD19B7BC3B12B7813F0010F08D12046FB
:10B3E800FFF7BCFC534B10B101221A7000E0187033
:10B3F8004E4B9B7943B12046FFF7B0FC20B14D4B33
:10B408001B780BB1FDF7D2FB2978DFF844A111F0C6
:10B41800010100F087819AF80030DFF838B118464A
:10B428000793FDF7BBFB079B002800F0B580424956
:10B43800002008704148424A90F800C013609C45BB
:10B44800404940F0898033689B8903F00F03032B40
:10B458001ED13D4BACF1300C18784FF00A0E059018
:10B468003A480EFB0C00DDF814E000EB0E0C0EF170
:10B47800010E5FFA8EFE70449CF8ADC090F8AD00E6
:10B48800C2F800C083F800E0002872D1187070E09C
:10B49800082B2CD12C4BACF130001B7800EB800C26
:10B4A8000CEB030E294BDFF8A0C013F80E300893FD
:10B4B8000BB98CF800309CF800E000EB8000059098
:10B4C80070440EF1010E5FFA8EFE8CF800E01F4BFF
:10B4D800DDF814C01B5C08900CEB0E00DFF86CE084
:10B4E80013601EF80030002B43D1174811E0072BDA
:10B4F80011D1BCF1300F10D11348037823B14FF0AC
:10B508002B0EC2F800E001E0C2F800C0013303F0DE
:10B51800010303702DE0062B2BD10B78013327E0B4
:10B52800241C0020081C002004020020C21C00204B
:10B53800031D002097110020334D0020061C002019
:10B54800CC1C0020BE1C0020321C0020C062020857
:10B55800EC1B0020091C0020DFF898E203709BF820
:10B5680000304FF0010C8EF800C013B10B78634423
:10B578000B7040238BF800300B784B4503D39B4B63
:10B5880009F1FF30187008781168201806F0DAF809
:10B598002B7843F004032B709AF80030232B2FD11B
:10B5A800924B09F1FF311A788A4229DA72B9326866
:10B5B8004AF6F33192688A4208D028318A4205D087
:10B5C8002046079306F0C8F8079BC8B118780130E1
:10B5D800C0B21870201806F0BFF828B9834B202194
:10B5E8001878201806F0AEF8814B40221A702B7894
:10B5F800804A43F004032B7000238BF8003013704B
:10B608009AF800302A2B10D1784B1A786AB1013A8F
:10B618001A70774B40221A702B78764A43F004034D
:10B628002B7000238BF8003013709AF80030432BEE
:10B638001FD16E4B1878484505D220182021079352
:10B6480006F080F8079B9BF800203AB91B7809F1AF
:10B65800FF32934202DA654A013313702B78644A49
:10B6680043F004032B7000231370624A8BF80030F8
:10B6780013709BF8003013B15F4A013B13709BF8BD
:10B688000030012B0ED1594B1A784A4501D20132AC
:10B698001A70584A002313702A7842F004022A705C
:10B6A8008BF800302B7803F00402D2B2002A71D054
:10B6B800524A6FF382031370002111225048F4F7A5
:10B6C80069FE504A494B11781B78994288BF13701C
:10B6D80011780F318B4202DD4A490F3B0B7011780C
:10B6E80047481022611806F048F84548F5F7A2F8CF
:10B6F80033684AF6F3319B68C2B28B4202D02831D4
:10B708008B4205D122B94048F5F794F8421CD2B2D1
:10B718000F2A3FD83A4820218018C2F11002F4F7C6
:10B7280039FE37E0DFF8D8B011225846F4F732FE78
:10B7380033684AF6F3329B68934202D02832934228
:10B7480009D1214604222E4806F017F8404639460A
:10B75800FFF7DCFA1EE021461022584606F00DF8E5
:10B768005846F5F767F802462021C2F110025844FE
:10B77800F4F710FE21464A46244805F0FEFF244A05
:10B788001020937882F8069043F0020393700146E4
:10B79800FDF700F99AF80030532B75D133689A6891
:10B7A8004AF6E4139A4208D1204605F0D5FF20B1A5
:10B7B8004AF6C320012105F0C5FF3368DFF838A039
:10B7C8009B68122B40D12046FFF7C8FA8346002811
:10B7D80030D0104BFF2219780F4BF9B90092019124
:10B7E8001B78782001330293FB3A1FE0BE1C00202F
:10B7F800334D0020321C0020091C0020031D0020AE
:10B80800A01C0020B51C0020A11C00203B1C00200F
:10B81800341C002097110020B31C00200021009246
:10B8280001911B787A200133029304220B4606F01B
:10B8380011F809E08AF800007D492046FFF7BAFAB6
:10B848007C4B83F800B0EFE020464946FDF7F8F856
:10B85800794B0020187033688AF800009B6849F615
:10B868008A52934202D10090013005E04AF606223E
:10B87800934206D1012300930146024603460DF088
:10B88800D9F86E48FDF774F8FEF788F92B7813F0AD
:10B89800010F17D033684AF6F3329B68934202D0FF
:10B8A8002832934204D140463946FFF72FFA09E07F
:10B8B8005F4B634A03F1100153F8040B8B4242F8C3
:10B8C800040BF9D133689A68122A1ED19B7BE3B125
:10B8D8002046FFF743FAC0B12B7813F0010F14D1BB
:10B8E800584B9A7922B9DA79574B1B789A420CD07F
:10B8F800564B1A780023303A05E055492A20C918D2
:10B9080001330874DBB29342F7DB326893680B2B80
:10B9180001D0122B0AD14A4B991D13F8010B20288C
:10B9280002D10D3003F8010C8B42F6D192684AF629
:10B93800E4139A4214D1434B9B798BB1099878B19F
:10B948004FF0000909EB040005F006FF18B1404B61
:10B958002A224B441A7409F10109B9F1100FF1D1E7
:10B968002B7813F0010F25D03A4B1B7803F0800396
:10B97800DBB2FBB133689A684AF6F3339A422D4B2F
:10B9880003D04AF61B418A420CD11B7833B9B8F16F
:10B99800000F0FD05F3388F801300BE057B15F22FA
:10B9A800FA5407E0244A1B78127810339B1A284A65
:10B9B8005F21D154284CA37803F00203DBB2002B9B
:10B9C80032D0FCF75DFF2049034628B90878652284
:10B9D800E11DFCF773FF12E03068B4F90430A27976
:10B9E80084680978122C01FB023105D1807B18B9D3
:10B9F8001449C97902FB0131184805F0BEFE3368C5
:10BA08009B68122B10D10820134A01460BB0BDE8E1
:10BA1800F04FFCF7BFBF0027B84600E0074609F122
:10BA2800FF395FFA89F9BBE40BB0BDE8F08F00BFBE
:10BA3800A01C0020BE1C0020B51C0020341C0020C7
:10BA480004020020C21C0020B31C0020081C002097
:10BA5800F40100209C370020141D00201B1D00202D
:10BA680024282DE9F041144626D16B4B43F6393290
:10BA78001B686A4D9B686A4E934206D12B7813F077
:10BA8800010F0ED02438674909E04AF61B42934259
:10BA98000AD12B7813F0010F03D063490020FCF77B
:10BAA800C1FF2978490800E02978301901310222BC
:10BAB800FCF7DEFF0234AAE0E72809D1574B5848C3
:10BAC8001978801801310322FCF7D2FF03349EE075
:10BAD800A3282AD1514D2B783F2B15D8104653490E
:10BAE800FCF7A0FF5148F4F7A5FE2A2124184C487A
:10BAF800E4B2F4F7CDFC002800F08A80297802220D
:10BB08000131FCF7B5FF83E05901494DC91869189F
:10BB180001F57E5110467031FCF784FF05F5904021
:10BB28000F30F4F787FE241871E0F22821D13B4F3B
:10BB38003B4D3978072605EB0208B1FBF6F1404684
:10BB480001310222FCF794FF39782D23B1FBF6F678
:10BB580088F80230F3009E1B8B1B364FDBB207EBD5
:10BB680083031988E21CA9529B78A81883700634AD
:10BB78004DE025280BD1304B46F661429A8045228C
:10BB88009A719A78053842F002029A703CE05E2871
:10BB98000BD1294B46F661529A8045229A719A78C0
:10BBA8003E3842F002029A702EE07C280BD1224BDC
:10BBB80046F244129A8011229A719A785C3842F0BF
:10BBC80002029A7020E0EC280BD11B4B46F6A552D6
:10BBD8009A8045229A719A78CC3842F002029A707B
:10BBE80012E0A7280BD1144B46F6C5529A8045227D
:10BBF8009A719A78873842F002029A7004E0E02835
:10BC080001D1541C03E018B1054B18550134E4B2B6
:10BC18002046BDE8F08100BF241C0020B31C002092
:10BC2800F4010020D10103088F0103084B09030820
:10BC38003CC10208ADEC0208141D002038B50A4BBF
:10BC480046F69B251B78002405FB030507E0074BF8
:10BC580022461978FFF704FF041B2D19044628789B
:10BC680008B11F2CF3D938BD071C0020B31C0020D5
:10BC780070B5002543F61C64204605F06DFD0646A8
:10BC880004F1080005F068FD16F0FF0F06D020F05B
:10BC98007F0010F0FF0F01D00135ADB246F23B1323
:10BCA8009C4201D00934E7E7284670BD38B5B0F9A1
:10BCB80000500B4C05EBC50505F57855243528468D
:10BCC80005F04AFDC1B211F0800F07D0238828463D
:10BCD800013B01F07F01238005F034FD208838BD49
:10BCE800021C0020454B2DE9F74F1B88444A0446A7
:10BCF80089461788DFF80C8123B14FF0000A0AE063
:10BD08009A4608E00529FBD198F8003043F004036F
:10BD180088F8003070E098F8003013F0030F0BD06B
:10BD280013F0010F02D0B4F1FF3F05D103F0020375
:10BD3800DBB21BB1012C01D03F19BFB23BB2B3F14A
:10BD4800FF3F04D0B3F57A7F08BF002701E040F237
:10BD5800E7370FFA87FB0BEBCB0303F5785303F1B7
:10BD68001C00019305F0F8FC10F0FF0F019B16D0A2
:10BD7800B9F1050F09D103F1240005F0EDFC20F01D
:10BD88007F0010F0FF0FC6D022E0B9F1000F1FD0DE
:10BD980003F1240005F0E0FC00F07F0618E00AF14A
:10BDA800010AB4F1FF3F1FFA8AFA04D198F800306B
:10BDB80043F0010305E0012C05D198F8003043F069
:10BDC800020388F80030BAF57A7F0DD03D46A2E725
:10BDD8004E4505D0B9F1000F02D0B9F1050F9AD13F
:10BDE800BAF1000F05D000E03D46054A2DB21560B6
:10BDF80002E0034BC3F800B0BDE8FE8F021C002030
:10BE0800CC1C0020D01C0020F0B503789BB05A1E33
:10BE1800D2B2792A0F4600F2C8805E01644AF3184C
:10BE28009B18644A46F69B261278457806FB02362C
:10BE3800E7213046F4F72CFB0446F0B930467C2164
:10BE4800F4F726FB0446C0B930462521F4F720FB59
:10BE5800044690B930462421F4F71AFB044660B929
:10BE680030464021F4F714FB044630B93046F92136
:10BE7800F4F70EFB0446002876D0A41B0FB14E48F9
:10BE880000E04E4831462246A619F4F759FD3046DF
:10BE9800E721F4F7FDFA30B128466946652246F6EF
:10BEA800A553FCF70BFD30467C21F4F7F1FA50B1AD
:10BEB800691EC9B201EB011101F5C241684644315E
:10BEC800112205F05AFC30462521F4F7E1FA38B181
:10BED800681EC0B26946652246F66143FCF7EEFC6F
:10BEE8003046F921F4F7D4FA38B1681EC0B2694671
:10BEF800652246F66153FCF7E1FC30464021F4F731
:10BF0800C7FA50B1691EC9B201EB011101F5E6414A
:10BF180068461731112205F030FC30462421F4F729
:10BF2800B7FA50B10FB1244800E024480019294657
:10BF38000222FCF79DFD02340BE00FB11E4800E021
:10BF48001E4800196946F4F717FC6846F4F772FCB6
:10BF58000419002F29D01A4A9378141943F00203C0
:10BF680093700023E37116E03046F4F763FC05464E
:10BF78001FB9124831462A4615E0102810DD2A4616
:10BF88000D483146F4F7DCFC0D4A9378551943F017
:10BF980002039370EC7110200146FCF7FBFC04E0EF
:10BFA800084831461022F4F7CBFC1BB0F0BD00BFA7
:10BFB80051F10208071C00201B1D0020183000202A
:10BFC800141D0020040200200C4B1B7813F0010202
:10BFD80002D000200A4905E003F00200C0B218B1FF
:10BFE80008491046FCF71EBD03F00403DBB20BB191
:10BFF8000549F7E705480121FFF706BFD01C0020D7
:10C00800F8C80208D7C8020819C90208051D002087
:10C0180070B5124D124C00201249FCF713FC28464B
:10C02800A1780222FCF724FDE81CE1780222FCF743
:10C038001FFD05F1080021790222FCF719FD05F121
:10C048000B0061790222FCF713FDA17905F10E00BE
:10C058000222BDE87040FCF70BBD00BFF4010020D0
:10C06800051D0020D16302082DE9F341504F514CC2
:10C078003B689D7C237813F0010F2FD1022243F6F1
:10C088001A610DF1060005F078FB4B4EBDF806303D
:10C098004FF0FF3033602946FFF724FE237843F042
:10C0A80001032370454B1B7813F0030F14D1B6F925
:10C0B8000010434801EBC10101F578511C310922F8
:10C0C80005F05BFB3F4B1B881BB13046FFF7EEFDCD
:10C0D80010B90020FAF79CF8FFF79AFF3A4E337828
:10C0E800552B0DD1DFF8D4803848FCF741FC98F87F
:10C0F80000304FF0FF306FF3410388F800300DE057
:10C10800442B2BD1DFF8B4803048FCF731FC98F889
:10C11800003001206FF3000388F800302946FFF74C
:10C12800E1FD98F8003013F0030F15D1224D244893
:10C13800B5F90010092201EBC10101F578511C3154
:10C1480005F01BFB1F4B1B881BB12846FFF7AEFDF4
:10C1580010B90020FAF75CF8FFF75AFFFFF734FF31
:10C168003378232B22D1154B184E1A7802F0FC0293
:10C178006FF382021A70FCF719FDB3786FF341036D
:10C18800B370134B1D7835B9FCF748FB3046FCF704
:10C19800EFFB3D600AE02278013DEDB242F0060275
:10C1A80022701D700B4B53F825303B60BDE8FC81B5
:10C1B800241C0020031D0020CC1C0020D01C0020C3
:10C1C800051D0020021C0020EC1B0020141D00206F
:10C1D800E31C0020F01C00202DE9F0411646104A0F
:10C1E8000F4653780E21C3F342034B43117803F5EE
:10C1F800FC43D8330B4D01F00701044603EB410122
:10C20800022205F0BAFAE81921780222FCF730FC7C
:10C218006178A8190222BDE8F041FCF729BC00BFEB
:10C22800B91C0020F4010020044B02225978044B69
:10C23800C1F3420118180131FCF71ABCB91C0020DF
:10C24800F401002010B5074B074C1B78074A03F090
:10C25800070304EB83031C88111814529B788B7016
:10C2680010BD00BFB91C0020ADEC0208F40100208D
:10C27800084B1B789B0902D0012B06D102E0102045
:10C28800054904E01020054901E005491020FCF7A4
:10C29800C9BB00BFB91C00209AD50208BBD502084B
:10C2A800DCD502082DE9F041DFF868800F4698F8E0
:10C2B8000010174DC1F382010446164605F1080027
:10C2C80001310222FCF7D4FB98F80010042201F097
:10C2D8001C0101F51241C031204605F04EFAE8195B
:10C2E80021780222FCF7C4FBF81C28186178022286
:10C2F800FCF7BEFBA819A1780222FCF7B9FBF01CD9
:10C30800E17828180222BDE8F041FCF7B1BB00BF74
:10C31800F4010020051C0020064B1B7803F0800365
:10C32800DBB233B1435C04482021C0180222F4F781
:10C3380031B870479C370020F40100202DE9F743FD
:10C34800654D664C2B6821789B68022203EB4101FE
:10C358000DF1060005F011FA2B68A9469A6843F614
:10C36800F4239A4208D100205D49FCF75BFBBDF835
:10C3780006804FF4B46303E0BDF806804FF46163B0
:10C38800B8FBF3F103FB11883C221FFA88F8B8FBCD
:10C39800F2F302FB1388CFB2DEB2022251483946CB
:10C3A800FCF766FB5FFA88F802224F483146FCF733
:10C3B8005FFB02224D484146FCF75AFB4C4B1B7869
:10C3C80013F0010F6ED04B4B4B4D1878232804D136
:10C3D8002B78012B62D8013305E02A2805D12B7868
:10C3E800002B5BD0013B2B7058E0A0F13003DBB28F
:10C3F800092B01D943284BD12B7873B9D9F80030D0
:10C4080039B29A6843F6F4239A4201D10A2200E02D
:10C418001122FDF7E3FBC7B216E0012B0ED1D9F8C4
:10C42800003031B29A6843F6F4239A4201D11722B8
:10C4380000E03B22FDF7D2FBC6B205E041463B22B5
:10C44800FDF7CCFB5FFA80F8D9F800309A6843F61C
:10C45800F4239A4209D13C235E434FF4B46303FBAF
:10C468000767B844ADF8068006E0384631464246CC
:10C478000FF055FBADF80600D9F8003020789B681E
:10C488000DF1060103EB4000022205F070F905E00A
:10C49800532803D100232B70FDF780FB1748297818
:10C4A800FFF73AFFD9F800309A6843F6F4239A4226
:10C4B80010D02078124965220023FCF7FFF90520E7
:10C4C8000B21104AFCF766FA21780F480131022245
:10C4D800FCF7CEFABDE8FE83241C0020B31C002024
:10C4E800D0050308040200200A02002012020020DE
:10C4F800031D0020EC1B0020BE1C0020E263020884
:10C508001B1D0020141D0020F501002073B5994B58
:10C51800994D1A7812F0010F05D12A7812F03802D5
:10C5280004BF2A706A701A78924E42F001021A709B
:10C538002B78914C13F038023ED19049097855294F
:10C5480004D113F0070F2FD0DA1D0AE044290CD1CB
:10C5580003F0070201323D3992FBF1F1C800411A9C
:10C56800521A62F3020323701EE053290AD1C3F35F
:10C57800C201013161F3C5032370637862F3430399
:10C58800637011E023290FD1FCF710FB33787C4A44
:10C5980043F0060333701378013BDBB21370794A1A
:10C5A80052F82320784B1A6000207849FCF73AFAB1
:10C5B8001C20FFF747FEDBE0082A2CD17449002035
:10C5C800FCF730FA0620FFF72FFE0C20FFF73AFEA3
:10C5D8001521182201A8FFF7FFFD684B1B78552B82
:10C5E80006D1637803F0FE03C3F34202013A07E081
:10C5F800442B09D1637803F0FE03C3F342020132EE
:10C6080062F343036370B3E0532B28D0232B40F02D
:10C61800AF802378A6E0102A51D15D490020FCF7AD
:10C6280001FA0620FFF700FE0C20FFF70BFE15218C
:10C63800182201A8FFF7D0FD6178564801F00101E2
:10C64800FFF76AFE4D4B1878232801D02A2804D119
:10C658006378DA4362F30003D4E7532804D12378DC
:10C66800C3F3C202013280E0A0F13003DBB2092B30
:10C6780001D943287CD16B7802AA03F001033B213E
:10C68800D41883F001024B43172606FB023214F834
:10C69800041CFDF7A3FA04F8040C6B780E22C3F30C
:10C6A80042035343287803F5FC43D83300F00700CE
:10C6B80003EB400001A90C3A05F059F858E0182A94
:10C6C8004DD133490020FCF7ADF90620FFF7ACFD4A
:10C6D8000C20FFF7B7FDFFF7CBFD284B1B78552B38
:10C6E80007D1237813F0C00F42D0C3F38112013A67
:10C6F80006E0442B07D123789A09012A38DC013255
:10C7080062F3871333E0232B04D12378C3F3C202E7
:10C71800023A2AE0532B2BD1FCF748FA33781E4A09
:10C7280043F006033370164B1648197840F8212059
:10C73800013119702378C3F3C201013161F3C503D4
:10C74800C3F381112370104B11B1012904D101E009
:10C758001C3202E0114A00E0114A1A6008E0114A4E
:10C7680000211170C3F3C202013A62F3C5032370BA
:10C778007CBD00BF031D0020B91C0020EC1B00205D
:10C78800E31C0020F01C0020241C002058D50208BF
:10C7980079D50208E5630208E86302082064020804
:10C7A8003C640208BE1C002073B5494B494D1A78F9
:10C7B80012F0010F04D12A7812F0030208BF2A7080
:10C7C8001A78434E42F001021A702B78414C13F04C
:10C7D80003022ED1404A1278552A03D1C3F38202AC
:10C7E800013A04E0442A06D1C3F38202013262F31B
:10C7F8008403237017E0532A03D15A1C62F3010300
:10C80800F7E7232A0FD1FCF7D1F93378334A43F0FD
:10C81800060333701378013BDBB21370304A52F8C9
:10C828002320304B1A6001A810211B22FFF73AFD84
:10C838004CE0012A4AD101A810211A32FFF732FD33
:10C84800254B1878232804D12378C3F341120132E9
:10C8580005E02A2807D12378C3F34112013A62F38D
:10C86800461323702CE0532804D12378DA1C62F392
:10C878000103F6E7A0F13003DBB2092B01D9432805
:10C888001ED12B7802AAC3F34113D4180C215A1CC9
:10C8980003F001034B4302F001021F2614F8041CA5
:10C8A80006FB0232FDF79AF904F8040C287801A96E
:10C8B80000F01C0000F51240C030042204F057FFBD
:10C8C80029780948C1F34111FFF726FD7CBD00BF57
:10C8D800031D0020051C0020EC1B0020E31C002089
:10C8E800F01C0020241C002058640208064B1B780A
:10C8F80003F08003DBB233B1435C04482021C01845
:10C908000322F3F747BD70479C370020F40100204D
:10C918004328F8B504460D46174606D1104B0026A5
:10C928001A786FF3C3021A7000E00E462046FCF72F
:10C9380035F990B10A4B303C1A780A2602F0080102
:10C94800C9B2002918BF002506FB05466FF3C302CC
:10C9580036B21A70BE42A8BF3E4630B2F8BD00BF1C
:10C96800031D00202DE9F3416E4F6F4E3B7843F0D5
:10C9780001033B70347844B94AF63B2004F0ECFEDE
:10C988006A4B6B491860204617E0012C02D1002041
:10C99800684912E0022C02D1002067490DE0032CFF
:10C9A80002D10020654908E0042C02D10020644926
:10C9B80003E0052C03D163490020FCF733F83178F4
:10C9C800D9B9614B1B78312B01D1013101E0302BF2
:10C9D80005D1564B4AF63B20196004F0B3FE5B4B79
:10C9E8001A785B4B02F08002D2B20AB1202202E030
:10C9F8004E4A12683032DA776EE001290BD00229EC
:10CA08000CD003290DD004290ED04AF63725052964
:10CA180018BF00250AE04AF6272507E04AF62B2525
:10CA280004E04AF62F2501E04AF633252946042278
:10CA380001A804F0A2FE474B474A03F1100153F83E
:10CA4800040B8B4242F8040BF9D1032243489DF8AA
:10CA58000410FCF70DF8032241489DF80510FCF777
:10CA680007F803223F489DF80610FCF701F83E48F6
:10CA780003229DF80710FBF7FBFF334B3B4C18785C
:10CA8800232804D12378022B22D8013304E02A2852
:10CA980004D12378E3B1013B237019E0A0F13003FE
:10CAA800DBB2092B01D9432812D194F8008002AADD
:10CAB800904418F8041CFF22FFF72AFF08F8040C1A
:10CAC800207802AA131813F8041C281804F03AFE58
:10CAD80027482178FFF70AFF1B4B1B78532B1FD1E0
:10CAE800224B00221A7033780133DBB2062B3370E5
:10CAF80004D0012B14D10D4B1B688BB1FDF74EF8F8
:10CB0800002333703B781B4A43F006033B701378CD
:10CB1800013BDBB21370184A52F82320174B1A60F6
:10CB2800BDE8FC81031D0020B31C0020CC1C0020A4
:10CB3800561F03087F200308A0200308C12003080C
:10CB4800E220030803210308EC1B00209C37002087
:10CB5800F4010020DC47030804020020050200203D
:10CB6800090200200D02002011020020BE1C002036
:10CB78005C640208E31C0020F01C0020241C002038
:10CB880070B5174C0D460646002120464FF4C17279
:10CB9800F3F700FCFF2D0AD1B10001F5D84120467A
:10CBA8006131042204F0E9FD23789BB970BDFE2DA4
:10CBB80001D1173E02E0FD2D02D10136267009E0B1
:10CBC800B60006F5D8406130401904F0C5FDC0B282
:10CBD800207020B10248BDE8704017F027BE70BD34
:10CBE800281F00202DE9F04117F052FE60B11020F7
:10CBF8008F49FBF717FF8F4B1B78432B40F0EF81D2
:10CC0800BDE8F04117F066BE17F054FE002826D0A4
:10CC1800894C23786BB110208849FBF703FF8848BB
:10CC28002D211030F3F734FC002800F0D88121784A
:10CC380010E010208349FBF7F5FE81482D211030C4
:10CC4800F3F726FC0446002800F0C98117F04AFED5
:10CC5800014620468222BDE8F041FBF709BF7A4C25
:10CC680043F6CC2223689B68934250D0774E744D8C
:10CC7800307803EB800004F06FFD0322014674480E
:10CC8800FBF7F6FE2368986846F6C55398422BD002
:10CC9800203B984228D03378013000EB830004F021
:10CCA8005BFD0322014605F11500FBF7E1FE236851
:10CCB80030789B68023303EB800004F04DFD0322BB
:10CCC800014605F11900FBF7D3FE236830789B680D
:10CCD800033303EB800004F03FFD0322014605F116
:10CCE8001D00FBF7C5FE0EE02D2103225948F3F77E
:10CCF80051FB2D2103225848F3F74CFB57482D21AF
:10CD08000322F3F747FB20232B772B762B75544B05
:10CD18001B7813F0010F00F0BD80236843F6CC2286
:10CD28009B68444D934261D04E4E484F32783878D4
:10CD3800D31803EB800004F00FFD4B4B014618603D
:10CD480028789846A0F13002D2B2092A01D943289E
:10CD58000FD109B2BA22FCF741FF236832789B68E9
:10CD68000146C8F800003878D31803EB800004F0B7
:10CD7800E9FC2B782A2B04D1337813B1394A013BCB
:10CD880013702B78232B0ED13378022B0BD8226803
:10CD980046F6A55192688A4205D020318A4202D0CF
:10CDA800304A013313702B78552B01D0442B0FD107
:10CDB800236831789B68A3F5D843B3F1610248BF73
:10CDC800A3F15E023B7803EBA202D0B2FFF7D8FED4
:10CDD800264B1B7803F08003DBB23BB13278184B4B
:10CDE80003EB820320225A749A74DA742B78532B3B
:10CDF80006D023689A6843F6CC239A4240F0EF8025
:10CE0800FBF7D4FE236846F661429B68934203D140
:10CE18000E4B0220197806E046F6C552934227D1F8
:10CE28000A4B002019780131BDE8F0410BF0D6BD5E
:10CE380085080308EC1B0020501400205C07030839
:10CE4800F4010020A6080308241C0020B31C0020BD
:10CE580005020020090200200D0200201102002016
:10CE6800031D0020BE1C0020CC1C00209C37002085
:10CE780046F6A552934204D15A4B01201978091855
:10CE8800D2E746F66152934240F0A980554B032001
:10CE98001978C8E7236849F68A529B6893423FD1BC
:10CEA800504E10205049FBF7BDFD31784F4D01EB36
:10CEB800011101F51C4101F5C5711022284604F045
:10CEC8005CFC2B4605F110012A461078474F78B9CB
:10CED8004749FBF7A7FD3846E721F3F7D9FA78B1B8
:10CEE8003178401B381801310322FBF7C1FD07E0F8
:10CEF80013F8010B10B9203003F8010C8B42E4D170
:10CF08003C4D2B782A2B03D13078FD21FFF738FED2
:10CF18002B78432B63D1307823680130C0B259E0B5
:10CF280043F6CC229342334E1AD010203249FBF7F5
:10CF380079FD33782A2B52D1304B1B689B68A3F5B7
:10CF4800D843B3F1610248BFA3F15E02254BFF212C
:10CF58001B7803EBA202D0B2BDE8F041FFF710BE88
:10CF68003378204D552B04D12B78142B01D1033B5A
:10CF78002B703378442B05D12B78122B02D1194B07
:10CF880015221A702B78DFF878805901C91801F535
:10CF98009041303100204144FBF744FD08F58E41B3
:10CFA800102028312F78FBF73DFD3378112F8CBFE7
:10CFB800032700272A2B05D12878FE21C01BC0B2E1
:10CFC800FFF7DEFD3378432B09D12B78173BDF1BA6
:10CFD8002368F8B2997CBDE8F04117F041BCBDE880
:10CFE800F08100BFB31C002064080308F40100208E
:10CFF8005BEA0208EC1B002022080308241C00201E
:10D008003CC1020810B50E4B1B78452B17D10D4BB0
:10D018001A7842F006021A700B4A1378022B0ED8BF
:10D028000A490B4C086844F82300013313708368DD
:10D038000B60FBF7FFFBBDE81040FBF7B7BD10BD69
:10D04800EC1B0020031D0020E31C0020241C0020F2
:10D05800F01C002010B50C4B04462146D8790EF080
:10D0680020FD68B1094B1B5D543BDBB2012B09D88D
:10D0780020460EF00DFCD0F1010038BF002010BD95
:10D08800022010BD022010BDC21C0020ED39002076
:10D0980008B50EF0F5FCC0B208BD00002DE9F04758
:10D0A800634B644C1A78994612F0010F624D65D0B3
:10D0B8002078FFF7CFFF614A2B181178604F93F85B
:10D0C800A031604E44293870336090460AD12D2B28
:10D0D80008D038B995F8A11101233B703160207848
:10D0E800FFF7D6FF98F80030552B10D133682D2B59
:10D0F8000DD03B785BB1013B514ADBB21370EB18A2
:10D1080093F8A0114F4B20781960FFF7C1FF98F8EA
:10D118000030232B19D14C4B20781B689B7C013B9A
:10D12800984212DA434B0130C0B21870FFF792FFF1
:10D138003870281890F8A0313360444B9B7803F07E
:10D148000203DBB20BB1FBF769FB98F800302A2B1E
:10D1580014D1207890B1374B0138C0B21870FFF75E
:10D1680079FF3870281890F8A0313360374B9B78D6
:10D1780003F00203DBB20BB1FBF750FB344EFCF7B4
:10D188000DFD237832789A4288BF337032780F3297
:10D19800934202DD2E4A0F3B1370DFF8C48000274C
:10D1A80030783818C0B2FFF755FF281890F8A0312A
:10D1B8000137102F08F8013F07D0254B1A78224B6A
:10D1C800BA181B689B7C9A42EADB99F8003013F086
:10D1D800010F13D01F4B1A781F4B02F08002D2B2F6
:10D1E8002AB1227831781032521A5F2105E022786C
:10D1F80031781032521A134909689954134DAB7893
:10D2080003F00203DBB25BB12078E91D652246F624
:10D218006153FBF753FB05200B212A46FBF7BAFBAA
:10D2280021780E4801310222BDE8F047FBF720BC07
:10D23800031D0020BE1C0020C0620208EC1B002059
:10D24800041C0020CC1C0020241C0020141D0020DD
:10D25800B51C00209C370020F4010020F5010020B7
:10D26800030200202DE9F041074610460D461446FA
:10D27800F3F7E0FAC3B28046B3B1AB4214D80B4E11
:10D2880020212A46F019F3F785F82046F3F7D2FA59
:10D29800C8EB05056D08EDB2EF1902462146F019F5
:10D2A800BDE8F041F2F7CEBFBDE8F081F4010020FF
:10D2B800F0B5124B1A1894781F46ECB10E7800237B
:10D2C8003A1892781A4112F0010F4FF001020BD070
:10D2D800A6420D7803D09A4042EA050502E09A403A
:10D2E80025EA02050D7004E09A400D7825EA02024D
:10D2F8000A700133082BE3D1F0BD00BFC21C002027
:10D30800312200230178194111F0010F02D004499C
:10D31800C9180A7501330132082BD2B2F2D170470D
:10D32800F4010020034670B50846674A31B1127807
:10D33800532A40F0C880533A1A7070BD1278302AC8
:10D3480024D162491C780A7822400ED00A7802411A
:10D3580012F0010F05D0012282401C7824EA020253
:10D368001A7001300828F1D10CE00878104110F04B
:10D37800010F04D0012090401C782043187001321E
:10D38800082AF2D15248002113221AE0A2F13100F2
:10D39800C0B2072824D84D4A1278024112F0010F72
:10D3A80000F091801C7854FA00F212F0010F4FF04F
:10D3B80001020AD012FA00F024EA000444481C7062
:10D3C8001232BDE87040F2F7E5BF82404049441C84
:10D3D8004C741C7822431A70102246F6A5536EE04E
:10D3E800132A0BD0552A17D13A4A3B4912781820EC
:10D3F80000FB0212527912F0200F64D00024344D41
:10D40800194620466C74FFF753FF304B9B78002B6E
:10D4180059D0204629464FE0142A0BD02A2A16D183
:10D428002C4A2D491278182000FB0212527912F06A
:10D43800200F48D0264C0022194662740120FFF7BD
:10D4480037FF224BDB78002B3DD0012033E0152A33
:10D458000BD0232A16D11F4A1F491278182000FB27
:10D468000212527912F0200F2DD0194C00221946C1
:10D4780062740220FFF71CFF144B1B79002B22D08B
:10D48800022018E0162A0BD0442A1CD1114A12494E
:10D498001278182000FB0212527912F0200F12D0D5
:10D4A8000B4C0022194662740320FFF701FF074B5B
:10D4B8005B7943B103202146102246F6C553BDE8E7
:10D4C8007040FBF7FBB970BDEC1B0020C21C0020AC
:10D4D800EE1B0020B61C0020283900202DE9F04F53
:10D4E80087B09DF840408146072C0D4605929A4624
:10D4F80037D1073C27462B78234113F0010F2CD056
:10D50800012623B24FF000080293512031463246DB
:10D5180033460096CDF8048004F09CF91B20414660
:10D52800A2194346CDF80080F5F7E8F837B911207D
:10D5380039463A4633460097F5F7E0F8534B20460C
:10D5480013F8242001276FF3000203F8242011990F
:10D55800F5F750FF2046F6F757F90134082CCAD1E1
:10D568000DE2012C03780CD10BB90B7823B3FF2300
:10D5780000930021464B01911B780C200133029344
:10D5880016E0022C09D10BB90B78ABB10021FF23AF
:10D5980000930191029134200AE0062C0CD10BB9BA
:10D5A8000B784BB10021FF23009301910291652074
:10D5B80004220B4604F04EF9BAF1010F99F8003035
:10D5C8002BD13BB1334B0020D9790246534600900A
:10D5D800F5F794F82B783BB12E4B0120D97900222E
:10D5E80003460092F5F78AF80020F5F7F5FE99F85A
:10D5F8000030002B5BD0284B1978002957D1274BD6
:10D608005B78002B53D0FF2300933A2001220B466E
:10D618000191029104F01EF949E063B1052C4FF025
:10D62800000102D100910F2001E000910B200A4671
:10D638000123F5F763F82B7883B1052C4FF000012F
:10D6480006D110200A4601230091F5F757F812E099
:10D658000C200A4601230091F5F750F8022C25D03A
:10D66800032C01D10E4B02E0042C02D10D4B1F7884
:10D678001DE0052C01D10C4BF9E7012C01D1044B1D
:10D68800F5E7062C0CBFFF27002710E090180020B4
:10D6980071190020C21C00207E180020971100205C
:10D6A800DC1E00200B4C0020A73B0020FF2799F828
:10D6B8000030002B00F0B580934B944E1A789846B2
:10D6C80002F02002D2B262B1317811F0010108D122
:10D6D800FF230093282001220B460191029104F0B8
:10D6E800B9F898F8003003F01003DBB26BB1317869
:10D6F80001F00201C9B241B9FF2300932920012298
:10D708000B460191029104F0A5F898F8033013F044
:10D71800010F0DD0317801F00401C9B241B9FF23DE
:10D7280000932A2001220B460191029104F092F8FD
:10D7380098F8033003F00203DBB26BB1317801F0E3
:10D748000801C9B241B9FF2300932B2001220B46DF
:10D758000191029104F07EF898F8033003F0040375
:10D76800DBB26BB1317801F01001C9B241B9FF23C6
:10D7780000932C2001220B460191029104F06AF8D3
:10D7880098F8033003F00803DBB26BB1317801F08D
:10D798002001C9B241B9FF2300932D2001220B4675
:10D7A8000191029104F056F810F076FD68B13178D5
:10D7B80001F04001C9B241B9FF2300934920012279
:10D7C8000B460191029104F045F898F8033003F0F4
:10D7D8004003DBB26BB1317801F08001C9B241B9C5
:10D7E800FF2300934E2001220B460191029104F081
:10D7F80031F8767816F0010613D14548314616F00F
:10D808009EFA58B1FF230093731C00211BB20293A8
:10D81800752001220B46019104F01CF80136402EB8
:10D82800EBD1119B3B4A19783B4B51B199F8001049
:10D8380011702A781A702B780BB1542005E0522009
:10D8480003E011702A7853201A7004F0D1FB119B61
:10D8580000261A78314B1A7099F80030334113F0CA
:10D86800010F2DD03146059816F069FA01220146BC
:10D8780028B933B2019000920293104605E00021C6
:10D8880033B200920191029324200B4603F0E2FF89
:10D89800BAF1010F05D1224B8020DA790521013236
:10D8A80008E0022C07F1010202D18020072101E0E3
:10D8B800802006213346F6F7E3FA3046F5F778FF7D
:10D8C8002B78334113F0010F55D000214FF0010B95
:10D8D80033B2029302205A460B46CDF800B00191AC
:10D8E80003F0B8FFDA45DFF83C801DD118F8263080
:10D8F80013EA0B0332D10A4A0520D179009359441F
:10D9080006EB0B0228E000BF9C370020331A0020EA
:10D9180074180020DC180020DD180020511A00209F
:10D92800C21C00209018002018F8263013F00103BC
:10D9380014D1022C0CD1134B1B7803F02403042BB5
:10D9480004BF114B83F800B000230093072001E0C7
:10D9580000930620791C721CF4F7D0FE119930460A
:10D96800F5F748FD3046F5F74FFF18F826306FF306
:10D97800000308F826300136082E7FF46DAF07B093
:10D98800BDE8F08F5A1A0020901100202DE9F041CF
:10D9980080460E46174646F28B75002438462146C7
:10D9A80016F0CDF988B1294608220B4803F0E5FEA8
:10D9B8000948414616F070F9074816F093F920B95E
:10D9C8000123A34032781343337001340835082CFF
:10D9D800E4D1BDE8F08100BF491A00202DE9F043E9
:10D9E80087B08046894604A847F2B511082203F09B
:10D9F800C4FE002440462146E7B216F0A0F90028EC
:10DA080043D03846F4F7B4FB0025661C024631467D
:10DA180011202B460095F4F771FE012321462A4672
:10DA28000420FF080095F4F769FE4AF6EB30381831
:10DA380003F092FE04F00703C1B2194111F001018D
:10DA48004FF002024FF001030AD00092019336B260
:10DA58007720294692182B46029603F0FBFE14E025
:10DA68000092019336B2232004220B46029603F05B
:10DA7800F1FEB9F1000F08D004A8214616F05FF9AD
:10DA880018B10548214616F044F90134402CB1D1AB
:10DA980007B0BDE8F08300BFB91800202DE9F74FA3
:10DAA800174698463B7805460C469DF830909DF8F9
:10DAB80034B09DF83820DFF8B8A043B102EA030378
:10DAC8003B7009789AF800208A18D31A03702378D3
:10DAD80083B122482146F5F743FE21491F4816F035
:10DAE800DBF81E480121FFF779FF1C484146224612
:10DAF800FFF74CFF1B4B00261E70297843F6F820D1
:10DB080003F020FE494646F2C96003F01BFE20469A
:10DB180039464A46F5F724FC134B42469E7039466F
:10DB28004B462046CDF800B00195FFF7D7FC2846B4
:10DB3800F8F7A6FB2B780D480D498AF80030F5F761
:10DB48000FFE11F01FFB88F800603E7026702E70E3
:10DB580003B0BDE8F04F04F055B900BF521A0020D9
:10DB6800D4180020001D002097110020351A00202D
:10DB78007E18002010B50B4B0B4C024603CB2060DF
:10DB880061600A48114616F0A8F82146074816F0C1
:10DB980083F8064816F0A6F8D0F1010038BF002037
:10DBA80010BD00BF5C2B00203F1A0020491A00203E
:10DBB80010B50A4CA37C4BB100200949FAF732FF93
:10DBC800084B1B78432B01D1433BA374A07C20B99D
:10DBD8000549BDE81040FAF725BF10BDEE1B00202F
:10DBE8009DEA0208EC1B00207CEA0208034B1A7825
:10DBF80001321A7001230370704700BF001D002016
:10DC080010B50C48FAF7B4FE0B4A002414700B4AFE
:10DC18000B4B14700B4ADC7014700B4A9C70147018
:10DC28000A4A14700A4A1470FAF7C0FF094B1C60BC
:10DC380010BD00BF141D0020C21C0020ED1B0020D9
:10DC480097110020041D0020111D0020281C002011
:10DC5800001D0020241C00202DE9F04F934B944E0A
:10DC680093F800903368DFF894829C7C914BF02203
:10DC78001A7098F800308BB00D2B354647463DD1C9
:10DC88008D4B93F803C0BCF1010F02D900208B49DA
:10DC98002FE01AD10024DC70894A8A4B8A498B48C4
:10DCA8008B4D04701C7014700C70CDF800C001947A
:10DCB8002D780295FFF7F2FEFAF778FF8548346071
:10DCC8000BB0BDE8F04FFAF753BE83487E49F5F72D
:10DCD80047FD824B824A03CB824B10601B78516010
:10DCE800532B57D198F800307F49013388F800301A
:10DCF80000200BB0BDE8F04FFAF794BE092B0FD106
:10DD0800784B1B78532B3DD1784B00221A700D238A
:10DD180088F80030764B1A7842F006021A707FE2D3
:10DD28000E2B37D16F4B1B78532B2BD171496A4877
:10DD380015F0B2FF6848FFF71DFF044640B198F898
:10DD480000300522013B88F800305B4BDA7067E24F
:10DD5800082246F2CA61624803F00FFD604966482E
:10DD680015F0BBFF01230093594B01941B785748CA
:10DD780002935549524A534BFFF790FEFAF716FFA4
:10DD880034604DE2232B40F04B820BB0BDE8F04FDE
:10DD9800FFF736BF631E48BFA31DDB10013303FB2B
:10DDA80009F91FFA89F909F5CC46A9F5A849A9F195
:10DDB80015094F4BCDF81C901A78CA3612F0010F8E
:10DDC8004A4C00F01E81474B1A789946432A40F086
:10DDD800C7803B780D2B40F0C3803F48217815F071
:10DDE800AEFF002800F0BC803D48217815F0A7FF61
:10DDF800002840F0B580079920780FFA81FB0BEBDB
:10DE0800D00003F0A9FC23784FF0010A03F00702C1
:10DE18000AFA02FADFF8E8805FFA8AFA10EA0A0FCB
:10DE2800C8F8000027D0244B5B78002B40F098807E
:10DE3800274BD879F8F782F9002800F09180D8F8B4
:10DE48000010CAF1FF0A20780AEA0101C8F8001098
:10DE58000BEBD00003F076FC20780FFA86FB0BEB77
:10DE6800D00003F079FC00EA0A012078C8F8001015
:10DE78000BEBD0005FE032B202EBD300059203F067
:10DE88006BFC10EA0A0FC8F800003BD140EA0A010F
:10DE9800059B2078C8F8001003EBD00003F052FC73
:10DEA8002178154815F035FF5AE000BFB31C002053
:10DEB800241C00200F1D00209711002042EB0208AF
:10DEC800041D0020ED1B0020111D0020281C00202F
:10DED800C21C0020141D0020521A00205C2B0020B8
:10DEE8006C180020EC1B002008EC0208BE1C002067
:10DEF800031D0020C9180020D4180020001D002090
:10DF0800CC1C0020924B5B7823B9924BD879F8F758
:10DF180015F9B8B92078DDF814C0CAF1FF0A0CEB7E
:10DF2800D00003F019FC8C4A00EA0A01059B20780E
:10DF3800116003EBD00003F005FC2178874815F049
:10DF4800F3FE0DE020780BEBD00003F005FC40EA6F
:10DF58000A012078C8F800100BEBD00003F0F2FBA0
:10DF680099F80030232B10D12A682378927C013A43
:10DF780093420ADA7A4A013313707A4B9B7803F09A
:10DF88000203DBB20BB1FAF749FC99F800302A2BEF
:10DF98000CD1237853B1724A013B1370714B9B78B3
:10DFA80003F00203DBB20BB1FAF738FC99F8003042
:10DFB800552B12D129682278897C694B08398A4205
:10DFC80001DA083200E000221A70664B9B7803F0F1
:10DFD8000203DBB20BB1FAF721FC99F80030442BAD
:10DFE8000FD122785E4B072A9CBF2A68927C083A98
:10DFF8001A705C4B9B7803F00203DBB20BB1FAF7A3
:10E008000DFCFBF7CBFD584A2378117892469942CC
:10E0180088BF137012780F32934202DD524A0F3BC9
:10E0280013702B684FF0000B93F81280CDF818B0DE
:10E03800B8F10F0F9ABFC8F120085FFA88F84FF0BF
:10E04800100839784FFA8BF30D2905D19AF800207A
:10E058009B18DB10454A04E09AF800209B18444AB4
:10E06800DB10D35C9AF8002005934FFA8BF39A18CB
:10E078000D2902F007094FEAE20202D13D49895C05
:10E088000691DDF81CC004930FFA8CF0101803F009
:10E0980063FBC0B2049B08909AF8000032B21818CB
:10E0A80002EBE00003F058FB39789AF80020049B53
:10E0B800C0B209919A1846E0059BDDF824C043FADE
:10E0C80009F12D4B01F0010100290CBFA521DB212D
:10E0D800BCF10D0F03F8081014D128494FEAE20CDF
:10E0E80011F80C1041FA09F111F0010F08D0DDF810
:10E0F80018C04CFA09F111F0010F03D0582110E0B3
:10E108002D210EE0DDF820C04CFA09F111F0010FC5
:10E1180001D0502105E040FA09F111F0010F02D0B9
:10E12800542103F8081009F101095FFA89F90BF184
:10E13800010B08F101080132B9F1080F5FFA8BFBF6
:10E148005FFA88F81CD0B8F1200FB5D125E000BFE0
:10E1580097110020C21C0020CC1C0020D4180020DD
:10E16800BE1C0020141D0020B51C0020C91800206A
:10E17800291900206C180020F4010020521A0020F0
:10E18800B8F1200F09D09AF800304FFA8BF2D21864
:10E198002B689B7C9A42FFF654AF23490B7813F007
:10E1A800010F17D02B68214A9B7C12780F2B02F0A5
:10E1B800800298BFC3F11003D2B294BFDBB2002330
:10E1C80042B122789AF800101032521A1849CB1826
:10E1D8005F219954174EB37803F00203DBB293B171
:10E1E800F11D652246F661432078FAF767FB2B6834
:10E1F8009B7C102B02D905200B2101E00020072170
:10E208003246FAF7C7FB2B689B7C102B08D921787C
:10E218000948013102220BB0BDE8F04FFAF728BCDB
:10E228000BB0BDE8F08F00BF031D00209C37002015
:10E23800F4010020141D0020F50100202DE9F04113
:10E24800002386B08DF81730624B1B78012B00F045
:10E258007682614C227872B1604B5B78002B40F07B
:10E268006E825F4D2B78002B40F0DA80FAF79EFC27
:10E2780009232B70D4E05A4B19781D46082900F25F
:10E28800CF8058490978232913D11A70FAF78EFCE0
:10E298005549564A0B7853B15548013B0478DBB2CF
:10E2A80044F0060404700B70524951F8233013608F
:10E2B800AEE24F4B1A7812F0010F04D101210A4344
:10E2C8008DF817101A70F4F74DFE28B92B781BB982
:10E2D8000DF11700FFF78AFCF4F752FE30B92B78DE
:10E2E800012B03D10DF11700FFF780FCF4F756FE60
:10E2F80030B92B78022B03D10DF11700FFF776FC0C
:10E30800F4F758FE30B92B78032B03D10DF1170021
:10E31800FFF76CFCF4F75CFE48B9F4F785FE30B9FA
:10E328002B78042B03D10DF11700FFF75FFCF4F7EE
:10E33800AFFE30B92B78052B03D10DF11700FFF78D
:10E3480055FCF4F799FE30B92B78062B03D10DF163
:10E358001700FFF74BFCF4F749FE30B92B78072B71
:10E3680003D10DF11700FFF741FCF4F74DFE30B96A
:10E378002B78082B03D10DF11700FFF737FC9DF818
:10E388001730002B4CD02B78082B47D8DFE803F048
:10E3980005080D101316191C1F000020164901E06E
:10E3A80016490020FAF73EFB3AE000201449F9E745
:10E3B80000201449F6E700201349F3E70020134929
:10E3C800F0E700201249EDE700201249EAE70020B3
:10E3D8001149E7E70F1D00207E1800209711002043
:10E3E800001D0020EC1B0020E31C0020241C002042
:10E3F800031D0020F01C002028F0020807F0020886
:10E4080049F002086AF002088BF00208ACF0020832
:10E41800CDF00208EEF002080FF10208FAF7C6FB89
:10E428008C4F3B783D46092B40F093808A4B8B4FAD
:10E438001978984611F00101894E23D113223046EC
:10E44800F1F7A8FF0123B374864A2378137003B940
:10E45800B374B37C13B1844B00221A70FFF7A8FB86
:10E468008048B17CFEF75EFF98F8003003F0FD03AA
:10E4780043F0010388F800307C4B1A7812B13A70E7
:10E4880000221A703B78002B4FD0FFF791FB75489C
:10E49800B17CFEF747FF734B1A78984622B10020EB
:10E4A80010216F4AFEF7DEFE2378387898F800408E
:10E4B8006F4924EA0302A0F152070A70FFB26D4ABD
:10E4C80023EA040E012F82F800E012D854B9BEF1F5
:10E4D800000F07D001230093674B01941B78614814
:10E4E800029365E1654B0422DA702B7801332B70B7
:10E4F8001BE0432819D1C3B9604C6778AFB95E4BAC
:10E50800D879F7F71BFE38B95D49FAF78BFA052376
:10E51800E37008332B7004E038465A49FAF782FA58
:10E52800E770594A594B1A6072E14E48FEF7E8FE07
:10E53800737C002B00F06C81554A127802F080023F
:10E54800D2B2002A00F06481524AD3182022DA7429
:10E558005EE10A2B31D1464809F078FAC6B2474C39
:10E5680036B3E378042B02D100204B4903E0022B99
:10E5780004D14A490020FAF755FA02E00BB90433EE
:10E58800E370314602224348FAF772FA334B1E7899
:10E59800232E00F0D4803046FAF700FB002800F064
:10E5A8003781312E40F034812B7801332B7002E013
:10E5B8003B7801333B70042332E00B2B32D12C48DB
:10E5C80009F02AFAC6B22D4C36B3E378042B02D1EF
:10E5D8000020334903E0022B04D132490020FAF726
:10E5E80021FA02E00BB90433E370314602222948CC
:10E5F800FAF73EFA194B1E78232E00F0A080304619
:10E60800FAF7CCFA002800F00381312E40F000819F
:10E618002B7801332B7002E03B7801333B700823E1
:10E62800E370F5E00C2B40F0F3801148002109F06D
:10E63800C9F9C4B2002C78D0104FBB783E46002BE5
:10E6480038D10D4BD879F7F779FD68BB03233B71B7
:10E6580075E000BF001D0020031D0020EC1B0020FA
:10E66800EE1B0020281C002090110020B81C002060
:10E67800111D0020041D0020C21C0020971100203D
:10E6880042EB0208BEEA020864640208241C002067
:10E698009C370020F4010020C6EB0208E7EB0208D3
:10E6A80084EB0208A5EB0208BE2016F035F9BB780A
:10E6B8000133BB70F378584A092B02D90020574917
:10E6C80015E010D1564B00241C70D470554B564A97
:10E6D8005649574801251C7014700C700470009539
:10E6E8000194029465E0082B04D152490020FAF7FE
:10E6F80099F911E0062B02D100204F49F7E7042BC6
:10E7080002D100204D49F2E7022B02D100204C49EA
:10E71800EDE70BB90833D370F378082B0BD84948C9
:10E7280021460222FAF7A4F905E0012300933C4BA5
:10E7380001941B7838E0444F3C78232C02D1FFF732
:10E748005FFA65E02046FAF729FA002860D0303CE5
:10E75800E4B2631EDBB2012B3C7031D8022C304D81
:10E768001DD1E879F7F7EAFC002830D03748FFF7E1
:10E7780001FA00282BD1082246F2CA61344802F077
:10E78800FCFF3249324815F092FA314946F2CA6024
:10E79800082202F0ECFF2F482D4915F09EFA0123BC
:10E7A8000024009301942B78214820491E4A0293A3
:10E7B8001C4BFFF773F9FAF7F9F9274B1C6027E0B0
:10E7C800032C25D1164BD879F7F7B8FC10B90C23D0
:10E7D800F3701DE000241D48214615F0B0FA28B159
:10E7E800E02016F099F8204616F0D2F80134402CB3
:10E7F800F1D11A4A00231370F3702B78184A0133A9
:10E808002B70154B1A60174B1A7842F006021A70D3
:10E8180006B0BDE8F08100BF9711002042EB020866
:10E82800C21C0020ED1B0020041D0020111D00202B
:10E83800281C0020DFEA020800EB020821EB02088E
:10E8480063EB0208F4010020EC1B0020521A0020A0
:10E858006C180020D4180020241C0020BE1C0020A6
:10E8680064640208031D002088234B43054A03EB18
:10E87800D003D35C00F0070053FA00F000F0010069
:10E88800704700BF4C0D002070B504461646157839
:10E8980039B912E00135EDB228462146FFF7E4FF09
:10E8A80048B9202DF6D970BD013DEDB22846214664
:10E8B800FFF7DAFF08B1356070BD002DF4D170BDE7
:10E8C800074B400119784423013909180548C9B292
:10E8D8000370173BC370013101300222FAF7C8B840
:10E8E800BE1C0020F4010020012802D0022806D115
:10E8F80002E01D20044904E01D20044901E0044908
:10E908001D20FAF78FB800BFE9E30208C8E3020840
:10E918000AE402082DE9F04FA44BDFF8E082F02268
:10E928001A70D8F8003087B09C6847F23753E11A5C
:10E938004C4244EB0104DD3A62439D4B9E5C03EB81
:10E948000209C6F30006F7B24246002F2DD1384619
:10E958009849FAF767F8984B1B78232B41F0A18167
:10E9680099F8013067F3041389F80130FAF71EF9B2
:10E97800924B1A7842F006021A70914A1378013BBA
:10E98800DBB213708F4A52F82330C8F800308E4B30
:10E998001E708E4B1E708E4B1E708E4B1F608E4BE2
:10E9A8001E708E4B1E7001F07CB98B4E96F800B02D
:10E9B800BBF1000F0AD04FF4D06161430BF1FF3077
:10E9C800342303FB00138649CB181D79854B1F7828
:10E9D80077B1854F2046397810F0BEFA002840F00C
:10E9E800FC83804938700870804607468146FDE3FD
:10E9F80078490B68A3F11200032809D9A3F116017D
:10EA0800032909D9A3F11A01032909D9B84605E050
:10EA1800B8464FF0010906E0B8460127C14602E0B2
:10EA28004FF00108B94664490978532940F0BA8182
:10EA3800BBF1000F29D1422060436C4A115C11F0F0
:10EA4800020F0AD0002B41F02C81013363F38301BC
:10EA58001154604A136001F024B9DFF854C113233C
:10EA680003FB04C35A7820466BF304125A70604BB8
:10EA7800022183F800B010F03BFA564801233370A6
:10EA8800C0F800B0FAF792F888E10BF1FF312046A0
:10EA9800C9B210F061FA002852D1564BDFF83CB1E8
:10EAA8001978012229B91A70474B8BF80010197090
:10EAB8009CE3049003920293FAF778F80498029B77
:10EAC8001870039A8BF800204B4A835C9146A3F197
:10EAD8003001C9B2092904D9413BDBB2052B01F247
:10EAE800E08001300A28EFD14FF00008474609EBD3
:10EAF800480015F059F97B080237FFB20A2F3E4D3E
:10EB080009F8030008F10108F1D1284610F014FEB5
:10EB1800002801F0C680284610F094FB002841F038
:10EB2800C08031782B7901390090C9B22046022281
:10EB3800019510F047FE02238BF8003001F0B1B8C0
:10EB4800DFF890B059460A68202A01D121232AE02B
:10EB5800212A25D14FF4D063634331781332013928
:10EB680002FB01331E4A4FF0000C9B18019303224D
:10EB78002B462046C9B2CDF800C0CDF810C010F021
:10EB880021FEFAF713F83278174B013A1A70DDF8BC
:10EB980010C01423CBF800C086F800C0114AF6E074
:10EBA8001E2A2DD11F23CBF8003001E30F1D0020B2
:10EBB800B03700203FD60208EC1B0020031D0020C0
:10EBC800E31C0020F01C0020091C0020321C00203F
:10EBD800B31C0020CC1C0020BE1C0020B51C00204B
:10EBE800143D0020011C0020B41C0020144A002001
:10EBF800021D0020BF1C0020E41C0020241C002053
:10EC08001F2A1BD14FF4D063634331781532013981
:10EC180002FB0133A84A4FF0000C9B1801932046D1
:10EC2800C9B206222B46CDF800C0CDF810C010F0AE
:10EC3800C9FDDDF810C0CBF800C0B9E2931F062B60
:10EC48000ED89E4B1A7819462AB901321A709C4B75
:10EC58001A789C4BBAE2012A40F0C88202239EE14E
:10EC6800A2F10D03042B39D8974996F800E091F8E2
:10EC780000C0DBB29048954ABCF1000F1DD04FF0A0
:10EC8800000C81F800C011784FF4D06262430EF195
:10EC9800FF3E0CF1340C0CFB0E228018C018417496
:10ECA800600186445FFA8EF000EB800000F5EE40CC
:10ECB8009730C01802F046FD98E24FF0010C81F839
:10ECC80000C04FF4D06161430EF1FF3E0CF1330CEC
:10ECD8000CFB0E1E7044C3185B7C58E0A2F11203B3
:10ECE8000B2B4BD87A4B31781878002844D0002069
:10ECF8001870A2F1120B63014A1ED218D2B218235F
:10ED08005A4302F5F042734B5FFA8BFBD73202EBA2
:10ED18004B02197810460392029302F013FD6E49D4
:10ED28004FF01A0C08784FF450716143013805917F
:10ED38000CFB0011029BDFF880E11B7859440EEBB5
:10ED480041018B75039A654B501C19780293CDF8D5
:10ED580010C002F0F7FC6048DDF810C00278059991
:10ED6800013A0CFB0212029BDFF84CC15A441B7893
:10ED78000CEB4202D37539E2012227E2DFF864B1D5
:10ED88009BF800302BB901228BF80020544A1370ED
:10ED98002CE2F9F70BFF00238BF800302046FFF731
:10EDA8008FFD23E243294ED1444A1278002A40F0CD
:10EDB8001D82454A1278002A40F01882BBF1000FE4
:10EDC80000F01482474A1278002A40F00F82212B63
:10EDD80031D01F2B33D03E4B197801291AD9B9F1FC
:10EDE800000F03D1B8F1000F00F00082394B02394F
:10EDF8001A7852FA01F010F0010F4FF0010004D018
:10EE080010FA01F122EA0102E0E110FA01F141EA07
:10EE18000202DBE100F0EA810BF1FF312046C9B2C2
:10EE280010F09AF820B9304B1B78002B40F0DE81A7
:10EE380000233370BCE12D4820230360B8E12B493F
:10EE48001E230B60B4E1232940F092801B4B1B78F2
:10EE5800002B40F0CB811C4B1978002940F0C6816B
:10EE6800204BBBF1000F4ED01A782AB11C480F2A4C
:10EE780001701F48017017E10BF1FF312046C9B23C
:10EE880010F06AF8002835D0114A137883B1B9F127
:10EE9800000F01D0082B09D90FB1012B06D9B8F101
:10EEA800000F00F0A381042B00F29C8101336EE770
:10EEB8002846012179E100BF143D0020021D0020F1
:10EEC800B21C0020101D0020CB1C0020801D00203B
:10EED800B71C0020B11C0020BE1C0020011D002012
:10EEE800091C0020B31C0020BF1C0020CC1C0020E3
:10EEF800321C00208B4B1A78511EC9B208296CD8D5
:10EF080001321A7069E0DFF85CC2132101FB04C109
:10EF180048786BF30410487002212046039202934C
:10EF28000FF0E6FF08F05AFCF9F740FE7E49087832
:10EF380040F0060008707D4801780139C9B20170B7
:10EF48007B48039A50F821107A4811607A4A82F86F
:10EF580000B07A4A82F800B0029BC0F800B083F88B
:10EF680000B0774B86F800B083F800B000F099BE87
:10EF78002A2935D1734B1B78002B40F03781724B0F
:10EF88001A78002A40F0328170490B784BB16A48F0
:10EF9800012B02706948027040F22881013B0B7016
:10EFA80024E1BBF1000F00F021810BF1FF31204675
:10EFB800C9B20FF0D1FF50B1654A137823B1012BC4
:10EFC80040F21481013BE2E628460021EDE0554A73
:10EFD8001378012B01D9013B13700022564BF5E041
:10EFE800442967D1574A1278002A40F0FF80574ACF
:10EFF8001278002A40F0FA804A4A1278002A40F033
:10F00800F580514A1278002A45D1514A1278012ACE
:10F0180009D9002F00F0EA804E4B1A78102A00F226
:10F02800E480013267E015D1B9F1000F09D04A4BED
:10F0380003201978013191FBF0F000EB4000091A28
:10F0480066E0002F00F0D280434B1978013101F0BF
:10F05800030163E00BF1FF32D2B21E2A00F2C68030
:10F06800212B00F0C3801F2B00F0C0800BF1010B97
:10F07800204686F800B0FFF723FC4FF4D0626243C5
:10F0880031783423013903FB0123344A2949D31841
:10F098001D79087883E00D2B0AD128460FF064FE0D
:10F0A80030B12F4B1A783F2A00F2A08001328DE050
:10F0B80001208EE0552940F09980224A1278002AD2
:10F0C80040F09480214A1278002A40F08F80154A37
:10F0D8001278002A40F08A801B4A1278002A6AD1E6
:10F0E8001B4A1278012A08D9002F7FD0194B1A78A9
:10F0F800012A7AD9013A1A7077E035D1164B197876
:10F1080011B10139197071E0B9F1000F03D0022172
:10F11800197091466AE0002F68D0032119701746CC
:10F1280064E000BFBF1C0020031D0020E31C00207A
:10F13800F01C0020CC1C0020091C0020321C0020E0
:10F14800B51C0020021D0020CB1C0020B31C002091
:10F15800B71C0020B11C0020011D0020143D002018
:10F16800801D0020B0370020BBF1010F3ED9212BB4
:10F178003CD01F2B3AD00BF1FF3B204686F800B05D
:10F18800FFF79EFB4FF4D062624331783423013994
:10F1980003FB01238E4AD3188E4A1D79107829461D
:10F1A800FFF762FB014618B928468A4AFFF76CFB4D
:10F1B800F9F7FCFC1AE00D2B0AD128460FF0D4FD14
:10F1C80030B1854B1A78012A10D9013A1A700DE02E
:10F1D800FF2081490FF0E6FC08E04FF000084746A1
:10F1E800C14603E04FF0010800E001273178DFF85D
:10F1F80054B2002970D19BF8003013F0010205D1F8
:10F2080043F001038BF80030724B1A60002520464A
:10F21800294610F03DF830B1422363436F4AD15C70
:10F2280041F00201D1540135202DF0D1223565433A
:10F238006A4E735D13F0020F43F3400015D0654C1E
:10F24800206810B9664900F096BC00206549F9F7B6
:10F25800E9FB735D13F00C0F43F3810540F0218542
:10F26800F9F7A4FC256000F01CBD14B920465E49DE
:10F2780000E05E49F9F7D6FB5D4803786BB95D4954
:10F288000A225D48F1F75CFB5C49132303FB041376
:10F298005A7842F010025A7004E0574858490A2236
:10F2A800F1F74EFB20460FF067FE564C014602224E
:10F2B80004F11900F9F7DCFB534B00221A70534B89
:10F2C8001B7803F08003DBB2002B00F0EA84504B7C
:10F2D8001B88E38100F0E5BC01392046C9B20FF074
:10F2E8003BFE002800F024844A4B62011B78013B56
:10F2F8009B18DBB205939BF8003013F0010F03D085
:10F30800414A1378002B42D04348F9F731FB059B5B
:10F31800102203EB031101F5E6414048173102F0D2
:10F328002CFA3D4B11229A712A4B1B6813B91020F5
:10F338003B4921E0012B02D110203A491CE0022B65
:10F3480002D11020384917E0052B02D11020374987
:10F3580012E01E2B02D1102035490DE01F2B02D1DF
:10F368001020344908E0202B02D11020324903E054
:10F37800212B03D131491020F9F754FB9BF80030B9
:10F38800214843F001038BF80030002303702C4B15
:10F398001A78002A00F0EE800599102201EB01137B
:10F3A80003F5E643173317481946059302F0E5F9C4
:10F3B80000229346134B995C002945D00BF1010BB1
:10F3C8005FFA8BFB0132BBF1100FF3D144E000BFB1
:10F3D800143D0020CC1C0020801D0020144A002071
:10F3E80081D60208A2D60208E4D6020868D7020825
:10F3F800011C0020AAD70208FA010020B03700201B
:10F40800CBD70208F4010020B51C00209C3700204F
:10F41800E9470308BE1C0020141D00201B1D002006
:10F4280023E30208B2D80208F4D80208BAD90208BD
:10F438005FDA020880DA0208A1DA0208C2DA0208F2
:10F44800B31C0020031D00209E4B202103EB0B0062
:10F45800C2F11002F0F79EFF9B49087858450DD974
:10F46800059A0138801802F077F938B9964B2021AF
:10F478001878059B0138C01802F064F9DFF88CB2DF
:10F488009BF8003018460293F9F788FBDC46029B8C
:10F49800DFF848B210B9432B46D101E0432B05D120
:10F4A80000238BF800304FF0200A31E08748884A63
:10F4B80090F800E087499E450FD1AEF130004FF03B
:10F4C8000A0E13780EFB001E0133DBB2137073446F
:10F4D80093F8AD307BB913700DE003709BF80030E2
:10F4E8004FF0000E82F800E02BB1774B18780F2808
:10F4F80001D80130187040238BF8003013789CF83D
:10F5080000200A20303A00FB0211C91891F8ADA07A
:10F518006D496C4A0878059B013802F800A05146ED
:10F52800181802F00FF90FE06B4B1B7803F08003FB
:10F53800DBB24BB19BF8003033B9634861490378BB
:10F54800FF22CB1803F8012C9BF8003013B1634A53
:10F55800013B13709BF80030012B10D15A4A1378E5
:10F568000F2B01D801331370594A00238BF8003050
:10F57800137004E004200C21594AF9F70BFA594A90
:10F5880013689346E3B94FF4D06262433178342468
:10F59800013904FB0124544AA4186178494AC1F38B
:10F5A800C30109B93F2004E0994201D9DB2000E0FA
:10F5B800A5200133DBB2907501320A2BF1D170E33B
:10F5C800012B13D14FF4D063634332783424013ACA
:10F5D80004FB0234444BE418637813F0070300F08B
:10F5E8006083142141485943832236E1022B24D1F8
:10F5F8003F4B882202FB05353178E8793D4A0139CD
:10F608000623202502F8015950FA03F515F0010FD9
:10F6180010D04FF4D0656543342606FB0155364EAD
:10F628007519ED791D4115F0010F01D0DB2500E0BA
:10F63800A5255570013BE4D233E3032B13D14FF4D6
:10F64800D063634332783424013A04FB02342A4BF2
:10F658001C19237A13F0010F02D0102027498AE2DF
:10F668001020274987E2042B13D14FF4D06363435A
:10F6780032783424013A04FB02341F4B1C19237AD4
:10F6880013F0020F02D010201E4974E210201E4908
:10F6980071E2052B3CD11627002533783422013B33
:10F6A80053434FF4D06202FB0433134A0549D3187D
:10F6B800585DC919013514F05DFB0237052DECD1F1
:10F6C800EFE200BFF4010020B31C0020061C00205C
:10F6D800321C0020C06202089C370020091C002050
:10F6E800141D0020CC1C00201C3D00200F0200200F
:10F6F8004C0D002013020020143D002057D90208A9
:10F7080078D902081DDA0208FCD90208EC1B00208F
:10F718009A1F062A00F2CA8005EB0511944F8A1831
:10F7280007EBC202D268934902F1100052F804EBC9
:10F73800824241F804EBF9D1063BDBB205EB051236
:10F74800D2188D48013207EBC20292F809C092F82C
:10F758000AE00278317881467AB94FF4D06363437E
:10F768003432013902FB0131844BCA5E844B42FAC0
:10F778000CF202EA0E021A7010E0022A0ED1814A37
:10F78800013912784FF0000800922046C9B20422CD
:10F79800CDF8048010F016F889F8008099F8003048
:10F7A800012B2AD1784BDFF8DC8193F800A0504672
:10F7B800F9F7F4F910B9BAF1430F1BD1DBF80030AF
:10F7C80005EB0512063BD21807EBC202D1686F4A57
:10F7D800914202D1002288F8002005EB0512D318C7
:10F7E80007EBC303504698F800101A7CFAF7F6F9AD
:10F7F80088F8000098F800A003E013B9604B93F86C
:10F8080000A0BAF1090F07D9BAF1630F8CBF4FF006
:10F8180003084FF0020801E04FF001085C4820217E
:10F828000322F0F7B7FD99F80030DBB94FF4D06345
:10F83800634332783424013A04FB0234554BE4180C
:10F84800A37813F0080F15D051483F2103226AE12D
:10F8580051485146C8EB0000424607B0BDE8F04F9A
:10F86800F9F706B94D4B1B7803F08003DBB2002B88
:10F8780040F01782DBF8003005EB0512D31807EBD0
:10F88800C30757F8243C414A9342E1D1384A8821BA
:10F8980001FB0525A3F58863AA68013B9A42D7D0E6
:10F8A800504607B0BDE8F04FFFF71EB8A3F10D02B0
:10F8B800042A2FD8D7B2222303FB05752C4B03EB60
:10F8C80085056D6C2846F0F7B5FF2946024629489C
:10F8D800F1F736F8324B1B786BB1304B1B7803F0DD
:10F8E8008003DBB21BB12F48202102221BE12E4BE3
:10F8F8002C4819780CE04FF4D063634332783424F1
:10F90800013A04FB0234294B26481C19E719797C73
:10F918008222A2E7123B0B2B00F2C3812222DBB228
:10F9280002FB0535124A163552F82520114902F115
:10F9380010008A4652F8045B824241F8045BF9D110
:10F948001B4DDFF874B0B8F1000F04D02A78012AF3
:10F958003BD1013209E0002F37D02A78012A2DD96E
:10F9680014490978032930D1013A2A702DE000BFE3
:10F978004C0D002004020020021D0020193D00202B
:10F98800B21C0020101D0020EC1B0020A7E3020879
:10F99800110200201C3D0020140200209C3700208A
:10F9A800CB1C002012020020801D0020143D0020E6
:10F9B800B71C0020011D0020B11C002005D183497F
:10F9C8000978032908BF8BF800202A789AB94FF4E0
:10F9D80050714C4332781A21013A01FB02447C4AA7
:10F9E800E318083302EB43039A798BF80020DA799D
:10F9F800764B1A7055E1774C202104F11800082243
:10FA0800F0F7C8FCB9F1000F00D1AFB16F4E3378F1
:10FA1800012B01D1704A01E04BB9704A1368236188
:10FA28005368CAF80430B9F1000F2ED00BE0022B4E
:10FA38000CBF6B4A6B4AF1E76B4A13682361536842
:10FA4800CAF8043027E19BF80000624A31210023FC
:10FA580050FA03F616F0010F01D0117601E02D26B9
:10FA68001676013301310132082BC9B2F0D15F4B50
:10FA78001B7803F08003DBB2002B41D02B78012BDD
:10FA88003ED9E4182023A3753AE0002F00F0038143
:10FA9800202108225648F0F77DFC56489BF80010B4
:10FAA8008222F8F7E5FF514B1B7803F08003DBB2A5
:10FAB80013B12B78012B02D83378032B20D12021C6
:10FAC80002224C48F0F766FC1AE050FA03F616F0EA
:10FAD800010F01D0117701E02D261677013301318E
:10FAE8000132042BC9B2F0D1404B1B7803F08003DC
:10FAF800DBB22BB12B78012B02D9E4182023A37693
:10FB08003A4B1B7803F08003DBB2002B00F0C9806E
:10FB18002B78012B40F0C580B8F1000F40F0C18070
:10FB280035482021082207B0BDE8F04FF0F732BC75
:10FB38009BF80030314D13F0010F04BF43F001036F
:10FB48008BF800302E78DEB92D210A222C48F0F7E8
:10FB580021FC04202B49F8F765FF2B4B1B78012B60
:10FB680002D11020294906E0022B02D11020284991
:10FB780001E02849102007B0BDE8F04FF8F752BF60
:10FB8800254B1C782046F9F709F8244B1C4A002815
:10FB98005BD0234F23493878A04247D130380C78BE
:10FBA800214E00EB80073C19345D04B90C700F78C6
:10FBB80000EB8000C4190137FFB2C0190F70315C27
:10FBC800345D00293BD11748017038E0011D002041
:10FBD800143D0020F40100205DE202087EE20208E4
:10FBE8009FE20208C0E20208D9E102089C3700201F
:10FBF8000C0200201202002004020020BF1C00207A
:10FC0800E41C00204CE40208B51C0020DBD90208E3
:10FC180099D90208BAD90208EC1B0020091C002057
:10FC2800061C0020321C0020C06202080120087057
:10FC380019783C7019B1092E9CBF36182E70297896
:10FC4800511801F8014C40211970197811B1164862
:10FC5800013901701978012909D12978092902D8AF
:10FC680012480131017000211970114B1970116887
:10FC7800104BC3F816105168C3F81A101289DA83AA
:10FC88000D4A127802F08002D2B252B12A789B183B
:10FC980020225A7505E09BF80000064A312100230E
:10FCA80013E707B0BDE8F08F091C0020BF1C002037
:10FCB800321C0020F40100209C3700201FB50446A8
:10FCC80011B100200B4901E008460B49F8F7AAFEDC
:10FCD800217810220139C9B201EB011101F5C241A5
:10FCE8004431684601F049FD102001466A46FDF797
:10FCF800B9FA1FBD4CC302088EC302080B4B1B7810
:10FD0800442B06D0552B037801D013B17047013B23
:10FD180001E003780133037003780BB9403302E044
:10FD2800412B01D1403B0370FFF7C8BFEC1B0020FB
:10FD38002DE9F74FDFF8C881DFF8D4A198F8003033
:10FD4800554643F0010388F800309AF80130624CB8
:10FD580023F07F039B46D3B100206049F8F762FE89
:10FD68005F482A21F0F794FB18B121788222F8F72E
:10FD78007FFE2278002A40F0AB802B6862F3CF33F5
:10FD88002B60584B1A7842F003021A70A0E0DFF893
:10FD98005491237099F800304E4603F00202D2B213
:10FDA8000192514F002A40D013F0010813D0584651
:10FDB8004E49F8F737FE3B78232B20D14C4B4D4A60
:10FDC8004D481A600121FFF779FF337803F0FE03ED
:10FDD8006BF3410312E040464849F8F723FE3B78AD
:10FDE800232B0CD1424B434A43481A600121FFF7A9
:10FDF80065FF337868F3000368F3410333703B7899
:10FE08002A2B65D1337803F0FE036FF34103337077
:10FE18002B6843F400432B600F232370364B18786C
:10FE280003B0BDE8F04F0DF0BBBC0DF003FC054678
:10FE380000282DD001213048FFF760FF3B78532B75
:10FE480012D13378019A03F0FD0362F30003337093
:10FE5800DAF8003043F40043CAF800300F23237067
:10FE6800254B18780DF09CFC3B78232B30D1337848
:10FE7800002203F0FD036FF3000333701E4B1A706A
:10FE8800F8F794FE1E4A137843F00603137015E042
:10FE98001C49F8F7C7FD3B78232B19D199F8003096
:10FEA80065F3410365F3000389F80030F8F77EFE37
:10FEB80098F8003043F0060388F80030124A1378A7
:10FEC800013BDBB21370114A52F82320084B1A6029
:10FED80003B0BDE8F08F00BF164D0020D0C3020864
:10FEE800F4010020AB3A0020EC1B0020F1C302080B
:10FEF800241C002080640208BE1C002012C40208D2
:10FF0800031D002033C40208E31C0020F01C00205D
:10FF18009C3700202DE9FF412C4D2D4C2B7843F0C8
:10FF280001032B70217801F00401C9B211B92948E5
:10FF3800FFF7E4FE284E3378232B21D12378274F6F
:10FF480013F004080AD0224A6FF382031370244B7B
:10FF580020483B600021FFF7B1FE11E0F8F726FECC
:10FF68002B78204A43F006032B701378013BDBB251
:10FF780013701D4A52F823303B60164B83F80080FB
:10FF88003378532B1FD12378052243F004032370C1
:10FF9800104B16491C78013CE4B204EB840000F5D0
:10FFA800CA40843001F0E3FB00201149F8F73AFD1C
:10FFB800FF23002100930134162004220B460191EF
:10FFC800029401F047FCBDE8FF8100BF031D00203B
:10FFD800AB3A0020BE1C0020EC1B0020241C002093
:10FFE8009C640208E31C0020F01C0020B86402088E
:08FFF800AFC302082DE9F0413E
:020000040801F1
:10000000984B04469A7812F0010F00F017811B8874
:10001000002B40F01381944D95F820303F2B40F297
:10002000D780012C14D1914B1B7803F00203DBB273
:10003000002B00F0C48095F820208B4B402A03D180
:10004000013283F82020FBE0482283F82020B6E02C
:10005000022C03D1482385F82030B0E0844E337859
:1000600003F02002D2B28AB195F82020402A0DD1A7
:10007000032C0BD07F4B804A03F1100153F8040B83
:100080008B4242F8040BF9D1412395E003F01003B1
:10009000DBB28BB195F82030412B0DD1032C0BD066
:1000A000764B754A03F1100153F8040B8B4242F86A
:1000B000040BF9D142237FE0F37813F0010F0FD046
:1000C00095F82020422A0BD16D4B6B4A03F11001A9
:1000D00053F8040B8B4242F8040BF9D143236BE035
:1000E00003F00202D2B27AB195F82020432A0BD154
:1000F000644B614A03F1100153F8040B8B4242F840
:10010000040BF9D1442357E003F00402D2B27AB1D0
:1001100095F82020442A0BD15B4B574A03F110017C
:1001200053F8040B8B4242F8040BF9D1452343E00A
:1001300003F00803DBB28BB195F82030452B0DD1CD
:10014000032C0BD0514B4C4A03F1100153F8040B14
:100150008B4242F8040BF9D146232DE00EF0A0F8B3
:10016000A0B14B4B1B788BB195F82030462B0DD1AD
:10017000032C0BD0474B404A03F1100153F8040BFA
:100180008B4242F8040BF9D1472315E0F37803F0D2
:100190004003DBB29BB195F82030472B0FD1032CE5
:1001A0000DD03D4B344A03F1100153F8040B8B4240
:1001B00042F8040BF9D1482385F8203078E095F80F
:1001C00020300133DBB2472B85F820307FF629AF92
:1001D00095F82060472E04D9234B002683F8206031
:1001E00001E00136F6B206F14007FFB212E02B48FB
:1001F000314613F0A8FD08B1032C04D1284B9B5DB8
:1002000023B1032C02D185F820600FE00136F6B24D
:10021000BE4203D03F2EEAD9402E07D1214B1E22E9
:100220001A70402385F82030BDE8F08195F8200051
:100230001149652246F66143F8F744FB012C37D19A
:10024000194B0D4A03F1100153F8040B8B4242F88D
:10025000040BF9D1044B93F820303F2B3CD90020FC
:1002600012493EE0141D0020F40100207F180020F8
:100270009C37002084CA02081B1D0020A5CA020862
:10028000C6CA0208E7CA020808CB020829CB02083E
:10029000083D00204ACB02088CCB02082919002017
:1002A000DF180020C01C0020952B030842CA02085A
:1002B000104BD87800F02000C0B220B1022C06D03C
:1002C00000200D490DE0032C01D10C4909E00C4B35
:1002D00093F820303F2B02D800200A4901E00A4958
:1002E0000020F8F7A3FB1020084A0146BDE8F041C2
:1002F000F8F754BB9C3700205DC1020863CA0208AE
:10030000F401002000CA02086BCB0208141D002073
:1003100010B5F8F74FFC084B1B7803F00403DBB271
:100320002BB106490020BDE81040F8F77FBB022042
:10033000BDE81040FFF762BE7F18002032C80208F7
:1003400070B5224B06461B78214CF3B9257819E08D
:100350002048294613F0F7FC78B123689D4202D962
:10036000FF2E02D007E0FF2E02D19D4208D202E00C
:1003700036B91DB913B9256012E00EB9013500E098
:10038000AD19EDB23F2DE3D90AE0013B202112481F
:1003900010222360F0F702F800201049F8F746FB1E
:1003A0000F48F8F7E9FA46F6614320780D496522CF
:1003B000F8F788FA084D216805F110000131022292
:1003C000F8F75AFB2D23AB7470BD00BFB31C00209F
:1003D000CC1C00202A1C0020F4010020110A030874
:1003E000141D00201B1D0020F8B5544BF02254486A
:1003F0001A700378044613F00E0518D1514A43F0E1
:100400000203156000F8013B13F042FC2C464E4BF2
:10041000E35C1BB14D48214613F07FFC0134402CB6
:10042000F5D14B4B1A7842F001021A70F8BD13F067
:100430000C0543D12E464548294613F084FC08B1EB
:100440000136F6B20135402DF5D11EB9237843F0BF
:10045000040331E000253F482946EFB213F073FC56
:1004600068B1394BEB5C53B13B4B01371F70002037
:10047000FFF766FF237843F00803237002E001359D
:10048000402DE8D1354D3A212846F0F705F838B12E
:10049000401BC0B20130281831460222F8F7ECFAAE
:1004A0002F4B1B78532B47D12B4B00201870FFF795
:1004B00047FF237843F008032370F8BD6FF341032F
:1004C000037003F00403DBB2254D23B1002025495E
:1004D000F8F7ACFA0EE02B78552B01D1FF2002E0A3
:1004E000442B02D10120FFF72BFF13200D211E4AC0
:1004F000F8F754FA2B78232B1ED1227802F002044D
:10050000D4B90F4902F0FB0264F3C3020A700D4A2A
:100510001460F8F74FFB0E4B1A7842F006021A707F
:10052000124A1378013BDBB21370114A52F82320B0
:10053000104B1A60084B1C70F8BD00BF0F1D002047
:10054000291C0020CC1C0020CC2900202A1C0020C3
:10055000031D002080180020B31C0020F40100209F
:10056000EC1B0020571B0308141D0020E31C002077
:10057000F01C0020241C002070B505460C461646D1
:100580003BB143004AF6C52018184018114601F047
:10059000DDF8054B182202FB0535F3092C1906F08E
:1005A0007F066370E67070BD2839002038B510B33F
:1005B000A0F14103DBB2432B1FD9C50900F07F0432
:1005C0000BD0052C19D90021601E0A460AF05EFAEC
:1005D000D0F1010038BF002038BD082C0FD9601EB3
:1005E000C0B229462A4609F0CBFE50B9402C8CBF38
:1005F0000020012038BD012038BD002038BD28462C
:1006000038BD284638BD0000F7B5604C312323744F
:100610005F4F01332376053B637463763B784AF67C
:10062000C5205B00181801F09BF8C0B220F07F02D3
:1006300000F07F01D2B28DF804108DF8002004F193
:10064000120359B9534A04F1150011889278618256
:100650009A7020210222EFF7A1FE0CE0D20904EBF0
:100660008202526A10886082927804F115009A70B2
:100670000222F8F701FA3878400000F52A40C63027
:1006800001F06EF8C0B220F07F0300F07F01DBB212
:100690008DF805108DF801303F4851B93D4B2031A0
:1006A0001A889B786283837002220330EFF776FE0C
:1006B0000BE0DB0904EB83035B6A1A8862839B7897
:1006C000022283700330F8F7D7F9344B1B7813F00C
:1006D000010F5AD0324D02A92A788B1813F8041C46
:1006E00013F8086C2F4B1B78232B04D1002A41D11F
:1006F000223B2B703EE02A2B04D1002A3AD0013A4B
:100700002A7037E0552B46EA010611D10DE02B780F
:1007100002AAD318013E13F8081CF6B23046C909E4
:1007200013F8042CFFF742FF98B9002EEFD121E017
:10073000442B19D115E02B7802A9CB18013613F8F8
:10074000081CF6B23046C90913F8042CFFF72EFF37
:1007500038B1134B3878197832460123FFF70CFF74
:1007600008E0902EE7D905E0532B03D1533B2B70C3
:10077000F9F718FA0C4B1B7803F08003DBB223B1B6
:100780002B782022023304F83320FEBDF401002030
:10079000B31C0020542703080E020020031D002074
:1007A000BE1C0020EC1B00209C37002002480021CA
:1007B0000922EFF7F3BD00BFD11C002070B50A4637
:1007C000002405E01B19811A2A2501345D54E4B286
:1007D0000E4D0F4B295D09B19442F3D1801A0019D7
:1007E00018182021121BEFF7D9FD0A4B1E785EB1B5
:1007F000432E04D10CB1013CE4B200232B5530460A
:10080000F8F7D0F900B12E5570BD00BFD11C002003
:10081000F4010020EC1B002038B5184C184DA078CE
:1008200000F01000C0B250B91649F8F7FFF8FFF712
:10083000BDFF236843F4801323600F232B702A78B5
:100840002AB92368FF2062F31453236038BD0E4891
:10085000C5792DB91C200821FFF7B0FF284638BD07
:1008600023680A496FF3145308222360F0F716F83F
:1008700000280CBF0120FF2038BD00BF9C3700209E
:10088000121D002095C80208D11C0020AC460308A8
:10089000F0B55C4C85B0667806F01006F6B2002E16
:1008A0003ED1594B1A78594B013A53F82230584AE5
:1008B000934204D1574B1A7842F0020207E002F14A
:1008C0001C018B4208D1534B1A7842F004020221DA
:1008D00061F3C7021A7019E03832934216D1FFF75C
:1008E0009BFF002800F08C8001284A4D06D12B7810
:1008F000022243F0010362F3C70306E03046464993
:10090000F8F794F82B7866F3C7032B70434B1A78EB
:1009100042F001021A70236843F4805323606FE0B1
:100920003C4D2B7813F0F80606D03D49002005B069
:10093000BDE8F040F8F77AB813F0070F41D003F0A4
:100940000202D7B24FB1122031460FF073FCFF23E1
:1009500000930196029643202AE003F00406F6B2C3
:10096000A6B1394638460FF065FC202102200EF072
:10097000BFF909F017FB0CF089FEFF2300930197E4
:1009800002974420394604223B4614E013F0010F3D
:1009900013D0012143F61C600FF04CFC3046F5F7F4
:1009A0003BFC204B45201E80FF23009301960296BE
:1009B00031460422334600F051FF00201A49F8F76F
:1009C00035F82B7803F0FA036FF341032B70174BC4
:1009D0001B78232B14D123686FF30C332360F8F7B3
:1009E000E9F80E4B1A7842F006021A70064A13789C
:1009F000013BDBB21370054A52F823200C4B1A60FE
:100A000005B0F0BD9C370020E31C0020F01C002046
:100A1000C0640208984A0020B6C80208031D0020DE
:100A2000F31E0308021C0020D21E0308EC1B00204A
:100A3000241C00201FB50446F5F7DAFCA8B14B20B2
:100A400001F0DAFAFF2300930121FF3B01933920E3
:100A500004220B460134029400F000FF064B0120F3
:100A60005A7842F004025A7004E0044B18880038A7
:100A700018BF012004B010BD983A00202C4D002072
:100A8000F0B51E4E0024337A0546013385B00F467B
:100A9000337210202146012223460094F1F732FEE2
:100AA00045B9FF230093019502974F202946042260
:100AB0002B4609E0012D09D1FF23009301940297F1
:100AC000502021460422234600F0C8FE337A052B2D
:100AD00011D1FA3301210024009327200B46042270
:100AE0000194029400F0BAFE044B1C7205B0BDE8FC
:100AF000F04001F053BA05B0F0BD00BFC21C0020A9
:100B00002DE9F04F974B87B01A78804699461AB175
:100B1000012A40F0E08130E0934B1A68934B9A42EF
:100B200000F0DB81F5F7D6F8914B5B7803F0020318
:100B3000DBB253B98F4B5B7803F08003DBB223B990
:100B400001F052FA08B909F02DFA8B4B1A686FF3CD
:100B500010421A60894B1878F8F724F8002800F042
:100B6000BC81FFF723FE864B3C221A70F7F766FE26
:100B700099F80030013389F80030814B1C787CB93A
:100B8000804B08F101011A78204664F3C30264F334
:100B900004121A70C9B2FFF773FF89F800409CE194
:100BA000794D404609F036FAF7F73CFE00207749C8
:100BB000F7F73CFF764F2B78AA46FB1813F8313C29
:100BC00023B91B200621FFF7F9FD86E16D4A0B21B1
:100BD000137804A8C3F3C004C3F3001603F0F703AB
:100BE0006FF304131370002389F80030062200F01D
:100BF000C8FD2A78394604A8303AEFF7F5FA0746D7
:100C000020B100274FF012093D4629E049F6775000
:100C100000F0A6FD0028F4D05E4D2F72F5F7C2F962
:100C20000446002840F059815B4A4F4B21461A6028
:100C3000FF2300930190029004220820234600F035
:100C40000DFE012223460E2021460094F1F75AFDA5
:100C5000524B1A7842F004021A700123AB713CE146
:100C60004946062204A800F08CFD9AF8002004A84A
:100C70004749303AEFF7B8FA002840F01D8128467E
:100C8000FFF7D8FE002840F02881DFF808B10121E5
:100C90008BF808002846F5F793F98146F5F782F9B5
:100CA000DA46002840F0B18048463D49EFF77AFC2B
:100CB000B0B901F0ABF82C4B14B916B9394A23E09E
:100CC00036B1394A1A60394B1A786FF3410205E0A0
:100CD000374A1A60354B1A7866F341021A70D3E02E
:100CE00048463449EFF75EFC20B148463249EFF7F9
:100CF00059FC58B9002C40F0F080002E40F0ED80F7
:100D000001F084F82D4A184B1A60BDE048462C4982
:100D1000EFF748FC50B949F67550012100F016FD77
:100D2000154A136843F400531360E3E74846254926
:100D3000EFF738FC38B9002C40F0CF80002E40F09F
:100D4000CC80214ADFE748462049EFF72BFC0028FA
:100D500040D1002C40F0C180002E40F0BE801C4AE3
:100D6000D1E700BF201C0020241C002014650208CD
:100D700086310020A73A00209C370020EC1B002081
:100D8000121D0020D01C0020081C00203CC10208BD
:100D9000D11C0020C21C0020306502081D25002047
:100DA000214803087C67020804690208031D00202B
:100DB00020690208B1470308F74903083C690208A3
:100DC000EC470308EE47030874690208B4490308B6
:100DD000C869020848464249EFF7E4FB002853D1AE
:100DE00001F014F83CB13F4A3F4B1A603F4B1A7870
:100DF0006FF3410270E0002E6FD03D4A3A4B1A600B
:100E00003A4B1A7864F3410266E048463449EFF7FA
:100E1000C9FB064620B900F0F9FF002C5DD01BE0AD
:100E200048463449EFF7BEFB002856D048463249C1
:100E3000EFF7B8FB38B9002C4FD1304A2A4B8BF86A
:100E400007501A6049E048462D49EFF7ABFB0646CC
:100E500050B9A4B100F0DAFF224A234B1A60234BA9
:100E60001A7866F3410237E048462649EFF79AFBC5
:100E700020B148462449EFF795FB00B96CBB234AE3
:100E8000194B1A6000F0C2FF07F56A5079308AF8F2
:100E9000075000F065FC8AF800009AF8070000F59A
:100EA000D640353000F05CFC8AF801001848F5F7B0
:100EB000CBF9402D11D107E00135EDB20137402DBE
:100EC00009F107097FF4CCAE08F101010020C9B295
:100ED000FFF7D6FD01E000221A7007B0BDE8F08FE1
:100EE000F047030820690208241C0020031D00208D
:100EF00004690208EE470308B4490308C8690208F8
:100F000021480308B1470308EC470308E4690208D5
:100F1000C21C002010B52148214903680A789C7B37
:100F2000944203D99C8914F0200F18D09A8912F0AA
:100F3000800F01D105E01C3B9A8912F0400FFAD0D6
:100F400000E01C33036000230B7003689B8913F0DF
:100F5000200F16D0134BDA79114B1A7011E00132C1
:100F6000D2B20A70986843F60653984209D101E05C
:100F70000132D2B2162A03D80B4853B29840F7D4A4
:100F80000A700A4A136843F480731360F7F756FC3B
:100F9000074B1A7842F006021A7010BD241C00207C
:100FA000B31C0020C21C0020000600889C370020D3
:100FB000031D002010B52349234A0B78D3B11068D4
:100FC000848914F0200F15D1013BDBB20B708468CB
:100FD00043F60652944228D104E013B1013BDBB240
:100FE00000E0837B162B03D8184C5AB29440F4D4FB
:100FF0000B701AE01368988910F0400F01D106E0D9
:101000001C33988910F0800FFAD0136002E00E486C
:101010001C3B036013689A7B0A709B8913F0200FB6
:1010200003D00B4BDA79074B1A700A4A136843F462
:1010300080731360F7F702FC074B1A7842F0060240
:101040001A7010BDB31C0020241C0020000600886C
:10105000C21C00209C370020031D0020084B1A688A
:10106000084B9A4204D003F580630C339A4205D1B1
:10107000054B1878003818BF0120704700207047D2
:10108000241C0020146502087E180020074B084A23
:101090001B68934202D03832934205D1054B187831
:1010A000003818BF0120704700207047241C002022
:1010B000C86902087E1800202DE9F04F7F4B804D53
:1010C0001970A0F11103DBB2012B87B00E46287016
:1010D00006D8122801D1113800E00020F5F7FAF8FF
:1010E0002B78522B0DD1F2F727F828B9F2F718F820
:1010F00010B9F2F739F820B1724B1A7842F00802B1
:101100001A70714B714C1B78002B2DD12168704ADD
:10111000914229D06F4A236013706F4A6F4811784B
:10112000037063F3C30163F3000163F307111170EC
:101130006B4A117863F3010111706A4A117863F305
:10114000C5011170684A1370684A117863F3410150
:1011500063F3000163F382011170654A116863F360
:101160000C311160634A13702368002B40F05681E4
:101170005F4F7B7803F02003DBB273B15E4B93F8D3
:101180000080B8F1000F08D149F67550414600F0D3
:10119000DDFA3B6868F34D333B60584B187810F02C
:1011A0001E0002D00020564907E0564B93F80480F9
:1011B0009946B8F1000F05D0534907B0BDE8F04F8C
:1011C000F7F734BC514F97F801B0BA46BBF1000FA6
:1011D0002DD0BBF1070F15D94D48F7F7CDFB4D4981
:1011E000B878652246F66153F7F76CFB3878072329
:1011F00010F003007B700EBF474940464749F7F7A0
:1012000015FC0CE0BBF1020F09D84148437823B12B
:10121000F7F7B2FB87F8018078E202237B70102099
:101220003B4A014607B0BDE8F04FF7F7B7BB3C4F6C
:10123000BB795BB187F806B000F0F6FB8E2059460B
:1012400001225B46CDF800B0F1F75CFA0020F2F71E
:10125000C7F8214A1F491378324843F00603137038
:1012600000230B70304923600B7089F80130037044
:10127000183303FB06FC2D49934611F80CC0884631
:101280001CF0080F04D130460593FFF739FC059B8D
:1012900003FB06835B7913F0100F04D02A78133A0E
:1012A000D2B2032A46D913F0200F79D02B78442BE1
:1012B00040D03DD8232B3DD02A2B3AE0B61C00204D
:1012C000EC1B0020D11800200F1D0020241C002042
:1012D00064640208E31C0020031D0020BE1C0020E3
:1012E000051C0020B91C0020C11C0020D01C0020BF
:1012F0009C3700200E1D00207E180020154D002078
:101300009FC102089711002030F10208BB1C002089
:10131000141D00201B1D0020A7C2020886C202085F
:10132000C21C0020B81C0020B31C0020283900205B
:10133000552B35D1794B1B78002B31D1784B93F855
:101340000080B8F1000F2BD143F6DB2000F008FA43
:10135000012825D13F23FB7189F8010043F638307D
:1013600000F0FEF93870F87900F5D640353000F01D
:10137000F7F978706B48F4F767FF9BF80030304658
:1013800068F341038BF8003008F044FEF7F712FCD5
:10139000654B66482360664BC3F800802B7803706A
:1013A0002B78432B0AD15E4B1B783BB9013389F86C
:1013B0000130604B3046236008F02CFE2878173847
:1013C000C3B2072B00F2A2815B49FF220AF0B4FBF3
:1013D0009AF80010594B60F301018AF8001001F0EF
:1013E0000301022900F092810122032041B1009003
:1013F00001929B7868309B1802930021033206E02B
:10140000009001929B786C200133029304220B46DA
:1014100000F024FAFF238AF8013077E1454A93422D
:1014200050D12878A0F14303DAB2122A22D8444AD4
:101430005BB29A401ED5432840F06881374B1B7839
:10144000002B40F0638100F0EBFC3E4B48B11A7872
:1014500003201109013191FBF0F000EB4000091A63
:1014600004E01A781109013101F0070161F3071254
:101470001A704BE1F7F796FB002823D0314F3A78EA
:1014800012F0F00308D163F307123A7023602E4B79
:101490001A7842F008020EE0102B13D100F0C0FCC5
:1014A00080B13B786FF307133B7000232360264B1A
:1014B0001A7842F0100230461A7007B0BDE8F04FBB
:1014C000FFF71EBB214B1E211A781E4E61F3460208
:1014D0001A70337813F0010F134B3DD022689A42F3
:1014E0000CD0A3F5B0639A4208D0FFF7B7FD28B936
:1014F000FFF7CCFD10B9AA30F1F772FF2268144B48
:101500009A4202D10020F1F76BFF2B78522B40F06A
:10151000C280104B53221A70BDE000BF7E1800201D
:10152000201C0020C21C0020E4690208B81C002016
:10153000F01C002014650208BD1C0020BB1C00200C
:10154000002000C0031D0020D01C0020811D0020B1
:101550001C6A0208EC1B002022689A420CD0A3F5FA
:10156000B0639A4208D0FFF779FD28B9FFF78EFDE6
:1015700010B9AA30F1F734FF2B78552B1ED1FFF7A5
:1015800019FD3378634843F0060333708378624F64
:1015900003F00203DBB24BB1F7F7EEF923681868EA
:1015A000FAF750FB3B786FF341033B705B4883785D
:1015B00003F00203DBB20BB1F7F7DEF92B78442B13
:1015C0001ED1FFF7A7FC3378524843F0060333706F
:1015D0008378514F03F00203DBB24BB1F7F7CCF93C
:1015E00023681868FAF72EFB3B786FF341033B70D2
:1015F0004A48837803F00203DBB20BB1F7F7BCF97A
:101600002B78522B09D13378002243F00103337039
:10161000434B1A70434B45321A70434B00271F70DF
:101620002B78232B37D1414B3A481F70404B1F700A
:10163000F7F7A2F93948F7F79FF933783D4943F0B6
:10164000060333700B78344AFBB13B4A013B1770F9
:101650003A4ADBB20B7052F82330394A23609B6858
:10166000934202D109F016FD15E002F5D2718B42CA
:1016700004D10120014606F097FE0CE002F50C7241
:10168000934208D12F4B1F7005E0117863F30711C7
:10169000117023603AE02C4B5B7813B10020F1F716
:1016A0009FFE23681F7B17F00F0702D1FBF7AEFCEC
:1016B0001BE0012F02D1F8F723FC16E0022F02D124
:1016C000F9F78CFB11E0082F05D84FF09C53BB4075
:1016D00001D5F9F733FE042F03D123689B6998479E
:1016E00003E0052F01D1F9F7F9F8337803F002038D
:1016F000DBB21BB123681868FAF7A4FA33786FF3EA
:10170000410333702B780BB1074A137007B0BDE863
:10171000F08F00BF141D0020031D0020341C00208A
:10172000BE1C0020EC1B0020061C0020C11C002059
:101730000E1D0020E31C0020B31C0020F01C002024
:10174000386A0208331C00209711002007B502AB4D
:1017500003F8011D19460122002305F0F7FA0EBD1A
:1017600007B5002302A901F8013D012205F056FB4F
:101770009DF807000EBD08B5002305F0E7FA00202C
:1017800008BD034610B508461446194605F046FB49
:10179000E0B210BD10B50346002484540846194633
:1017A00005F03CFB204610BD37B50546002400E09F
:1017B0001446012260190DF1070105F02FFB9DF879
:1017C0000730621C203BDBB25A2BF1D920463EBDCC
:1017D000F8B500252C461E4B1C21585D01FB043139
:1017E000400000F574506230043102220134FFF7EA
:1017F000C2FF1C355C2CEED143F6C13420B204226A
:1018000005341449FFF7B7FFA4B243F6E9339C420D
:10181000F4D1002549F274372C4615E007EB460059
:1018200004EB440100B259180222FFF7A4FF01366D
:10183000F6B2094B5A199278B242EFD80134803788
:101840000335142CBFB201D00026F2E7F8BD00BF6B
:1018500070950208B3470308809F02082DE9F347FB
:10186000044615468A46022243F61A610DF1060027
:101870001E46BDF930909DF828809DF82C70FFF72A
:1018800080FF2F4B2F499A78BDF906008A705A784D
:1018900000EBC000CA701A7900F578500A715A79C5
:1018A0001C304A719A791B7845EAC6158A710C700A
:1018B00081F80190CB710D7200B20922FFF75BFF36
:1018C0001EB1214B1A8801321A80BDF8063001334F
:1018D0009BB2B3F57A7FADF8063002D30023ADF8A2
:1018E000063002220DF1060143F61A60FFF743FFAE
:1018F000BDF80600154B188000B200EBC00000F5E3
:10190000785000F11C05243000B2FFF729FF10F0D9
:10191000800F03D00C4B1A88013A1A8028B200219C
:10192000FFF714FF0A4B03F8148003EB44046770BD
:10193000BAF1000F02D00120F4F76EFCBDE8FC877D
:10194000A04A0020DA1C0020021C00208431002064
:101950001F2F00202DE9F743324B1D78303DEDB2AB
:10196000C5F10606F6B23EB305F11207402413E0B6
:1019700008F101080FFA89F000215FFA88F8FFF7F3
:10198000E5FE09F10109B0451FFA89F9F0D1013CE2
:101990000737E4B2BFB21CB1B9464FF00008E7E721
:1019A0000B35013428B20021E4B20135FFF7CEFE39
:1019B000B442ADB2F5D132E0122425B268462946D0
:1019C0000622FFF7DEFE9DF8003043B19DF805309A
:1019D0002BB99DF803308DF804308DF805300734AD
:1019E000062228466946A4B2FFF7C5FEB4F5E97F92
:1019F000E3D168460B210622FFF7C3FE9DF80030B5
:101A000043B19DF805302BB99DF803308DF80430B3
:101A10008DF805300B2069460622FFF7ACFEBDE8C5
:101A2000FE8300BF081C002070B509F033FB0BF0EB
:101A3000CFFE05F0D7FE05F0FDFDF1F737FF9F481B
:101A4000F4F71CFC43F6D120FFF78AFE9C4B9D4C1B
:101A5000187043F6D020FFF783FE9B4B187043F6B7
:101A6000DC20FFF77DFE994B187043F60450FFF71A
:101A700077FE974B187043F60550FFF771FE954BB4
:101A8000187043F6DA20FFF76BFE934B187043F69D
:101A9000D920FFF765FE914B187043F6CF20FFF772
:101AA0005FFE8F4B187043F6CC20FFF759FE8D4B2D
:101AB000187043F6D220FFF753FE8B4B187043F695
:101AC000DD20FFF74DFE237801280CBF43F0010312
:101AD0006FF30003237043F6E020FFF741FE237805
:101AE00001280CBF43F080036FF3C713237043F644
:101AF000E720FFF735FE7D4B01281A6843F6ED20FD
:101B00000CBF42F000526FF35D721A60FFF728FEBF
:101B1000774B18B91A7860F3000202E01A7842F0A5
:101B200001021A7043F6EA20FFF71AFE63780128D3
:101B30000CBF43F001036FF30003637043F66E21A3
:101B400011226C48FFF71DFE6B4800210322EEF7BF
:101B500025FC00246748235C312B03D12230214629
:101B600012F0DBF80134112CF4D1224643F6F611C1
:101B70006048FFF706FE224643F63A215F48FFF72A
:101B800000FE0CF0CDFFF4F785FE43F6E120FFF7F1
:101B9000E7FD5B4C237860F30003237043F6E220FB
:101BA000FFF7DEFD237860F34103237043F6E42062
:101BB000FFF7D6FD237860F3C303237043F6E620D6
:101BC000FFF7CEFD237860F34513237043F6E92039
:101BD000FFF7C6FD237860F38613237043F6E520F4
:101BE000FFF7BEFD237860F30413237043F6EB2068
:101BF000FFF7B6FD237860F3C713237043F6F72091
